:10000000005600203165000081640000916400000A
:10001000A9640000C1640000D96400000000000071
:10002000000000000000000000000000F16400007B
:10003000016500000000000011650000216500005E
:10004000696400000000000000000000B10B010026
:10005000E10A01005D0B010000000000000000004B
:1000600091430000A9EF000089EF0000F90B0100A7
:10007000000000000000000000000000190C01005A
:100080002DE9F843054688464FF0A0441C4EDFF8A2
:1000900078901C4F237E002BFCD1A37E2BB94FF010
:1000A00001022274A37E002BFBD072B6735DF3B9FC
:1000B00000F02EF8C0B90122D9F8103043F0040343
:1000C000C9F8103087F83220BFF34F8F00BF30BF20
:1000D00087F83200D9F8103023F00403C9F8103043
:1000E000BFF34F8F62B6D5E700BF30BFFAE70023FA
:1000F0007355B8F1000F00D0C04762B6BDE8F88371
:10010000982800200000105000ED00E000000000E2
:100110005FF800F0D9420000FFFFFFFFFFFFFFFF85
:10012000FFFFFFFFFFFFFFFFFFFFFFFFFFFFFFFFDF
:10013000FFFFFFFFFFFFFFFFFFFFFFFFFFFFFFFFCF
:10014000FFFFFFFFFFFFFFFFFFFFFFFFFFFFFFFFBF
:10015000FFFFFFFFFFFFFFFFFFFFFFFFFFFFFFFFAF
:10016000FFFFFFFFFFFFFFFFFFFFFFFFFFFFFFFF9F
:10017000FFFFFFFFFFFFFFFFFFFFFFFFFFFFFFFF8F
:10018000FFFFFFFFFFFFFFFFFFFFFFFFFFFFFFFF7F
:10019000FFFFFFFFFFFFFFFFFFFFFFFFFFFFFFFF6F
:1001A000FFFFFFFFFFFFFFFFFFFFFFFFFFFFFFFF5F
:1001B000FFFFFFFFFFFFFFFFFFFFFFFFFFFFFFFF4F
:1001C000FFFFFFFFFFFFFFFFFFFFFFFFFFFFFFFF3F
:1001D000FFFFFFFFFFFFFFFFFFFFFFFFFFFFFFFF2F
:1001E000FFFFFFFFFFFFFFFFFFFFFFFFFFFFFFFF1F
:1001F000FFFFFFFFFFFFFFFFFFFFFFFFFFFFFFFF0F
:10020000FFFFFFFFFFFFFFFFFFFFFFFFFFFFFFFFFE
:10021000FFFFFFFFFFFFFFFFFFFFFFFFFFFFFFFFEE
:10022000FFFFFFFFFFFFFFFFFFFFFFFFFFFFFFFFDE
:10023000FFFFFFFFFFFFFFFFFFFFFFFFFFFFFFFFCE
:10024000FFFFFFFFFFFFFFFFFFFFFFFFFFFFFFFFBE
:10025000FFFFFFFFFFFFFFFFFFFFFFFFFFFFFFFFAE
:10026000FFFFFFFFFFFFFFFFFFFFFFFFFFFFFFFF9E
:10027000FFFFFFFFFFFFFFFFFFFFFFFFFFFFFFFF8E
:10028000704700BF034613F8012B002AFBD1181A50
:100290000138704700487047CCDF010024207047C8
:1002A0000620704708B506F05DF808BD08B506F0F1
:1002B000D7F843690148984708BD00BFCCDF01006B
:1002C00010B50C4611461A46012807D010B1022875
:1002D0000BD010BDE0B200F047F8FAE7BDF80830E7
:1002E000C9B2E0B200F082F8F3E7E0B200F046F9FC
:1002F000EFE700BF054B00229A80DA805A819A818D
:10030000B42119811A765A769A767047A42900206A
:10031000014B1878704700BFA429002010B4044690
:10032000034B0FCB84E80F00204610BC704700BF82
:10033000A82900200346054901F114024869186004
:10034000098B927999809A7118467047A4290020E8
:10035000044B187E012803D0987E003018BF01207E
:10036000704700BFA429002010B504461D4B1B7820
:1003700013F0030F02D010F00C0F15D114F0030F7F
:100380001CD113F0080F02D014F0040F22D113F087
:10039000040F15D014F0080F12D0124B00229A80CF
:1003A000DA80B4221A810BE005F0DCFF02690D4B04
:1003B0001A61FFF79FFF00F019F901E0FFF79AFFBC
:1003C000084B1C70084C204600F090FE204600F0C0
:1003D0003DFB10BD034B00229A80DA80B4221A81C3
:1003E000EEE700BFA4290020D4DF010010B50446C9
:1003F00000F0A4FF042C00D010BDFFF789FF10F01F
:100400000C0F05D000F0A3FF0368984700F0F8F840
:10041000564C204600F0B8FE204600F0BDFB544B81
:100420001A78042A30D0082A46D0514B5B89B3F59C
:10043000616F05D34E4B0021598199890131998112
:100440004B4B99894EF66023994250D0484BD9883E
:100450004EF6602399424ED0454B99884EF6602364
:1004600099424CD012F0080F4DD1414B1B8BB3F584
:10047000807F76D03E4B9B7E13B1013B3C4A937606
:100480003B4B1A7E5A76B7E73949CB8801339BB28A
:10049000CB803849A1FB0301490901EB8101A3EBA2
:1004A000C1039BB2002BC0D1314B59890131598115
:1004B000196901311961B8E72D490B89013B0B819D
:1004C0008B8801339BB28B802B49A1FB0301490927
:1004D000C1EB0111A3EB81039BB2002BA5D1244BEF
:1004E0005989013159811969013119619DE7204B01
:1004F00000219981AAE71E4B0021D980ACE71C4B53
:1005000000219980AEE700F022FF03689847036856
:10051000984760B9164B1B7813F0080FA5D0134805
:1005200000F06CFE78B1124BB4221A819DE700F006
:100530000EFF0368984700F0B2FD0128EAD10C4B8A
:10054000B4221A81E6E70A4B1B7813F0080F8CD00F
:10055000074B1B89002B88D105F082FF0368984761
:1005600083E7034B06229A768AE700BFD4DF0100B7
:10057000A4290020CDCCCCCC8988888810B5072848
:1005800019D8DFE800F019041D201823262C05F0E7
:10059000E9FE044605F064FFC3684FF48062002161
:1005A00020469847FFF7A6FE0E4800F09FFD04F195
:1005B000F00000F038FA10BD0A4800F0BBFDFAE781
:1005C000094B1975F7E7084B5975F4E7064B997510
:1005D000F1E7054BD975034800F088FDEBE7024BC6
:1005E0001976E8E7D4DF0100A429002008B58022AD
:1005F0000021024819F085FB08BD00BFC02900207A
:100600002DE9F04F85B082460022924911F8323030
:100610006FF3C71301F8323001EBC20358786FF360
:10062000C710587098786FF3C7109870D8786FF328
:10063000C710D87018796FF3C710187158796FF315
:10064000C710587198796FF3C7109871D8796FF304
:10065000C710D8710132102AD8D1DAF80030984783
:1006600003900023029345E04FF001084FF0140C73
:10067000B5423AD801974FF04C0933464646984662
:100680002BE04FF001084FF0140CF1E7425C42F010
:100690008002425402F07F0202EB0C0BBBF14C0FC4
:1006A0000FDD425C69F30602425401339BB29C4267
:1006B0000FD319461EF80320D209E7D0002EF4D03C
:1006C000E4E7624410F801B062F3060B00F801B0F1
:1006D000EBE70135ADB2A84507D3A742F9D8019B96
:1006E0005C4A02EBC50E7046E3E7029B01330293BE
:1006F0000A2B66D09DF80880DAF8283040469847E3
:10070000012805D0DAF82830404698470228ECD175
:10071000DAF80C30404698478146DAF81030404607
:100720009847834603014C4A82FB0326F218DE17E2
:10073000C6EBE2264FEAC903484A82FB03271F445F
:10074000DB17C3EBA727DAF8183040469847DAF8EA
:10075000083040469847002814BF10240424B6B23D
:10076000351B25EAE575ADB226440F2EA8BF0F262E
:10077000B6B2BBB21F1B27EAE777BFB21C44072CF7
:10078000A8BF0724A4B2DAF8083040469847A9F178
:1007900043091FFA89F940F2B23399453FF664AF35
:1007A000BBF16E0F7FF66DAF002814BF4FF0140C35
:1007B0004FF0010C002814BF4FF001084FF0000863
:1007C00056E70026234F1FE0043AE55C62F3060576
:1007D000E55404E0013AE55C62F30605E5540133B3
:1007E000082B0ED0C25CD209F9D1C25C02F07F02A4
:1007F000122AEFD8032AE7D8E25C6FF30602E2542C
:10080000EDE70136102E04D0002307EBC6000446A6
:10081000E8E7039B1BB1002421460E4D05E0FFF7DE
:10082000E5FEF8E70134102C0DD0002305EBC400E1
:10083000C25C02F07F02092A84BF013189B2013310
:10084000082BF5D1EEE7034BA3F8801005B0BDE807
:10085000F08F00BFC0290020E1000EE049D6B9F2B8
:100860002DE9F04F83B0064601911446036898477E
:1008700070B13E4A92F88230013382F88230A1464C
:10088000002C5ED00027B8469346DFF8E8A037E09A
:10089000FFF7ACFE4FF00008019B83F8008055E0A5
:1008A000F3682046984740B333692046984720B301
:1008B000F36820469847054633692046984700016B
:1008C0008AFB00230344C017C0EBE32080B2ED0095
:1008D000274B83FB05232B44ED17C5EBA325ADB2B6
:1008E0000BEBC000435D03F07F03122B05D808F12A
:1008F00001085FFA88F8019B1C7001374F4510D042
:10090000FCB2B36A204698470128C9D0B36A204692
:1009100098470228C4D0B36A204698470328ECD1F0
:10092000BEE7B8F1000F0CD0104BB3F88030402B6D
:1009300010D8B8F1010F09D012D90023019A137011
:1009400004E04FF00008019B83F80080404603B0AC
:10095000BDE8F08F4FF00008019B83F80080F5E7B9
:100960004FF00008019B83F80080EFE7C0290020CA
:1009700049D6B9F2E1000EE0431E9BB24FF6FD727C
:1009800093421CD84B1E9BB293421AD809010E4BBE
:1009900083FB01231944C1F3CF21C0000B4B83FB20
:1009A00000231844C0F38F20094B03EBC101085CFE
:1009B00000F07F0013288CBF002001207047012029
:1009C00070470120704700BFE1000EE049D6B9F240
:1009D000C0290020F8B506460F4C2568238903EB93
:1009E00083035B00F4336B8005F03AFD0435238903
:1009F00003EB830307690A22314605EB4300B8473E
:100A0000238901339BB22381226852789A4201D80C
:100A100000222281F8BD00BF442A0020704708B59B
:100A2000FFF7D8FF08BD10B5044605F019FDC368EF
:100A30004FF44472002120469847034B1C60462324
:100A400063700A23237010BD442A002030B5A5B07E
:100A50000446436898474F4B1B7913F0030F09D0A6
:100A6000A368984710F0080F21D1A368984710F0A9
:100A7000040F1CD1474B1B7913F00C0F09D0A3684E
:100A8000984710F0020F41D1A368984710F0010F6A
:100A90003CD1A36898473F4D2871E36804A8984764
:100AA000BDF81830EB8000236B8125B030BD0025E8
:100AB00001950295ADF80C5005F0D2FCC3680A22EE
:100AC000294601A898479DF80430022262F30203E8
:100AD0008DF80430E36810A89847BDF80430BDF8DD
:100AE000462062F30F13ADF80430E3680CA8984772
:100AF000BDF83E30ADF80630E36808A898470B9B78
:100B0000ADF8083001A8FFF765FFB3E700250195B0
:100B10000295ADF80C5005F0A3FCC3680A222946E3
:100B200001A898479DF80430032262F302038DF870
:100B3000043063689847BDF80430028862F30B13F1
:100B4000ADF80430134A52891209C3F3072362F344
:100B500007138DF80530E36820A89847BDF8823068
:100B6000ADF80630E3681CA89847BDF87030ADF8C2
:100B70000830E36818A89847BDF86E30ADF80A3021
:100B8000E36814A89847179BADF80C3001A8FFF74D
:100B900021FF7EE7442A00202DE9F04FA9B004464A
:100BA00043689847A368984710F0080F04D1A368DA
:100BB000984710F0040F39D0236898470368984786
:100BC000054600F06CFA80B123689847036898479F
:100BD0008146002704970597ADF8187002460A2150
:100BE00004A800F048FAB846EEE0284600F05BFAA8
:100BF0000028E9D163689847B0F86030002B40F0D6
:100C00007381B84BDD880135E36818A89847BDF8B3
:100C100068309D4200F0D781E3680EA89847B14B39
:100C2000BDF84020DA805A8901325A8129B0BDE8E6
:100C3000F08FF36828469847336928469847236819
:100C4000984703689847834600F035FAB0F1000AE8
:100C5000C0F2448163689847C388ADF80830636880
:100C600098470389ADF80A30636898474388BDF810
:100C700008201344ADF80C30636898478388BDF8AA
:100C80000A201344ADF80E305FFA8AFADBF80C3014
:100C9000504698470190DBF810305046984702AA1A
:100CA0000146019800F0C0F9002840F019814FF486
:100CB000C973ADF8083040F66A03ADF80A3040F267
:100CC000A623ADF80C3040F62413ADF80E30DBF857
:100CD0000C30504698470190DBF81030504698474A
:100CE00002AA0146019800F09FF9003018BF0120C8
:100CF0009DF8223060F345138DF8223063689847E1
:100D000090F86330C3F302039DF8242063F30202DA
:100D10008DF824206368984790F866A00AF0FD0AD1
:100D20006369984701280ED14AF0020A6368984720
:100D300090F86830FF2B06D06368984790F86830C9
:100D4000013380F868306368984780F866A063686C
:100D50009847BDF8243090F8662062F3C803ADF8D8
:100D60002430B368284698479DF8253060F3820305
:100D70008DF82530B369284698471F2828BF1F20C3
:100D8000BDF8223060F38A13ADF82230F3692846AB
:100D900098471F2828BF1F209DF8233060F3C70302
:100DA0008DF82330336A28469847C0F38F001F28F8
:100DB00028BF1F209DF8253060F3C7038DF825302C
:100DC00007A8FFF707FE0137D9F800309847FBB2B4
:100DD0008342BFF40FAFFBB228AA134413F8905C10
:100DE000CDF81C80CDF82080ADF82480D9F82830CB
:100DF00028469847012805D0D9F828302846984732
:100E00000328E0D123689847036898470646E368BB
:100E10000AA89847BDF82CA005F022FBC3680A2257
:100E2000414607A898479DF81C306FF302038DF8E0
:100E30001C30B36A28469847012814BF00200120BF
:100E40009DF81C3060F3C3038DF81C30BDF81C30D6
:100E5000BDF82E2062F30F13ADF81C304FEA1A12C2
:100E60009DF81E3062F303038DF81E309DF820308C
:100E70006AF303038DF82030F36828469847BDF8DD
:100E80001E3060F30F13ADF81E30336928469847C3
:100E9000BDF8203060F30F13ADF82030236912A89D
:100EA00098479DF822309DF8482062F301038DF8A1
:100EB0002230736A284698479DF8223060F38303F6
:100EC0008DF8223003F00C030C2B7FF4B2AE9DF8AA
:100ED000223043F00C038DF82230AAE6404607E7A3
:100EE000012005E7442A002000230A930B93ADF864
:100EF00030302368984703689847064600F0DBF8CF
:100F0000051E4FDB05F0ACFAC3680A2200210AA8CF
:100F100098479DF82830012262F302038DF82830AB
:100F2000E36814A89847BDF82830BDF8562062F34E
:100F30000F13ADF828306368984790F8603013F0CD
:100F4000020F3AD16368984790F8603013F0040FAD
:100F500035D16368984790F8603013F0080F30D1AE
:100F60006368984790F8603013F0100F14BF0622A2
:100F700000229DF82A3062F303038DF82A30EDB287
:100F8000F36828469847BDF82A3060F30F13ADF890
:100F90002A30336928469847BDF82C3060F30F1388
:100FA000ADF82C300AA8FFF715FD636898470023B9
:100FB000A0F860301B4A538123E60122D9E70422BE
:100FC000D7E70522D5E700250A950B95ADF83050F7
:100FD00005F046FAC3680A2229460AA898479DF8F0
:100FE0002830042262F302038DF82830E36824A835
:100FF0009847BDF82830BDF8962062F30F13ADF87E
:101000002830E36820A89847BDF88E30ADF82A3024
:10101000E3681CA898471F9BADF82C300AA8FFF77F
:10102000D9FCF9E5442A0020134672B112888242A5
:101030000DD89A8882420CD3DA888A420BD358881A
:1010400088428CBF0020012070470020704700209C
:101050007047002070470020704710B504460846CE
:1010600011460023224600F0B3F90021204600F08B
:10107000DCF9C0B210BD08B5002300F0A9F908BD25
:1010800008B500F0A5F908BD08B5002100F0CDF9BC
:10109000C0B208BD08B500F0C8F9C0B208BD08B5B7
:1010A00000F06EF908BD08B500F07EF908BD08B57E
:1010B00000F052F908BD08B500F0DEF908BD0000E7
:1010C00010B5436898470488003418BF012405F020
:1010D000C7F98368224603210220984705F0C0F92A
:1010E0008368224603210420984710BDF8B50746BF
:1010F0000F4B1B68BBB1002425460D4E56F825301A
:1011000053B156F82530984703682BB156F825306F
:1011100098470368384698470134E4B2254656F8A4
:101120002430002BEAD13846FFF7CAFFF8BD00BFD4
:101130001C120020F8B50746124B1B68F3B10024BF
:101140002546104E56F825308BB156F82530984775
:1011500043683846984750B156F825309847C368D9
:101160002BB156F825309847C36838469847013464
:10117000E4B2254656F82430002BE3D13846FFF779
:101180009FFFF8BD1C1200202DE9F04107461A4BC5
:101190001B68002B2DD000242646174D05E0013496
:1011A000E4B2264655F824301BB355F82630002B00
:1011B000F5D055F8263098474368384698470028B8
:1011C000EDD055F82630984790F81480BB689847C2
:1011D00018EA000FE3D055F8263098478368002BB3
:1011E000DDD055F826309847836838469847002860
:1011F000D5D0BDE8F08100BF1C1200202DE9F041E0
:1012000007461C4B1B68002B32D000242646194D84
:1012100005E00134E4B2264655F824302BB355F8E6
:101220002630002BF5D055F82630984743683846CD
:1012300098470028EDD055F82630984790F814804C
:10124000BB68984718EA000FE3D055F82630984756
:101250000369002BDDD055F82630984703693846DE
:1012600098470028D5D0012000E00020BDE8F0819B
:101270000020FBE71C12002008B54368984700785F
:10128000C0F3400008BD704730B587B0044603681E
:1012900098470368984702461F4903A800F0E1FCFD
:1012A0009DF8153013F0020F2ED0BDF80C30CD3B59
:1012B0009BB240F29D22934229D8BDF80E2040F601
:1012C0007B039A4225D99DF81430043BDBB2382BBE
:1012D00001D9002019E00023019302934FF002038B
:1012E000012565F387138DF8043005F0B9F84368DC
:1012F00001A898476368984790F8603043F002036C
:1013000080F86030284600E0002007B030BD0020A3
:10131000FBE70020F9E700BF502A002008B54FF492
:101320009F7354224021024800F086FC08BD00BF94
:10133000502A002000487047ECDF010008B5022861
:1013400000D008BD1946104600F04AFDF9E70148F3
:10135000704700BF04E0010038B5054603689847B0
:1013600048B10024AB68E0B29847034630B9013475
:101370000A2CF7D100E00023184638BD0123FBE713
:1013800038B505460368984750B10024AB6AE0B20F
:101390009847012806D001340A2CF7D1002000E03C
:1013A000002038BD0120FCE738B5054603689847A2
:1013B00050B10024AB6AE0B29847032806D001344C
:1013C0000A2CF7D1002000E0002038BD0120FCE706
:1013D0002DE9F84F824689461646984600252F4645
:1013E00009E07B1CDBB20AF807404B451BD01F46C7
:1013F00001350A2D17D0ECB2B36A20469847002871
:10140000F6D0F368204698478346336920469847CC
:10141000B8F1000FE5D0424601465846FFF704FEFA
:101420000028DED1E4E7BDE8F88F2DE9F843074650
:1014300088460024264604E00136F6B201340A2C20
:1014400017D0E5B2BB6A284698470028F6D0FB685B
:101450002846984781463B6928469847B8F1000FCF
:10146000EAD0424601464846FFF7DEFD0028E3D1B8
:10147000E4E770B2BDE8F88338B5054603689847DD
:1014800060B10024AB6AE0B2984728B901340A2C55
:10149000F8D14FF0FF3038BD60B2FCE74FF0FF30BD
:1014A000F9E7000008B5436898470078C0F3C0002A
:1014B00008BD064B43221A80BE225A8040F2F53204
:1014C0009A8040F6B502DA80704700BF6C2A00208F
:1014D000F0B585B0044643699847244DA876236843
:1014E000984703689847024605F1080102A800F0F2
:1014F00078FA9DF80830022B03D00025284605B065
:10150000F0BDBDF80A70BDF80C602A463146384679
:10151000FFF78AFD05460028F0D0002300930193D1
:101520004FF00203042262F38503012565F387135C
:101530008DF8003047FA02F38DF8023046FA02F3D4
:101540008DF8033006F00F0646EA07168DF80460A2
:1015500004F086FF4368684698476368984790F8A8
:10156000603043F0080380F86030C7E76C2A002041
:1015700010B584B00D4C46230393642302931E23BD
:101580000193032200921223012104F1080000F0CC
:1015900001FA43232380BE23638040F2F533A38006
:1015A00040F6B503E38004B010BD00BF6C2A0020F4
:1015B0000048704708E0010008B543689847037881
:1015C00013F0240F14BF0120002008BD38B5436874
:1015D0009847C58804894188294482882244034B5E
:1015E0005D809C80D9801A8138BD00BFA42A00206C
:1015F0002DE9F04784B08046436898470378C3F3E9
:101600008009C3F34017D8F8143098473F4D85F848
:101610002600D8F80030984703689847024605F13D
:10162000140102A800F0DDF99DF808A0BDF80A60D9
:10163000BDF80C40AA1C21463046FFF7F5FC30BB34
:1016400005F10A0221463046FFF7EEFC034600286A
:101650005AD1184604B0BDE8F0872C4B1A7000230D
:10166000F7E71FB3294B1B78012B1FD00023F0E7AE
:10167000D8F80430984790F8603043F0040380F8BD
:1016800060300123E5E70023E3E70023E1E70022E0
:10169000BAF1010FE1D0BAF1020FF4D1B9F1000FA4
:1016A000DFD01FB9194B1B78002BEED1002301931B
:1016B0004FF00203012262F3850362F387138DF872
:1016C0000030124D2B788DF8013033118DF8023037
:1016D00023118DF8033004F00F0444EA06168DF848
:1016E000046004F0BDFE4368684698472B78002BE1
:1016F000BED0D8F80430984790F8603043F020030B
:1017000080F860300123A4E70122C1E7A42A002069
:1017100030B587B00546036904A898479DF8133093
:10172000FBB9264C462303935D23029324230193A4
:101730000523009312230222114604F1140000F045
:1017400029F96B689847C588018942882A448388AB
:101750000B446580A180E28023816F2140F6F40272
:101760001FE0164C0A2303935D2302932423019365
:101770000723009312230322022104F1140000F036
:1017800009F96B689847C588018942882A4483888B
:101790000B446580A180E280238140F22C4140F619
:1017A0006602064B43205881998140F2F531D98178
:1017B0001A8200221A7007B030BD00BFA42A002090
:1017C0000048704720E0010010B50446028B038AF0
:1017D0009A4202D90123C375037594F82730012B6F
:1017E00012D0A37C012B14D0A27D0D4B53F82230D4
:1017F00020469847012811D0022814BF002002205B
:10180000A38D0133A38510BD0423E3750123237544
:10181000E7E70523E37501232375E5E70120EFE7FB
:101820002C120020C289B0F91A30B0F922105B1ACC
:10183000002BB8BF5B42934218DCB0F91C30B0F902
:1018400024105B1A002BB8BF5B429A4210DBB0F940
:10185000282043889A4207DCB0F92C304089834223
:10186000CCBF002001207047002070470020704747
:101870000020704770B5044690F82650012D05D918
:10188000AB1EDBB2012B08D9002070BD012303750C
:101890000020A0750323E375F7E7068D013636B205
:1018A0000685FFF7BFFF08B901232375032D01D07B
:1018B0000020EAE723889E42BCBF0123237563888A
:1018C0009E42C4BF012323750023A375627D237B41
:1018D0009A4201D00020D8E7B4F92A30A288934276
:1018E000BCBF01222275E2889342C4BF0123237545
:1018F000B4F92C3022899342BCBF0122227562893F
:101900009342C4BF0123237500236385237D4BB11C
:1019100000202075A685E38B6383238CA38301239A
:101920006375B2E7002363750220AEE710B5044685
:1019300090F8263023B9438D01334385002010BD34
:10194000012B25D1FFF76EFF18B90223E3750123A0
:10195000237501222285637D1344DBB26375A27572
:10196000B4F92210E183B4F9242022843BB1237D11
:101970002BB9607D012814BF00200120DFE7002083
:1019800020750123A38560856183A2836375F0E7D9
:101990000020D4E730B4BDF80850BDF80C400280F8
:1019A000438001FB02F292B2AB1A8380A21AC2807A
:1019B000058144810173BDF81030C381BDF8143036
:1019C0000382002303754375438583850385C375AF
:1019D0004FF6FF7242838283C2830284837530BCD8
:1019E0007047F0B585B005460C46164600230193B6
:1019F0000293ADF80C30898B608BFEF7BDFFD0B140
:101A00000A2201A93046FEF72BFF012822D9002324
:101A1000237563756385A3852385E3754FF6FF7290
:101A20006283A283E2832284A3752B706B80AB80D8
:101A3000284605B0F0BD0023237563756385A38533
:101A40002385E3754FF6FF726283A283E2832284CB
:101A5000A375D5E79DF8047000B3F368384698473E
:101A60006084336938469847A084B36A38469847FB
:101A700084F82600B3693846984720833046FFF73C
:101A800016FBA0B9002384F827302046FFF79CFE00
:101A9000628BA38B28706A80AB80C9E74FF6FF7317
:101AA0006384A384002384F826302383E6E701239C
:101AB00084F82730E9E700BF70B504460E46157874
:101AC0008B6A28469847012801D0012070BD002369
:101AD00023806380A380E38023816381A381E381EA
:101AE00023746374227E02F0F80263F3C302227649
:101AF000F36828469847A081336928469847E081D3
:101B0000237C01332374E0E72DE9F04104460F46BE
:101B10001678CB683046984780463B6930469847F0
:101B20000546BB6A30469847032841D0A389A8EBF5
:101B300003031BB22380B4F902209A42B8BF1A46AD
:101B400016466280B4F904709F42A8BF1F46A78062
:101B5000E089281A00B2E080B4F908208242B8BFB8
:101B600002462281B4F90A108142A8BF0146618170
:101B7000B4F9125001EB050C604553DA491B884259
:101B800050DD521B904203DC227E42F0020222769C
:101B9000EA1993424BDA7F1BBB4248DD721B93422A
:101BA000DEBF237E43F0080323760120BDE8F081E9
:101BB00000232374B4F90020E38A9A4222DB217EB9
:101BC00001F00801002914BF0020102059428A4268
:101BD00006DC227E12F0040F04BF40F00800C0B201
:101BE000B4F9062093420FDC237E13F0020F0BD1D1
:101BF00040F00400C0B29142D8DB237E13F0010F05
:101C000008D0D3E70020E1E7914207DB237E13F001
:101C1000010F03D140F00200C0B2C7E7002808BF9F
:101C20000120C3E7217E41F001012176A9E7227E50
:101C300042F004022276B1E741828282C38200230D
:101C4000038043808380C380038143818381C38178
:101C500003744374027E02F0F80263F3C302027657
:101C600070472DE9F04186B004460D461646002324
:101C70008DF81730314903AA03C982E803000093A5
:101C80000193ADF808300A2269463046FFF7E5F9BE
:101C900080469DF800708DF81770B36A38469847F3
:101CA000002831D0B8F1010F2ED1B36938469847DA
:101CB000AB8A834228D3B3683846984720BBF36881
:101CC0009DF817009847804633699DF8170098479C
:101CD00007462B7C06AA02EB830353F80C3C0DF15C
:101CE0001702314628469847A989EA896B7C5E1C11
:101CF0006E7421806280A4F80480E7802372607291
:101D0000204606B0BDE8F08100232B806B80AB80BD
:101D1000EB802B816B81AB81EB812B746B742A7E02
:101D200002F0F80263F3C3022A7623806380A38063
:101D3000E380237201236372E2E700BF38E0010011
:101D4000014B1888704700BFE82A00200A2070471E
:101D5000024B5B6803EB0010807B7047E82A002091
:101D6000024B5B680001185C704700BFE82A002046
:101D7000024B5B6803EB001040887047E82A0020A4
:101D8000024B5B6803EB001080887047E82A002054
:101D9000024B5B6803EB0010C0887047E82A002004
:101DA000024B5B6803EB001000897047E82A0020B3
:101DB000024B5B6803EB001040897047E82A002063
:101DC000024B5B6803EB001080897047E82A002013
:101DD000024B5B6803EB001040787047E82A002054
:101DE000014B198058607047E82A0020004870476E
:101DF00040E001000048704718000020004870478C
:101E0000E404002010B5064C04F110000DF03AF87F
:101E1000207504F118000DF03BF82077204610BD26
:101E20004C050020024A4FF4F071024809F0E6BD6B
:101E30006CA901002C0500200149024809F06ABE86
:101E40006CA901002C050020024A4021024809F03B
:101E5000D5BD00BF80A901007005002001490248DE
:101E600009F058BE80A901007005002000487047A5
:101E700088050020704700BF704700BF10B5054CB3
:101E800004F10C000CF0FEFFE3682075236120468E
:101E900010BD00BFD805002000487047300000206A
:101EA00070B546780C4CB500294604F114000B4A75
:101EB00009F0A4FD31462046094A09F09FFD294654
:101EC000201D084A09F09AFD294604F10800064A37
:101ED000BDE8704009F092BD1406002070AA010010
:101EE00084AA0100A0AA0100BCAA010010B50A4CF6
:101EF0000A4904F1140009F00DFE2046084909F0D2
:101F000009FE201D074909F005FE04F108000649F5
:101F1000BDE8104009F0FEBD1406002070AA0100C3
:101F20001CAA010034AA01004CAA010010B5054CFE
:101F300004F10C000CF0A6FFE36820752361204635
:101F400010BD00BF34060020004870474800002044
:101F500010B5074C074A04F108000C2109F04EFDAA
:101F60002046BDE81040044A062109F047BD00BFE5
:101F700070060020E8AA010000AB010010B5064C75
:101F8000064904F1080009F0C5FD2046BDE81040EF
:101F9000034909F0BFBD00BF70060020E8AA010098
:101FA00000AB010000487047A0050020704700BF4B
:101FB000704700BF10B5064C04F10C000CF068FF30
:101FC000207504F110000CF069FF204610BD00BF21
:101FD000A8060020004870476000002070B5067811
:101FE0000C4CB500294604F114000B4A09F006FD1B
:101FF00031462046094A09F001FD2946201D084ABC
:1020000009F0FCFC294604F10800064ABDE87040CE
:1020100009F0F4BCE40600207CAB010090AB0100A9
:10202000A8AB0100C0AB010010B50A4C0A4904F18D
:10203000140009F06FFD2046084909F06BFD201DD2
:10204000074909F067FD04F108000649BDE81040A2
:1020500009F060BDE40600207CAB010090AB0100FC
:10206000A8AB0100C0AB010010B5064C04F10C0098
:102070000CF00EFF207504F110000CF00FFF20464D
:1020800010BD00BF040700202DE9F0410CF0F6FE62
:102090000446FFF7B7FE0546FFF748FF0746FFF780
:1020A000E3FF224606462946012001F05FFE224654
:1020B0002946022001F05AFEFFF7E0FE8046FFF7B6
:1020C00079FF054622464146092001F04FFE22468F
:1020D00029460A2001F04AFE22463946052001F031
:1020E00045FE22463146062001F040FEFFF79AFEEB
:1020F000BDE8F041FFF7A8BE10B5FFF7C5FF094BDB
:102100001B689847084B1B689847084B1B68984703
:10211000BDE81040064A074B127853F822305B683E
:10212000184700BF90110020F4100020BC100020C0
:102130005D16002070AC010070B5FFF763FE044629
:10214000FFF7F4FE0646FFF78FFF0546FFF774FE24
:10215000FFF784FE2146012001F056FE21460220B1
:1021600001F052FE3146052001F04EFE29460620C0
:1021700001F04AFEFFF782FE0546FFF71BFF04460B
:102180002946092001F040FE2146BDE870400A20A2
:1021900001F03ABE70B500249CB011AE2146304625
:1021A0002C220BADCDE90B44CDE90D440F94ADF8D5
:1021B000404017F0A6FD08ABCDE90233CDE9054458
:1021C000CDE900560648049309940894CDF82740B9
:1021D0002B4604682A4629460B20A0471CB070BD38
:1021E000882B00200B4A0C4B127810B553F8223084
:1021F000DB689847FFF7CEFFFFF79EFF074B1B6991
:102200009847074B1B699847BDE81040054B1B6971
:10221000184700BF5D16002070AC0100901100202F
:10222000F4100020BC10002070B5064607F0D6FD63
:10223000194D012804462B781CD09EB99C421BD016
:10224000012B1AD0154E56F82330DB6898472046EC
:102250002C7007F0C9FD2B7856F82330BDE870408C
:102260005B681847012E12D0032EE7D1022B03D052
:102270000224E5E7012B00D170BDFFF7B3FF204634
:102280002C7007F0B1FDBDE87040FFF735BF002BA3
:10229000F2D00024D4E700BF5D16002070AC01002E
:1022A000614A2DE9F04F1278604B8BB053F8223021
:1022B0005F4C9B689847C0F3074307930990C0F3AE
:1022C000072A07F097FD064607F098FDB3792278B4
:1022D00083469A4204D0B07905F0B6FCB3792370F6
:1022E000544B0124986805F035F80025ED23DFF8FC
:1022F00068815148DFF85491504F0593224621469A
:102300004346CDE90309CDE901550094642000F06E
:102310009BF93B6898F800209978914213D0F321FB
:10232000CDE901552546464A023305910392CDF881
:102330001090009422462146642000F085F93B6805
:102340009B7888F800300DF095F83B688DF82300F5
:10235000DB7883422CD1BBF1000F3ED1002D3CD164
:10236000079B002B43D0737E002B49D1337E002B7B
:1023700055D1079B012B01D10EF0F8FD7222314B94
:1023800000921A683049314B632000F0AFF9FFF733
:1023900029FFFFF7B1FE77222D4B00921A682A49D8
:1023A0002A4B632000F0A2F901200BB0BDE8F08FAA
:1023B00001224FF4817100232648CDE90491CDE933
:1023C000013303900DF1230364200092114600F0C5
:1023D0003BF93B68D8780DF039F8002007F014FD80
:1023E000337E002BCAD0002007F0FEFCC6E7337E08
:1023F0007BB95046FFF718FF01200BB0BDE8F08F06
:10240000337E002BF5D0284607F0EEFC4FF0010A92
:10241000EFE7079807F0E8FC4FF0010AE9E72846E4
:1024200007F0E2FCA5E700BF5D16002070AC0100DC
:102430005C160020080A00203CAC0100340A002091
:1024400048AC01004C070020E4AB01002CAC0100BB
:102450005007002064AC0100840700202DE9F047FC
:1024600092B00446884607F0C5FC00233F4FC27D6A
:10247000C7E900333B81002A56D094F82B0094F82A
:102480002AA094F82990504594F8281038D8A0F143
:10249000160EC21FA0F10F065FFA8EFED2B2F6B280
:1024A000894521D84B4612E0A3F10A04022C4ED8EC
:1024B00000EB431438F91450012437F914C0AC452B
:1024C000B8BF27F814500133DBB299420CD3022A6B
:1024D000EAD9022E2BD89C1F022C28D800EB4315DA
:1024E000022438F91550E8E70130C0B20EF1010EB0
:1024F0000132013682455FFA8EFED2B2F6B2CFD2F9
:102500003E2200210DF10A0017F0FBFB002340F2F0
:102510000155822400971A4602A91E20ADF80850E2
:102520008DF80D4007F014FE12B0BDE8F087BEF143
:10253000020FC8D8A3F10A04022C11D99C1E022C48
:10254000C1D800EB431438F914500324B5E79C1E9E
:10255000022CB8D800EB431438F914500024ACE72F
:1025600000EB431438F914500424A6E76016002049
:10257000F0B5204E83B0054601F1200014461F46F9
:102580007160FDF77FFE1C4B1C4A99682130376053
:102590004860946060782278E37802FB00F203F0F0
:1025A0007F0303FB02F3164C22790B60D3B2012B9D
:1025B00001D003B0F0BD7721FF221E46114F3970C4
:1025C00022712379FF2B10D120222946684617F06B
:1025D00069FB009B032B04EB830206DC019BD2F812
:1025E000052006FA03F31342EBD105233B7003B039
:1025F000F0BD00BF34210020580A00203C0C002010
:10260000F4210020080B002070B504460E46154644
:10261000049A194620F8022B20341E2217F030FCB1
:1026200020463146DF2217F02BFC45B13046FDF73E
:1026300029FE2946C0F1DF02204417F021FC204684
:10264000BDE87040FDF71EBE2DE9F041C4B0044660
:102650000E4615460146202204A81F4617F022FB0D
:10266000049B032B0EDC01221F48059900EB83031A
:10267000D3F805C002FA01F313EA0C0F02D0037974
:10268000934202D044B0BDE8F0814FF000084FF40F
:102690008072414604A817F034FB4F9B42460093DA
:1026A0004D994E9B04A8CDE90288FFF7ADFF9DF838
:1026B0000BC04A9B4B9A8DF80F0063F3060C204623
:1026C0004C9C62F3C71C3B4604A902AA8DF8086023
:1026D0008DF809508DF80C808DF80E408DF80BC0E8
:1026E000FFF746FFCEE700BFF42100202DE9F041BF
:1026F000C4B004460D4616460146202204A81F46D3
:1027000017F0D0FA049B032B0EDC0122194805991F
:1027100000EB8303D3F805C002FA01F313EA0C0FB0
:1027200002D00379934202D044B0BDE8F0814FF06B
:1027300000084FF48072414604A817F0E2FA4A9B61
:102740003246009329463B4604A8CDE90288FFF7AC
:102750005BFF43468DF80F0002AA04A92046ADF89E
:1027600008808DF80B808DF80C808DF80E80FFF7B7
:10277000FFFED9E7F4210020F0B5644687B001F0F0
:1027800069FD002601F0B8FD0125042040F22F3735
:102790002369A268DB68E168CDE901560090064D27
:1027A00006480597CDE903057220FFF74DFF236921
:1027B000D86807B0F0BD00BF00AE010068AD0100F1
:1027C0002DE9F04F91F81CE090F802C00F460EFB87
:1027D0000CF5097D85B00191DDF838804DB3444694
:1027E000002605EB450C08EB0C1C226294F82450E3
:1027F00084F8246094F8255084F8256094F82650D5
:1028000084F8266094F8275084F8276094F82850BC
:1028100084F8286094F8295084F8296094F82A50A4
:1028200084F82A6094F82B5084F82B603034A44547
:10283000DBD1BEF1000F32D03D460026074603F142
:10284000FF3921B3CB4600242B69062213F804A0DC
:1028500002A84FEA6A01013117F024FABA780AF0A7
:10286000010306FB0233029A03EB4303920002EBDF
:102870000313039943441BF8012F186A01EB8101EC
:102880008A4002431A622B7D0134A342DCDC2B7F99
:102890000136019AB342914401DD297DD1E705B0AB
:1028A000BDE8F08F2DE9F041002482B0089D2A6236
:1028B0002A6595F8242085F8244095F8252085F888
:1028C000254095F8262085F8264095F8272085F89C
:1028D000274095F8542085F8544095F8552085F800
:1028E000554095F8562085F8564095F8572085F8BC
:1028F000574095F8282085F8284095F8292085F834
:10290000294095F82A2085F82A4095F82B2085F84B
:102910002B4095F8582085F8584095F8592085F8AF
:10292000594095F85A2085F85A4095F85B2085F86B
:102930005B400A7D12B30F465E1E3B69062213F808
:10294000048068464FEA6801013117F0ABF908F0DE
:102950000108009A4FEA48039844930003EB0813D8
:1029600001992B4416F8012F186A01EB81018A4066
:1029700002431A623B7D0134A342DEDC02B0BDE8B3
:10298000F08100BF2DE9F04F97B06846D1F80130D3
:1029900006AF1E7D1D7F796006FB05F3D1F8092087
:1029A0005C00FA62DA1DD208A0EBC200854604F191
:1029B0000803DB08DB0006A8ADEB030DF86006A8F2
:1029C000ADEB030D06AAADEB030DFB6ABC60DB6843
:1029D000BA623B620A2322467400A046FF217B6153
:1029E000386117F08EF906AB7B62B3007B637A69BE
:1029F0007B681F2AD3F8053040F3198110464446FE
:102A0000954901FB02F102EB421200EB421202EB8C
:102A1000C23201F1404102F140422031013241F025
:102A20001F0103F5B46019625A629A62303383421F
:102A3000F9D18A480122049089488D21039004230A
:102A40000020A04602900192059100937C6907F155
:102A50003C0311466420FC63FFF7F6FDBC680021CF
:102A60002246B86A17F04DF92246FF21786A17F01E
:102A700048F9142344463B6301F0ECFB01F03CFCB5
:102A80000421FB6A4FF0000CDB6800919621059150
:102A90007249202204917349722003910121CDE9EA
:102AA000011C0F21FFF7D0FD45B34FF000093B6A31
:102AB000D7F824A0A3F1040BBB6AA3F10208002EEF
:102AC00000F0AB80D446DE464346A0445EF8042FB7
:102AD00033F8020FBCF800108242C8BF90B28A429D
:102AE000B8BF91B2434518802CF8021BEED109F112
:102AF00001097B6B4D459B44A244E0D13B6B013BFC
:102B00003B63B9D1A046002D35D09B46BB6AD7F8B0
:102B10000C90023BFB617B6AD7F81480023B3B635D
:102B20003B69BD61A3F1020AB6B150460021D7F856
:102B300030C0FD6935F8023F3CF802EF30F8022F53
:102B4000A3EB0E039A42C8BF09F8018001F101010D
:102B5000C8BF03808E42EDD1FB690BF1010B23440A
:102B6000FB613B6BA24423443B63BB69B1445B45BF
:102B7000DAD1A046BD69A9217869FB6A0130786184
:102B8000DB680591354904220491364904460391D6
:102B9000002001210092CDE9011020220F216420A4
:102BA000FFF752FD3E2C7FF422AFAC222B4B00925C
:102BB0002D4900226420FFF799FD0020CDE9010096
:102BC0000120AD21254B294A00900493FB68642025
:102BD0000591039229463246FFF736FDAF221F4B7F
:102BE0000092234900226420FFF780FD1B4B4FF029
:102BF000B00C049300230224CDE901331D483B6946
:102C0000324603902946CDF814C000946420FFF7A3
:102C10001BFD4437BD46BDE8F08F09F101097B6B10
:102C20004D45A0449B44A2447FF449AF66E77A69CE
:102C300044461146084800FB02F002EB421201EB49
:102C4000421202EBC23203F5B46118625A629A6210
:102C500030338B42F9D1ECE62084100200AE010043
:102C6000B8AD010068AD0100C4AD0100D8AD0100F0
:102C7000E4AD0100F4AD01002DE9F04FD2F8018080
:102C8000D2F805C098F81C9098F814A0B9F1000F7C
:102C900022D04FF0000E0139BAF1000F17D00C46C8
:102CA0008678D8F810200EFB06F60AEB020712F819
:102CB00001BB14F8015F0BF00103334403EB430342
:102CC0000CEB031303EB5B039742DD73EFD10EF1C3
:102CD000010ECE455144DFD1BDE8F08FF0B5DCE9FF
:102CE000002087B064460F46FFF7C6FFD4E90221F3
:102CF000002040F239360125CDE90100054C064897
:102D00003B46CDE90304059600956420FFF79CFC43
:102D100007B0F0BD00AE010030AD01002DE9F04F6D
:102D20008DB082788A4602EB4202120100AFADEB11
:102D3000020D6E46F8610021684616F0E2FF4FF47E
:102D4000B4620021C84816F0DCFF9AF81450BE6146
:102D500035B3DAF810000124054406E053688542D3
:102D600043EA0E0EC2F804E01AD010F8013B03F05B
:102D7000010C4FEA4C0262441F2B04FA03FE06EBDF
:102D80000212EBDD117A203B8C4604FA03F3C1F307
:102D900001010B4363F3010C854282F808C0E4D1C2
:102DA0009AF81C30BB62002B00F08381DAF81820FF
:102DB000002411460120FA62194412F8013B00FA7E
:102DC00003F3914244EA0304F7D1FB693C6293F8B0
:102DD00002C0BCF1000F00F07D810021BA69C7F884
:102DE0002CA010460D464FF0010B4FF019099246EA
:102DF0003B6AC3F313065FFA86F8C6F3072E360C58
:102E000001EB41030AEB03135C781A7A6FF3C304F6
:102E10005C709C7A02F0030224F03F049C7293F8E9
:102E20002E401A7224F01F045D7283F82C5083F830
:102E30002D5083F82E4003F1080280F80BB080F883
:102E40002F909379013123F00F0333438C4582F89F
:102E5000048082F805E000F130009371D0D14FF08A
:102E600040533A6AD7F82CA09A64BB6A002B00F052
:102E70002A81DAF81830FB6200234FF0010B7B62E5
:102E80009946794BBB624FF0000CFB6A29F00302B4
:102E900013F80930BC6A0BFA03F8C8F31308C8F337
:102EA0000D039B00BB604FEA98337B60131D3A61B2
:102EB000FB60C7F81480A6464FEA4C05BB69654421
:102EC00003EB051505F13008764628686968AA689D
:102ED000EB68103545450EF1100E0FC6F4D123886E
:102EE000796A9AF80B2061F309032380002A40F0E5
:102EF000BD8023687A6962F31F332360FB699AF807
:102F00000C00DB783A6A0BFA03F3013842EA03015A
:102F10009AF81C20032800F2C880DFE800F0825BEA
:102F20003602206894F82E5043EA103025F01F0531
:102F3000C0F31403013A45EA13454A45A08584F8D5
:102F40002E500FDDFA6A4A445078EAB20BFA00F0CC
:102F50000343C3F3140322F01F0242EA1342A38582
:102F600084F82E20B9F1000F08D0FA6A4A4412F80A
:102F7000012C0BFA02F21343C3F3140383F4FF137F
:102F800083F4FF5383F01F032AE0E36A013A4A45C2
:102F9000C3F3140311DDFA6A4A44507894F82E20E2
:102FA0000BFA00F00343C3F3044022F01F02024374
:102FB000A38584F82E20C3F31403B9F1000F0FD0BA
:102FC000FA6A4A4412F8012C0BFA02F21343C3F3D3
:102FD000140305E0226843EA1233DB43C3F314030E
:102FE000E2681940A07B94F82E30C2F3130222EA63
:102FF0000102A18520F00F0023F01F03C1F304415B
:1030000040EA12401943A281A07384F82E10303494
:10301000BCF1000F15D1DAF818304FF0010CFB624B
:1030200049E794F82E20C3F31403194022F01F023D
:1030300042EA1142A18584F82E203034BCF1000F01
:10304000E9D07A6A9AF81C302032C2F309027A6217
:10305000BA6A09F1010960324B45BA6233DDDAF828
:103060001830FB620FE700BF98000460FB6A3A6902
:103070009918FA689D1811F8013B20680BFA03F3C0
:10308000226843EA103363F31F328D422260F2D18B
:103090002389BA6803F0030313432381A37A7A6870
:1030A00023F03F031343A37228E7E36AC3F3140337
:1030B00096E7FB6993F802C0BCF1000F07D14FF00F
:1030C0004053C3F848C03437BD46BDE8F08FBB6AF3
:1030D0003B6282E64FF040533A6A9A64CCE600BF06
:1030E0002DE9F041827800AF02EB42021201ADEB14
:1030F000020D884605460021684616F002FE302281
:103100000021614816F0FDFD6FF01F019DF80130B0
:1031100098F80C2003F0F40343F00903013A8DF80A
:1031200000108DF801306C46032A03D8DFE802F066
:10313000948002024FF0FF324FF04051002094F88B
:103140002E3084F82C2043F01F0384F82E3084F8AE
:103150002D20C1F830014FF00132192604F130055D
:1031600028462346C4F80F20C4F81320C4F81720BB
:10317000C4F81B20E277E27284F82F60D3F800C015
:103180005E689968DA681033AB42C0F800C04660E8
:103190008160C26000F11000F0D198F814303BB3A8
:1031A000D8F81000012603EB000C06E053688445B4
:1031B00043EA0808C2F804801AD010F8013B03F073
:1031C000010E4FEA4E0272441F2B06FA03F804EB7D
:1031D0000212EBDD117A203B8E4606FA03F3C1F3AF
:1031E00001010B4363F3010E844582F808E0E4D14A
:1031F0002646DFF894E0F44630687168B268F368F8
:103200001036AE420EF1100EACE80F00F3D1DFF82D
:1032100080C06034654630687168B268F368103603
:10322000A6420CF1100C0FC5F4D1BD46BDE8F081EB
:103230004FF0FF324FF04051002094F82E3084F8C8
:103240002C2023F01F0343F00F0384F82E3084F862
:103250002D20C1F830017EE701224FF04051E8787F
:1032600094F82E308240C2F3044523F01F03074830
:103270002B43C2F3072584F82C2084F82D5084F8C2
:103280002E30C1F8300166E738060460FFFF0F00FA
:1032900068060460F0B50D46A9B04C220021044632
:1032A00002A816F02EFD00204FF040522978ADF80C
:1032B000040082F8A8106978BDF80420A87861F3AA
:1032C0008A12C2F3072160F3C601ADF804208DF81D
:1032D0000510BDF8041002AB0DF12A025985023326
:1032E0009342FBD14FF04056002286F8A7202F7D55
:1032F000C7B14FF0010C2969013911F8013F28A825
:1033000018441C2B00F8982C02F1010208DD96F8F5
:10331000A7001D3B0CFA03F30343DBB286F8A7308A
:103320009742EAD102A915A84C2216F0DFFC15A994
:103330004C22094816F0DAFC4C2215A9074816F071
:10334000D5FC29462046FFF7E9FC20462946FFF731
:10335000C7FE024829B0F0BD4C00046000000460C4
:103360002DE9F04FD0F80D40D0F80160D4F800C03E
:10337000D6F820E09CF800309CF8012096F80090E8
:10338000D5185FFA85F808F1010B03F1010A0F4621
:10339000591ED0F8090089B08EF829B08EF8228025
:1033A0008EF824A08EF82510B9F1000F4CD0013210
:1033B0008EF8272000238EF828301A46636893F889
:1033C000008008F03F0802F114030EEB43039978E4
:1033D000013268F30501112A9970F4D119211C4BAF
:1033E0001C4A83F82F1030339342FAD133796BB1F2
:1033F00043685BB1164D9CF80D2031460095384668
:10340000FFF7DEF923685A781B78D51849F6404350
:1034100001356D0093FBF5F540F2E9100122002122
:10342000042608AB43F8045D0B4C05900B48CDE92E
:103430000121CDE90304114600966420FFF704F949
:10344000034809B0BDE8F08F0A3B8EF82730B1E79A
:10345000980004603806046000AE010078AD0100F9
:103460002DE9F047D0F80D80D0F80150D8F80030A1
:103470002C6A93F801C01B7895F800E00CEB03026E
:10348000D2B202F1010A03F101090F46591ED0F828
:10349000096082B084F875A084F86E2084F870907A
:1034A00084F87110BEF1000F3BD00CF1010C84F8D0
:1034B00073C000231A4684F87430D8F804C09CF80E
:1034C000020000F03F0002F1140304EB430393F801
:1034D0004E10013260F30501112A83F84E10F2D12B
:1034E0009CF80010114AC901301D08F087FAD8F87D
:1034F00004300F4A197806F10800C90108F07EFA75
:103500002B7953B1736943B1D8F80020094C527B31
:10351000294638460094FFF7C5F9064802B0BDE8D1
:10352000F0870A3B84F87330C3E700BF4CAD01005D
:1035300064AD010038060460F0B500264FF040533A
:1035400001250424D0F80D20D0F80110506812682D
:10355000467090784FF00F0E83F82C01D0784FF41E
:10356000B47C83F82D01107A83F82A01907A83F8CD
:103570002B01107983F82E01507983F82F010F78F1
:10358000C87883F825714F7983F88E7083F88400AA
:1035900083F8815083F8806083F8AE4083F8AF40B1
:1035A0000E7993F8890086EA050767F3051002276C
:1035B00083F8890093F8A10066F3041083F8A10052
:1035C00083F88D4083F8B05083F8C5E0A3F8C8C0F5
:1035D00083F8CC70947B087A83F800418C7983F867
:1035E0000541CC7983F80A4183F80D01497A83F8C3
:1035F0001011117B83F8DA10D27A83F8A020BDE88D
:10360000F04000F095BB00BF4FF0405310B5D0F82C
:103610000D10D0F809204C68526893F84111607879
:10362000054B02EBC01003EB0141802216F05EFB5C
:1036300063780133637010BD8007016070B5194B6A
:1036400084B01B78044613B106F0D4FBC37ED4F8D3
:103650000130DB7A23B3D4F80930DE6806F1800547
:1036600006F50866A5F1800000231946DA018258A4
:103670004DF823200133042B1144F7D100225DF8CB
:103680002230D401A1EB430301325B10042A035121
:10369000F5D10430A842E7D105F50075B542E1D176
:1036A00004B070BD971700204FF040532DE9F04152
:1036B000012604240025D0F80D20D0F8011012684E
:1036C0004FF00F0890784FF0030E83F8E000D078A9
:1036D00083F8E100107983F8E200507983F8E30081
:1036E000107A83F8E600907A83F8E7004F79C8787B
:1036F00083F88E7083F8840083F8816083F88050AB
:1037000083F8AE4083F8AF400F7993F8890087EAD9
:10371000060C6CF305104FF01E0C83F8890093F82B
:10372000A10067F3041083F8A10083F88D4083F8AB
:10373000B06083F8C58083F887E0A3F8C85083F8A9
:10374000CCC0907B83F80001887983F80501C879A3
:1037500083F80A01497A83F81011117B83F8DA1093
:10376000D27A83F8A020BDE8F04100F0E1BA00BFB2
:103770004FF040532DE9F04101260025D0F80D10FF
:10378000D0F80100D1E900219478497883F8E0402D
:10379000D4784FF0040883F8E14014794FF00F0E0D
:1037A00083F8E2405479B14083F8E340147A31441D
:1037B00083F8E640947AC9B283F8E7404779C47841
:1037C00083F88E7083F8844083F8816083F880509A
:1037D000077993F8894087EA060C6CF305144FF0DB
:1037E000030C83F8894093F8A14067F3041483F82D
:1037F000A14083F88D8083F8B06083F8C5E083F83A
:1038000087C0A3F8C85083F8CC10917B83F80011CF
:10381000817983F80511C17983F80A11417A83F817
:103820001011117B83F8DA10D27A83F8A020BDE85A
:10383000F08100BF2DE9F04F99B0734C06AF07F14E
:10384000240A7861714D0E4694E80F008AE80F0053
:1038500007F1700307F134087B6407F11003504649
:103860004146CAF80830CAF80C50FCF709FD94E844
:103870000F00674C88E80F0007F11003404607F17E
:103880004401C8E90234FCF7FBFC012000F06CFCA9
:103890003861002800F0B3800023E9461A46D0F8CA
:1038A00001505C48297D2C7FB961FC6101FB04FB60
:1038B0006978B96029792B71F96002F1140300EB82
:1038C00043035988013241F4F861112A5980F4D137
:1038D00069460BF10703DB08A1EBC3039D46D6F84D
:1038E0000D20D6F809C0136806AC5B78DCF8081028
:1038F00020465A467B60C7F820C016F0F7F97B686F
:10390000BBF1000F09D0224604EB0B0012F8011B9B
:103910000431824202F8011CF8D148F001024AF059
:103920000101CDE90021012019465A46234602F043
:1039300033FF3B6A5A461868214616F0D7F940F221
:1039400041304FF0000B4FF0010C3B6ABA691B6825
:10395000F969DFF8CC8005902F48CDE901BBCDE9AE
:103960000308CDF800C06420FEF76EFED7F81CA057
:10397000DA4518DD5846D7F818C0D7F820E0BCF172
:10398000000F0DDD00222B7DDEF81C1000FB032351
:10399000895C14F803B0013259446245E154F2D114
:1039A00001305045EBD1324621467869FFF764F982
:1039B000D7E9062140F24B3000250126CDE90480ED
:1039C000164823460390CDE9015564200096FEF782
:1039D0003BFE2A46BB680F4C03F01F0002F11403A4
:1039E00004EB43035988013260F38A11112A59808C
:1039F000F4D13B693A7BD3F801301A71CD464C378C
:103A0000BD46BDE8F08F00BFD89E010079270000B9
:103A1000DD2C0000000004603CAD010030AD010071
:103A200000AE01002DE9F04FADF50D7D06AF7860D9
:103A30008A4600F065FA061E40F3C580002403E0C4
:103A40000134A64200F0BF802146012000F066FA52
:103A50000028F5D007F1140E0546F446D0F80140D1
:103A600004F12008664620686168A268E3681034A3
:103A700044450CF1100C0FC6F4D1002620684FF419
:103A8000F072CCF800008EF80460C5F801E0DAF8B6
:103A90000D3001211B6807F138005B781C46FB6084
:103AA00016F02FF9ADF5F16D06AB184631464FF41F
:103AB000F06216F026F9012C40F389800124A1461A
:103AC000031FDFF82081BB60DAF8055005F10F0B0A
:103AD00005F2AF555846112221460BF1300B16F076
:103AE00010F9AB45F6D1012240F27A330425394969
:103AF0006420CDE902610593114607F11003CDF86A
:103B00001080CDF8049000953C61FEF79DFD00F01B
:103B1000A1FB00F0F1FB40F27E332F4A0593CDE983
:103B200002624FF0C04320220F210095CDF8108093
:103B3000CDF804907220FEF787FD4FF0C043B968BE
:103B4000DFF8A4C007F13802186851F8045F0433A5
:103B50008542BCBF14700860634502F10102F3D1D5
:103B60004FF463731D4A0593CDE9026207F13803F0
:103B7000CDF81080CDE9009620220F216420FEF7B9
:103B800063FDFB680134A3429ED15246786807F179
:103B90003801FFF771F84FF46474002201201049D6
:103BA00007F13803CDE9012200900391CDF8108090
:103BB000059420220F216420FEF746FD07F50777C4
:103BC000BD46BDE8F08F0023D3F80130FFDEDFF8FB
:103BD0001480DAE788AD010098AD010030AD010036
:103BE000A0AD010000AE01008007006008B500F044
:103BF00083FB022000F0B8FAD0F80930986808BDBD
:103C000008B500F079FB012000F0AEFAD0F80930D9
:103C1000D86808BD30B4D0F80D20D0F8093052680B
:103C200015789DB19C685B68803C03F17C00E41AC8
:103C300000EBC515A0F18003221853F8041F83423E
:103C400042F8041FF9D18030A842F3D130BC70474C
:103C5000704700BF002070474FF0405393F8412158
:103C6000002082F0010283F8412193F8432182F081
:103C7000010283F8432170472DE9F047482286B0BE
:103C8000FF212A4816F03DF801A80BF0FBF880460A
:103C900002A80BF0FDF8074603A80BF0FFF818F098
:103CA000FF081DD04FF0000A4FF001091F4E04AD70
:103CB000019B082213F80A402846610004F003041F
:103CC00015F0F0FF04EBC404049A3444059BA15C96
:103CD00009FA03F30AF1010A0B43C245A354E7D1E1
:103CE00017F0FF071FD04FF000094FF001080F4EEB
:103CF00004AD039B082213F809402846610004F034
:103D00000304043404EBC404344415F0CBFFDDE9B0
:103D10000423A15C013308FA03F309F101090B4301
:103D2000B945A354E5D106B0BDE8F087742C002056
:103D300008B50BF085FB054B1B78984204D018465C
:103D4000BDE808400BF05EBB08BD00BF8407002043
:103D500010B50BF075FB04460BF066FB844203D0F4
:103D6000BDE810400BF04EBB10BD00BF30B50138B0
:103D700085B00C460A2810D8DFE800F03B3E0F3B28
:103D800026110F0F2611060003A80BF07BF8224620
:103D9000C1B2039801F07AFDA06305B030BD03A85D
:103DA0000BF076F80223C5B203992A460093204609
:103DB00004F1150300F092FC22462946039801F015
:103DC00079FBA06305B030BD03A80BF05BF80223BC
:103DD000C5B203992A460093204604F1150300F06A
:103DE0007DFC22462946039801F022F8A06305B025
:103DF00030BDCB7A002BD0D010462146FFF74AFACF
:103E0000206205B030BD00BF0138092808D8DFE8BE
:103E100000F00808080705050505050500238B6364
:103E2000704700230B627047037810B5022B0446DD
:103E30000BD0042B03D10022D0F801301A620023EA
:103E40006374A374E374237510BDD0F809000849A6
:103E5000043007F05FFED4F809000649083007F087
:103E600059FE00236374A374E374237510BD00BF6F
:103E700018AE010038AE0100002230B504460D46F0
:103E800083B002AB43F8042D18460E4A152107F003
:103E9000B5FD22780C4B294653F82230204698472E
:103EA000C4F80500A06822686568E168019B986015
:103EB0001A605D60D960226901981A61227D1A75C5
:103EC00003B030BD10AE010074AE01000B4B1A6898
:103ED0000AB90CE01A46D2F81130002BFAD10023AF
:103EE000C2F8110043748374C3740375704718607B
:103EF000002343748374C374037570476C160020E9
:103F0000054B1B6833B10020D3F811300130002B72
:103F1000FAD17047184670476C16002070B5164BE2
:103F200088B01B687BB1002402E0D3F8113053B194
:103F30001A788242F9D101340029F6D0A142F4D195
:103F4000184608B070BD4FF4E17001220024042629
:103F500008AB43F8041D094D05900948CDE901243B
:103F6000CDE90305114600966420FEF76DFB23465C
:103F7000184608B070BD00BF6C1600205CAE010092
:103F800064AE010070B5094E82B034684CB1084D82
:103F90000194D4F81140294601A807F0BBFD002C7C
:103FA000F6D10023C6E9003302B070BD6C160020C4
:103FB00054AE0100F8B5446805460AF05FFFACB1A5
:103FC00023780B2B12D80B4E0146074656F8333098
:103FD00020469847D4F8110040B10378394606EBE3
:103FE000C3066860736898470120F8BD00206860C8
:103FF000F8BD00BF8807002010B504460AF03EFF58
:10400000636843B11C78054A014652F834201846CB
:104010009047012010BD184610BD00BF8807002042
:1040200038B5446805460AF029FF4CB12278054BA3
:10403000014653F832302046984700236B6038BD64
:104040006C6038BD8807002070B582B005460C460C
:104050000AF014FF4FF0405393F84121014682F0DB
:10406000010283F8412193F8432182F0010283F891
:104070004321286818B90CE0D0F8110058B1027833
:10408000A242F9D10A4A686002EBC4025368984719
:10409000012002B070BD4FF40B76064D064C009621
:1040A0002B46002221466420FEF720FBF7E700BFE5
:1040B000880700205CAE0100A4AE010038B504689A
:1040C00005460AF0DBFE6CB16B685BB92178064BE4
:1040D0002A6803EBC1035B6801466A602046984783
:1040E000012038BD002038BD8807002008B54FF0FA
:1040F000405393F8243093B172B60A48FFF7DEFFBD
:1041000058B10123084A1375BFF34F8F4FF0405247
:104110000020064908721370937062B608BD0BF058
:104120005FFAE9E76C160020000010509828002084
:1041300008B572B60948FFF7C1FF60B10422084B09
:104140001A75BFF34F8F4FF04053012200200549ED
:1041500008721A709A7062B608BD00BF6C16002013
:104160000000105098280020054B1B6833B11A78C6
:10417000824203D0D3F81130002BF8D11846704793
:104180006C160020044B11B143F820107047034A0D
:1041900043F82020704700BF54070020513C000026
:1041A0000B4B70B51C680AF069FE7CB10546094EE0
:1041B00023782046294656F823309847D4F81140F2
:1041C000002CF5D1BDE87040FFF7C2BD70BD00BF47
:1041D0006C1600205407002008B50E4B5A6802B137
:1041E00008BD01461846FFF72FFF0028F8D00A4BFC
:1041F0001B680BB10BF0F4F90123084A1375BFF3E8
:104200004F8F4FF040520020054908721370937091
:1042100008BD00BF6C160020BC2800200000105014
:104220009828002038B50023064D074C074A084956
:104230002B72236011600BF045FCBDE83840FFF79E
:1042400055BF00BF982800209C1700209817002019
:10425000ED400000002330B401240649064D074814
:10426000074A0B7207492B60047030BC1160FFF7DE
:104270003DBF00BF982800209C1700209717002002
:1042800098170020ED400000002330B401240649B7
:10429000064D0748074A0B7207492B60047030BC73
:1042A0001160FFF745BF00BF982800209C17002031
:1042B00097170020981700203141000008B50BF037
:1042C00015FC00230249034A0B60136008BD00BFC0
:1042D000981700209C170020024B5868003018BF28
:1042E000012070476C160020024B1868B0FA80F06D
:1042F000400970476C16002008B5074908200AF0ED
:10430000CFFFFFF74DFF0BF0F1FB00230349044AF9
:104310000B60136008BD00BF593C000098170020D7
:104320009C17002008B572B60BF0E0FB002308498B
:10433000084A0B60136062B6074A516831B1536096
:1043400006490820BDE808400AF0AABF08BD00BF22
:10435000981700209C1700206C160020593C000084
:1043600008B5044908200AF09BFFBDE80840FFF7A4
:1043700017BF00BF593C000008B50449082015F0DC
:10438000A7FDBDE80840FFF70BBF00BF593C000088
:1043900008222F4838B52F4C436822602E4ACBB1F3
:1043A000002519781570022937D0D3F8113093B150
:1043B0002748FFF7FFFD002846D00123274A137541
:1043C000BFF34F8F4FF04052002025490872137001
:1043D00093700DE0137001250021224B20481F4AE5
:1043E0001B680572117503B198471948FFF718FE4D
:1043F00010221D4B2260D3F80021120708D500229D
:1044000008241A481A49C3F880410270C1F84021B3
:104410004FF0405300225A7038BDD3F80D20516838
:104420000A784978013A9142BFDAFFF7E5FD58B1C1
:1044300001230A4A1375BFF34F8F4FF040520849CA
:104440000D7213709370D3E70122054B1A72CFE7F8
:104450006C160020A40C00209617002000001050BD
:1044600098280020B828002000E100E0A00C0020DF
:1044700000000250B8B4850005F10A0323F00703D9
:10448000002800AFADEB030D11DD6B46043A154477
:104490000239181F31F8024F52F8043F03FB04F3AE
:1044A000AA424FEA132440F8043F1460F2D1BD46FB
:1044B000B8BC70472DE9F043089D1DB34FF04C0C7C
:1044C00001264FF00009079CD2B20CFB054CC9B283
:1044D0009719C0B20F44A1F10A08A1F1030EFFB26F
:1044E00080448644002B14BF45467546A070267153
:1044F000E7706171A27184F81990A676E5714C3469
:104500006445EFD1BDE8F083F0B5012A83B01646CB
:1045100005460C461F462DDC0146684615F0C2FBD9
:1045200036B3009B3F2B1D46A8BF3F25019A002BA9
:10453000134405F03F05B8BF00253F2B1A46A8BF1E
:104540003F22002B4FF0000102F03F03B8BF0023D1
:1045500004F1100207EB420C09B30A19103207EB01
:104560004202907965F3050090710131B142F3DBAD
:1045700003B0F0BD104607F00BFA044106FB04F44B
:104580000F2C294606DD0122684615F08BFB01261B
:10459000009BC7E73246684615F084FBC1E79CF8EC
:1045A000062063F305028CF80620DEE7F0B5012A49
:1045B00083B0154604460E461F462DDC014668466C
:1045C00015F070FB009B2DB33F2B1C46A8BF3F246A
:1045D000019A002B134404F03F04B8BF00243F2B82
:1045E0001A46A8BF3F22002B4FF0000102F03F0304
:1045F000B8BF002306F1100207EB420CF1B18A1993
:10460000103207EB4202907964F30500907101319A
:104610008D42F3D103B0F0BD104607F0B9F9F307AE
:1046200044BF06416E4321462A46684654BF06F100
:10463000FF36013615F036FB009BC5E79CF80620D7
:1046400063F305028CF80620E1E700BF70B5DCF8E3
:104650000C3086B0644600259847FFF74DFED4E93C
:1046600001230121042040F253261B690295CDE964
:104670000001064D06480596CDE903057220FDF7B9
:10468000E3FFA368186906B070BD00BFF0AE01007B
:10469000FCAE010070B5644686B0DCF8083098477F
:1046A000FFF72AFE002201214FF475760425636886
:1046B00008481B690292084A0596CDE90320CDE916
:1046C000005114227220FDF7BFFF6368186906B01D
:1046D00070BD00BFF0AE0100FCAE01002DE9F04F4F
:1046E00087B006AF4578D7F82890D01D20F0070096
:1046F00009FB05F5ADEB000D0DF1180A0E4650460D
:10470000002190461C4615F0FCFAA94541DB4FF00C
:10471000000B08F1FF3922224FF0FF31204615F03F
:10472000F0FA33784FFA8BF0B8F1010FE0542DDD39
:104730004FF0000E6FEA060C711C11F8012BA35606
:10474000B3F1FF3F05D1431CAB42ACBF00235BB2CA
:10475000A35498421AD092FBF5F005FB10200128D3
:1047600014BF01204FF0FF30204482569A420DD0F2
:104770000CEB01029145A1EB060200F095809045FB
:1047800001DD1846D9E7BEF1000F4CD1BBF1000F97
:1047900046D09323DFF828B1009300225B464549B9
:1047A0006420FDF7A3FFB8F1000F6CDD013EB146B8
:1047B00006EB080119F8013F93FBF5F205FB1232F5
:1047C0004945E254F6D10121992000223A4BCDE926
:1047D00004B0CDE9011203930091234642466420C0
:1047E000FDF732FF0AF1FF3316F8012FA256B1454B
:1047F00003F8012FF8D1012100249D252F48CDF881
:1048000010B003905346642042460595CDE901144B
:104810000091FDF719FF20460437BD46BDE8F08F33
:104820004FF0010B77E7012189200022224BDFF8AE
:1048300090B0CDE9011205900091CDE9033B4246CD
:1048400023466420013EFDF7FFFE06EB08010AF156
:10485000FF3316F8012FA256B14203F8012FF8D109
:10486000012400218D251548CDE901410390CDF8A3
:1048700010B0642053464246059500942146FDF74A
:10488000E3FE2046C8E70121992500200A4ACDE928
:1048900001100392CDF810B02346059500914246D1
:1048A0006420FDF7D1FEA6E79045BCDD4FF0010E78
:1048B000184642E71CAF010040AF01000CAF0100F9
:1048C000F0AE01002DE9F843D2F801600746727896
:1048D0000D46012A984618D9002814DD00244FF00F
:1048E0004C094D1E00E07278510094FBF1F301FB7E
:1048F000134315F8010F611009FB03830134FFF71F
:1049000003FEA742EFD1BDE8F8830028FBDD0024B9
:104910004FF04C09331993F915306110002B05DB6A
:1049200009FB03837278285DFFF7EEFD0134A7428F
:10493000F0D1BDE8F88300BF70B5644686B0DCF8FE
:1049400000200B4BFFF7BEFFD4E9012301214FF4F8
:1049500017760020074D084C1B68CDE9010005962D
:104960000091CDE903457220FDF76EFE06B070BDE3
:1049700014080460F0AE0100DCAE01002DE9F8433C
:10498000D2F801501E466A78012A1ED900281ADD85
:1049900001F1FF3821244FF04C0908EB000700E03B
:1049A0006A78510094FBF1F301FB134318F8010FEF
:1049B00004EBD47109FB03634910FFF7F7FD47458A
:1049C00004F1FF34ECD1BDE8F8830028FBDD0C4690
:1049D0004FF04C0905F1140808EB000718F9013FE6
:1049E000C8F13601294401EBD171002B4FEA610176
:1049F00005DB09FB03636A782078FFF7D7FDB8452C
:104A000004F10104EAD1BDE8F88300BF30B5644683
:104A100087B0DCF800200B4BFFF7B0FF40F2DD352C
:104A20000121002263680848084C1B68CDE9012277
:104A3000CDE903040595009114227220FDF704FED0
:104A400007B030BD98060460DCAE0100F0AE010096
:104A5000F0B4147980F8E8405579049C80F8E95066
:104A6000957980F8EA50D57980F8EB50957A80F8FE
:104A7000EE50157B80F8EF508D790E7880F88E50CF
:104A800090F8895045F0300580F8895090F8A15091
:104A90006FF3041580F8A150CD7880F8A950002E4E
:104AA00051D180F8986090F88B5045F0010580F85E
:104AB0008B500125072700264FF0060C80F88D70DB
:104AC00080F8B05080F8C56080F8815080F8805040
:104AD00080F8AEC080F8AF700D79002C80F884505B
:104AE000557CB8BF033480F89F50957CC4F38F0485
:104AF000DBB280F89E5080F89C60A0F8CA4080F835
:104B0000CD30D37C80F80031CB7980F805310B7A39
:104B100080F80A314B7A80F81031137D80F8DA3052
:104B200090F8A330917D61F3061380F8A33090F8DC
:104B3000A330D17D61F3020380F8A330537DF0BC34
:104B400080F8A0307047012580F8985090F88B507D
:104B50006FF3000580F88B50ABE700BF2DE9F047FD
:104B6000D0F80160D0F80930747882B06400D0F8D1
:104B70000D5033B10F46024619687878274BFFF77E
:104B8000A1FEB76B95F80DC08CB34FF04C093846B9
:104B90004FF0000809FB04790CF01F0C0CF0030E19
:104BA0004FEA8E1E4FEA9C0C002101F1100300EB2E
:104BB000430393F806A0DA790AF03F0A22F00702CD
:104BC00001314AEA0E0A42EA0C02112983F806A0D2
:104BD000DA71EAD190F84A3080F8488023F01F0358
:104BE00080F8498080F84A304C308145DCD13378F8
:104BF0002A78A9786878CDE90074FFF75BFC40F665
:104C00001400234600902A4631464FF04050FFF7EB
:104C10001FFF02B0BDE8F047FFF79AB81408046020
:104C200049F64043014411440331490093FBF1F13B
:104C300040F2A51070B501220026042588B008AB0B
:104C400043F8041D064C05900648CDE90126CDE940
:104C50000304114600956420FDF7F6FC08B070BD12
:104C6000F0AE0100CCAE01002DE9F04FD0F80130DC
:104C7000D0F80D605C785A798BB0650096F80380A7
:104C8000002A46D0D0F809209269002A41D0197D27
:104C900096F810B0DB68F1B14FF04C0E9446614AC3
:104CA0000CEB010A0EFB052E03F1FF3919F8013F49
:104CB0005B0865B110335B4A58001118CB799CF83A
:104CC00000704C3267F3C7037245CB71F5D10CF11C
:104CD000010CD445EAD1002D00F09E804C225149B0
:104CE0000B4602FB051283F825B04C339342FAD1F0
:104CF00001AF38462422002115F003F8B8F1020F65
:104D000021D0B8F1040F45D0B8F1010F52D00021E5
:104D10002AE001AF38462422002114F0F2FFB8F156
:104D2000020F10D0B8F1040F34D0B8F1010F41D008
:104D3000002DECD170783278B178FFF771FF3948E7
:104D40000BB0BDE8F08F002DF4D03B46552105EBAC
:104D5000C500384403F1090203F8011B9A42FBD154
:104D60009842F7D19DF804104FF0000C2D4C3846B6
:104D7000002301E010F8011FE2180133092B117222
:104D8000F8D10CF1010C654504F14C04D2DD17F8A3
:104D9000091FECE7002DCDD03B46AA2105EBC5004D
:104DA000384403F1090203F8011B9A42FBD1834204
:104DB000F7D1D7E7002DBDD0B9464FF0000EDFF890
:104DC00068804946DFF864C0002311E0012C05D15A
:104DD000032B03F0010201DC724506D003EBC30292
:104DE00008781CF8022002430A700133082B06D011
:104DF000022CEBD19E45F1D10133082BF8D10CF1F7
:104E0000010CE04501F10101DED10EF1010E754505
:104E100009F10909D5D1A5E72946242201A814F0F2
:104E200070FF87E7140804607D2C0020742C00209C
:104E30002DE9F04F83B04C230C4692F8018000AF6F
:104E40004FEA480603FB06F3ADEB030D0021914644
:104E500005461A4668467B609A4614F052FF69463A
:104E60005FFA84FC002E53D06B461A240DEB0A0027
:104E70005A781C7002F0EC0242F002025A704C3375
:104E80009842F5D1BCF1000F28D000204FF04C0B18
:104E90004FF0010E013D05E05369013023436045A9
:104EA00053611ADA15F8013F09EB030292F9152054
:104EB0001F2B0EFA03F40BFB0212EDDD147E203BD8
:104EC000A2460EFA03F3C4F301041C43013064F359
:104ED000010A604582F818A0E4DB86B100234C2566
:104EE0005524B8F1020F07D105FB0312D07C54748E
:104EF00020F001009474D07401339E42F1DC7A6892
:104F0000054814F0F3FE04480C37BD46BDE8F08FA9
:104F1000BCF1000FF3D0B8E714080460F0B5D0F886
:104F20000130D0F809701E7D87B0FD69BB6806B3FB
:104F300000224FF4807C14E0786835F8124050F875
:104F400022002402012838BF0120B4FBF0F0B0F5A4
:104F5000DC7F28BF4FF4DC7023F812000132B2422C
:104F600007D028880028E7D123F812C00132B242C6
:104F7000F7D140F20726002002254A78064C07495F
:104F8000CDE90100CDE903140596009501216420C7
:104F9000FDF75AFB07B0F0BDF0AE0100B0AE010066
:104FA0002DE9F04F97B0814606AFDFF8D8C16E4EBD
:104FB00007F11C0807F12C0407F10C05F960BA6130
:104FC00096E80F0088E80F00C8E9025C40462146D9
:104FD00007F16803FB63FBF753F996E80F00634E94
:104FE00084E80F00C4E90256204607F13C01FBF7B4
:104FF00047F9FB6899F80120D3F80160D3F80D5008
:105000007078D3F809A08001C7E9042A44F00104AC
:1050100006F0BEFCE98948F00105DAF800303A698B
:10502000CDE9004501F074FCDAE900013D69EB4689
:10503000EA1DAB0022F007020A33ADEB020D23F0AC
:1050400007037A690DF11808002DADEB030D7960A7
:10505000F368146906AED7F80CA014DD002205F140
:10506000FF3C9C44013B13F8011F18B110F801E00C
:1050700008F802E01CB154F8211046F822106345EC
:1050800002F10102EFD1F0B140F22122059200229B
:10509000CDE901220122364B11460092354A6420A7
:1050A000CDE9033243462A46FDF7CEFADAF801305D
:1050B000DAF80D10DA789AF800300132092B497BC2
:1050C0001ED0052B3ED094B10024042001214FF4C2
:1050D000107C0294CDE90001264C27483346CDE9E7
:1050E00003042A46CDF814C06420FDF7ADFA494602
:1050F000F868DD46FFF712FF4437BD46BDE8F08F84
:105100007B6840F64A30CDE903630091CDE9015850
:105110004FF4F0734FF4487101F0C2FC4FF40C7C73
:105120000420164A1349002304910121CDE90113FB
:105130007B6800900392CDF814C02A466420FDF7E6
:1051400083FAC0E77B6840F64A30CDE903630091FB
:10515000CDE9015882234FF4487101F0A1FC4FF4CE
:105160000F7C0420064ADDE7E89E01003949000073
:1051700054AF0100F0AE010068AF01005CAF010068
:1051800088B901004D460000F8B59B0003F10A0400
:1051900024F0070400AF002AADEB040DEC460CDD53
:1051A000BC69ACF10405013C224414F8016F51F8CC
:1051B0002660944245F8046FF7D11A46614614F010
:1051C00095FDBD46F8BD00BF10B5D0F80140D0F840
:1051D00009204B781169227DE46882B0084600946A
:1051E000FFF7D2FF02B010BD70B5D0F80150D0F873
:1051F0000940EE6882B04B782A7DD4E9031000960E
:10520000FFF7C2FF287D2269A16802B0BDE87040A7
:10521000FFF730B9D0F809304A7818699200D96898
:1052200014F064BD2DE9F047D0F80160D0F80930E2
:10523000747882B06400D0F80D5033B10F46024646
:1052400019683878274BFFF799FBB76B95F80DC0B5
:105250008CB34FF04C0938464FF0000809FB047935
:105260000CF01F0C0CF0030E4FEA8E1E4FEA9C0C44
:10527000002101F1100300EB430393F806A0DA7953
:105280000AF03F0A22F0070201314AEA0E0A42EA16
:105290000C02112983F806A0DA71EAD190F84A309D
:1052A00080F8488023F01F0380F8498080F84A3056
:1052B0004C308145DCD133782A78A9786878CDE9FB
:1052C0000074FFF7F7F84FF4D360234600902A46A6
:1052D00031464FF04050FFF7BBFB02B0BDE8F0474E
:1052E000FEF736BD980604602DE9F04FD0F8013086
:1052F000D0F80D605C785A798BB0650096F8038021
:10530000002A44D0D0F80920906900283FD01A7DA7
:10531000D96896F810E0E2B14FF04C0ADFF88891B6
:1053200001EB020C013811F8013B10F8017FC3F1C9
:10533000210393FBF5F205FB12320AFB029223F0E4
:10534000010320331344DA79614567F3C702DA7148
:10535000E9D1002D00F0A1804C2253490B4602FBFD
:10536000051283F825E04C339342FAD101AF384659
:105370002422002114F0C5FCB8F1020F21D0B8F1AD
:10538000040F45D0B8F1010F52D000212AE001AF3F
:1053900038462422002114F0B4FCB8F1020F10D0DA
:1053A000B8F1040F34D0B8F1010F41D0002DECD189
:1053B00070783278B178FFF733FC3B480BB0BDE82A
:1053C000F08F002DF4D03B46552105EBC500384445
:1053D00003F1090203F8011B9A42FBD19842F7D16D
:1053E0009DF804104FF0000C2F4C3846002301E0CC
:1053F00010F8011FE2180133092B1172F8D10CF1DA
:10540000010C654504F14C04D2DD17F8091FECE7E7
:10541000002DCDD03B46AA2105EBC500384403F151
:10542000090203F8011B9342FBD18342F7D1D7E76E
:10543000002DBDD0B9464FF0040CDFF8748005F1A3
:10544000040A49461948ACF1040E002312E0012C6D
:1054500005D1032B03F0010201DD964507D003EBD4
:10546000C30291F800B0825C42EA0B020A70013379
:10547000082B06D0022CEAD19C45F0D10133082B31
:10548000F8D10130804501F10101DED10CF1010CB0
:10549000E24509F10909D4D1A2E72946242201A84D
:1054A00014F02FFC84E700BF98060460742C0020E1
:1054B0007D2C00202DE9F04F83B04C23567800AFAF
:1054C000750003FB05F3ADEB030D9046834689465B
:1054D0001A46684600217B609A466C4614F011FC1F
:1054E000002D5BD06B4600200DEB0A015A78187036
:1054F00002F0EC0242F012025A704C339942F5D19C
:10550000B9F1000F2EDD00214FF04C0A4FF0010ED3
:105510000BF1FF3C07E05369013143EA0B0B89456E
:10552000C2F814B01DDD1CF8013F08EB0302C3F103
:10553000210092F915201F280EFA00FB0AFB0242F7
:10554000E9DD107EC3F1010383460EFA03F3C0F3D5
:1055500001001843013160F3010B894582F818B04E
:10556000E1DC8DB100234FF04C0C6FF05500022EA2
:1055700007D10CFB0342D17C507421F001019074DF
:10558000D17401339D42F2DC7A682146054814F05B
:10559000ADFB04480C37BD46BDE8F08FB9F1000FF4
:1055A000F2DDB0E79806046070B5D0F8092086B047
:1055B000D4699368218851B356689D1E301F3836D0
:1055C00001E034F8021F50F8042F0902012A38BF05
:1055D0000122B1FBF2F2B2F5DC7F28BF4FF4DC729E
:1055E000864225F8022FECD140F2C2350022022477
:1055F0000C480D49CDE90122CDE903100595009431
:10560000142201216420FDF71FF806B070BD4FF48D
:1056100080709A1E03F11C0122F8020F8A42FBD10E
:10562000E2E700BFF0AE0100B0AE01002DE9F04F9F
:1056300095B06F4E06AF07F11405DFF8D0C1B96021
:105640003A6196E80F0085E80F0007F1600307F163
:1056500024047B6307F10803C5F80CC028462146E3
:10566000AB60FAF70DFE96E80F00624E84E80F007B
:1056700007F10803C4E90236204607F13401FAF7BE
:10568000FFFDBB6844F00104D3F80160D3F8099032
:105690007078C7F80C90D3F80D8045F001058001B3
:1056A00006F076F9B8F80E10D9F800301422CDE9DA
:1056B000004501F02DF9357DEA46EA1DAB0002F404
:1056C000FC720A33ADEB020D03F4FF63F9680DF1D0
:1056D0001808ADEB030DF268D9E9000306AE7B6054
:1056E0000C69D7F8089085B10023013A12F8011F20
:1056F00018B110F801C008F803C01CB154F821100B
:1057000046F8231001339D42F0D100B340F28E32AF
:10571000059200224FF0010B374BCDE90122374AA9
:105720005946CDE90332CDF800B043462A466420FD
:10573000FCF78AFFD9F80130D9F80D10DA7899F81A
:1057400000305A440A2B497B1DD0062B3DD094B122
:1057500040F2AE34002001214FF0040C0594029079
:10576000264C27483346CDE903042A46CDE900C13B
:105770006420FCF769FFD546B868FFF715FF3C3792
:10578000BD46BDE8F08F7B6840F64A30CDE9036343
:105790000091CDE901584FF4F0734FF4487101F0D6
:1057A0007FF940F29E3C0420164A144904910021DE
:1057B000CDE901B159467B6800900392CDF814C041
:1057C0002A466420FCF740FFC1E77B6840F64A3078
:1057D000CDE903630091CDE9015882234FF448716C
:1057E00001F05EF940F2AA3C0420074ADDE700BF61
:1057F000E89E01000D4A000074AF0100F0AE010008
:1058000088AF01007CAF0100B8B9010095460000E7
:1058100010B5D0F80140D0F809200B781169227D2D
:10582000E46882B008460094FFF7AEFC02B010BDF9
:1058300070B5D0F80150D0F80940EE6882B00B780E
:105840002A7DD4E903100096FFF79EFC287D22698B
:10585000A16802B0BDE87040FEF70CBE4FF04053A7
:1058600093F84111D0F80930090401F1C041D8681A
:1058700001F58431502214F039BA00BFD0F8093054
:105880000A7818699200D96814F030BA2DE9F04707
:105890004C2692F8018000AF4FEA480406FB04F65C
:1058A000ADEB060D824689466846324600216D46BC
:1058B00014F027FA002C5ED06B461A200DEB06017F
:1058C0005A78187002F0EC0242F002025A704C331F
:1058D0009942F5D119F0FF012AD00AF1FF304FF0BB
:1058E0004C094FF0010E014405E05369814243EA3F
:1058F0000C0353611BD010F8013F93FBF4F204FB3F
:1059000012321F2B0EFA03FC09FB0252EDDD92F856
:1059100018C0203BE2460EFA03F3CCF3010C43EA35
:105920000C0363F3010A814282F818A0E3D1F4B1B9
:105930002B4655212E44B8F1020F05D1DA7C59745B
:1059400022F001029974DA744C339E42F3D100269E
:105950004FF04C080A4B08FB065118464C2214F035
:10596000C5F903460136B44203F15403F3D10448A8
:10597000BD46BDE8F08719F0FF01AED1F7E700BFE3
:105980004409046008B50520FEF7EEFB10B1D0F81D
:105990000930186908BD00BF08B5FEF7ADFC052049
:1059A000FEF7E2FB10B1D0F80930186908BD00BF5E
:1059B00008B5FEF7A1FC0920FEF7D6FB10B1D0F820
:1059C0000930186908BD00BF4FF0405393F84131CA
:1059D0004A78D0F8090003491B049200C0681944B2
:1059E00014F084B96808016008B50620FEF7BCFB16
:1059F00010B1D0F80930186908BD00BF08B5FEF72E
:105A00007BFC0620FEF7B0FB10B1D0F80930186916
:105A100008BD00BF8200014814F068B9A01700203B
:105A2000F0B4D0F809300B4E1C6906F1300735464A
:105A30000FCDBD4220606160A260E36006F11006F8
:105A400004F11004F3D107CE20606160A260F0BCC5
:105A5000704700BFA017002008B5FEF74DFC0A20D4
:105A6000FEF782FB10B1D0F80930186908BD00BFFD
:105A70002DE9F043002ADDE907EC21DD4C2707FB87
:105A80000EC7013901EB020811F8016FBEF1000FDA
:105A90004FEA8606C6F10A064FEA66060CDD644642
:105AA00010367600A519EA7993F800904C3469F322
:105AB000C702A742EA71F5D1414503F10103E3D1E1
:105AC000BEF1000F09DD4C2303FB0ECEC0B28CF8F3
:105AD00025000CF14C0CF445F9D1BDE8F08300BF72
:105AE000F0B40024D0F80D70D0F801C07D7BDCF854
:105AF000380005F01F0505F00306B601AD0804F1F6
:105B0000100300EB43039979DA7901F03F0122F0A9
:105B10000702013431432A43112C9971DA71EED115
:105B2000002290F84A3080F8482023F01F0380F8C4
:105B30004A3080F84920BC783D7863007A789CF838
:105B40000010DBB2EE18C67082700471447185716A
:105B500000297FD00A3A1344C371002401254FF075
:105B60004053447685763A7983F8E8207A7983F849
:105B7000E920BA7983F8EA20FA7983F8EB20BA7A37
:105B800083F8EE203A7B83F8EF209CF8062083F818
:105B90008E2093F8892042F0300283F8892093F810
:105BA000A12064F3041283F8A1209CF8032083F859
:105BB000A920002952D183F8981093F88B2042F045
:105BC000010283F88B204FF040530122002104246E
:105BD0004FF4F97083F88D4083F8B02083F8C51036
:105BE00083F8812083F880209CF8044083F8844067
:105BF0007C7C83F89F40BC7C83F89E4083F89C109B
:105C0000A3F8CA0083F8CD20FA7C83F800219CF821
:105C1000072083F805219CF8082083F80A219CF8C6
:105C2000092083F810213A7D83F8DA2093F8A32025
:105C3000B97D61F3061283F8A32093F8A320F97DC0
:105C400061F3020283F8A3207A7D83F8A020F0BCE0
:105C5000FEF77EB8033A1344C3717EE783F8985089
:105C600093F88B2064F3000283F88B20ABE700BF2E
:105C70002DE9F04FB0F1000885B0D2F801A046DD63
:105C800099464FF0000B4F1E4C239AF80160CBF160
:105C9000210404EBD4740BF00305012E4FEA6404D5
:105CA00003FB059517F8011F34DC324602A813F0F8
:105CB000F9FF46B3029B3F2B1946A8BF3F21039A29
:105CC000002B134401F03F01B8BF00213F2B1846C1
:105CD000A8BF3F20002B00F03F004FF00002B8BFEC
:105CE000002004F1100C05EB4C0C4AB3A318103340
:105CF00005EB430393F806E061F3050E83F806E035
:105D00000132B242F1DB0BF1010BD845BCD105B039
:105D1000BDE8F08F3046019105F03AFE044106FBE4
:105D200004F40F2C019906DD012202A813F0BAFF3A
:105D30000126029BBFE7324602A813F0B3FFB9E782
:105D40009CF8063060F305038CF80630D8E700BFF6
:105D5000F0B5D0F809308BB01968D0F80150DE6882
:105D6000D0F80D4021B102462D4B0620FFF780FFF1
:105D70006B7953B14EB101272A7DE968284D207C0B
:105D80003346CDE90075FFF773FE0022E378CDE9D5
:105D90000722012B8DF8242016D1224807AD0DF1E2
:105DA0002506002303EBC301415C0133082B42EAC3
:105DB0000102F7D105F8012BAE4200F1010001D03C
:105DC0002A78EEE79DF81C2007A80023144D01E077
:105DD00010F8012FE9180133092B0A72F8D149F69E
:105DE0004041A0786378227803EB400313440020FD
:105DF000053301225B00A226042591FBF3F40290F7
:105E000009490A480491039007AB0596CDE9005271
:105E1000114664200794FCF717FC01480BB0F0BD55
:105E2000C8070460742C0020A8AF010094AF0100E3
:105E3000F0B50546B3B068B3421E022A01D933B0AB
:105E4000F0BD03AF1C46BC4603F1400E6646206819
:105E50006168A268E368103474450CF1100C0FC639
:105E6000F4D15E26389B13AC186859689A68DB68D1
:105E70000FC4389B186959699A693B4607C4389A18
:105E80001A49908B2A4620800C6800960021012038
:105E9000A047D4E70E46144603AF0146BC2238465D
:105EA00013F02FFF31683846802213F01FFF24685B
:105EB00023AE04F1300C354620686168A268E368BF
:105EC0001034644506F110060FC5F4D120686168EE
:105ED000A268BC2407C60022044800943B4604681C
:105EE00011460120A04733B0F0BD00BFB0DF010074
:105EF000F8B50023114C1946236063603C2210481A
:105F000013F0FFFE00F02EFA4FF480620D4B0E49A5
:105F10000E4E0F4C9B68886030689A606368851CE1
:105F20009847A3680746984739460246284613F023
:105F3000DDFE236934689847E080F8BD542B0020CB
:105F4000D82C0020580A002034210020080A002004
:105F5000B0DF01002DE9F04F264C0E46217885B0C8
:105F600081420546DDE90E899246DDF840B020D039
:105F7000A378AB4202D005B0BDE8F08FE378002BE8
:105F8000F9D09B221C4B00921C4900226420FCF794
:105F9000ADFB2DBB4FF4F0600121F368184C246871
:105FA0000E902A460846A446039405B0BDE8F04F7B
:105FB00060471F466378002BDAD093220E4B009285
:105FC0000E4900226420FCF791FBCDF800B04B464F
:105FD00008F1100207F110012846FFF729FFC7E773
:105FE0006B1E022BC7D84FF470700121044C53462E
:105FF000D5E700BF542B002020B0010030B00100D5
:10600000B0DF01002DE9F04F5E4C87B0109D647940
:106010000495DDE91156039614B907B0BDE8F08F79
:1060200091460290A0228846574800219A4613F0D4
:1060300068FEB8220024554B009264200022544987
:10604000FCF754FB05F1FF3BA446524B4E48DFF8EA
:106050004CE1CDF814904FE0002A0CBF012202223F
:106060004FF487664270029A047032F91420049D3E
:1060700006FB02F28EFB02761644D217C2EBE62232
:1060800040F6241655F82450428038F91420C5F300
:10609000072706FB02F28EFB02961644D217C2EBCC
:1060A000E6228280059A32F81460EAB2BF1AC5F37C
:1060B0000742C2EB1565AF42C6804FF04D024BDD83
:1060C00002FB07F7BF1107814581039A3AF8145084
:1060D000125D85818273029A0CF1010C32F9142051
:1060E0001A8038F914205A8001340A2C197100F1F1
:1060F000100003F1060335D01BF8011F1A7900299F
:10610000AAD1002AF0D04FF48766B3F90050B3F952
:10611000022006FB05F540F6241606FB02F28EFB74
:1061200005678EFB02964FF003091644D217C2EBA7
:10613000E622039E047080F80190365D2F44ED172F
:10614000C5EBE725C1800181418181810CF1010C02
:10615000458082808673C7E702FB05F5AA1102819C
:106160004781B2E70C4BCDF840C01B680322029375
:10617000029C02210120A446034B07B0BDE8F04F6A
:10618000604700BF542B0020E817002020B001001A
:106190006CB00100D82C0020B0DF01008100088025
:1061A00010B584B003F026FE174B4279197891425E
:1061B00016D04479154AE4B21C70136803938CB965
:1061C00040F21F12124B0092124922466420FCF743
:1061D0008DFA02210094234622460846039CA047DC
:1061E00004B010BD40F21712094B00920A49002278
:1061F0006420FCF77BFA0023022100930846012269
:10620000039CA04704B010BDDC170020B0DF0100E4
:1062100020B00100ECAF0100D4AF010010B582B096
:1062200003F0E8FD437F93B14FF498720446094BA5
:106230000092094900226420FCF758FA002307481D
:1062400063771A460468009319460220A04702B0FB
:1062500010BD00BF20B001005CB00100B0DF010044
:10626000F0B587B003F0C6FD104CC37F22789A4288
:106270001AD0012200254FF4A277C67F0C490D4B9E
:10628000009204910393114623460597CDE90155E9
:1062900064202670FCF7D8F9074922782B460C6851
:1062A000009506210220A04707B0F0BDDE170020B0
:1062B00020B001000CB00100B0DF010010B582B0C9
:1062C000FFF7ACFFFFF76CFFFFF7CAFF002304499D
:1062D00000930C681A4604210120A04702B010BDAB
:1062E000B0DF010030B583B091B1838B028B1949C7
:1062F0001A446E2A0B781FDDB0F924001BB300246A
:10630000154A1460013BDBB202200B70106004E000
:106310000846114A0F4B11601970104C23788342C4
:1063200008D000230E49024600930D682070072113
:106330000220A84703B030BD0020074A1060002BA0
:10634000E0D11068E9E70123034AA0281360F8DDD3
:106350002323D9E7E4170020E0170020DD170020F1
:10636000B0DF010000487047881800204FF48060BB
:10637000704700BFF9F786BF13F0B8BC13F0C1BC7B
:106380000F2330B5012583B0054C00930022054B47
:10639000054964202570FCF7A9F903B030BD00BFA2
:1063A0001A29002010B1010020B101003C23F0B5F2
:1063B00005460E461446144F8BB0009300223B4610
:1063C000124964200994CDE90756FCF78FF94FF084
:1063D0003F0C0121002004220D4BCDE90110009259
:1063E0000393CDE9047C07AB03226420FCF72CF96E
:1063F000003418BF0124074B03EB450203F8156076
:1064000054700BB0F0BD00BF10B10100B4B001007A
:10641000E8B00100542B0020162330B583B00446A9
:10642000009300220B4B0C496420FCF75FF90B4AE8
:1064300040F2F1211346104623F8021B0C21256877
:106440006468C2F802505C6003B0BDE8304003F0FD
:1064500005BD00BF10B1010094B001001C33002045
:10646000004870473CB101001EF0040F0CBFEFF371
:106470000880EFF309808169004A104799F4000011
:10648000684620F007018D4601B401BC854670477F
:1064900072B61EF0040F0CBFEFF30880EFF3098013
:1064A000004A10471966000072B61EF0040F0CBFB8
:1064B000EFF30880EFF30980004A10471D660000E3
:1064C00072B61EF0040F0CBFEFF30880EFF30980E3
:1064D000004A10472166000072B61EF0040F0CBF80
:1064E000EFF30880EFF30980004A104725660000AB
:1064F000684620F007018D4601B401BC854670470F
:10650000684620F007018D4601B401BC85467047FE
:10651000684620F007018D4601B401BC85467047EE
:10652000684620F007018D4601B401BC85467047DE
:10653000684620F007018D4619B507232B4CB02083
:10654000237308F05FFF0021294A2A4BA1709A4269
:106550000CD2111D03335B1A23F0030326480B44AE
:1065600050F8041B42F8041B9A42F9D1234A244BE9
:106570009A420CD2111D03335B1A23F00303214806
:106580000B4450F8041B42F8041B9A42F9D11E4AEE
:106590001E4B9A420AD20020111D03335B1A23F0CE
:1065A00003030B4442F8040B9342FBD1EFF3088240
:1065B000174B9A4205D94FF0CD3143F8041B9A424C
:1065C000FBD84FF6FF72094B1A8708F01BFE08F044
:1065D00025FE1049002008F0C7FD044600F04EF8E3
:1065E000844200D0FEE70AF047FBFBE700001050B2
:1065F0000056002098560020800000000000002077
:10660000341200206CE0010034120020F42A002033
:106610005C340020FCFB0100704700BF704700BFE6
:10662000704700BF704700BF014B93F821007047CF
:10663000C0FB0100014B187E704700BFC0FB01008A
:10664000014B587E704700BFC0FB0100014B987E94
:10665000704700BFC0FB0100014BD87E704700BFF0
:10666000C0FB0100014B986A704700BFC0FB0100EE
:10667000014BD86A704700BFC0FB0100014B18688E
:10668000704700BFFCFB01002DE9F04F4FEA820B81
:1066900083B00BF10A0525F0070500AFADEB050D42
:1066A0006D463B604B68D1F80080064614468A462A
:1066B0007B60C0475A462846002113F022FB012286
:1066C00002FA06FB1BF1FF3B17D37B689847814614
:1066D000BBF1000F00D0C047002CF3DDAC46002119
:1066E0005CF8043B59F8042B013113448C424CF8FC
:1066F000043CF5D11BF1FF3BE7D2002C09DD294614
:10670000002251F8043B01323341944241F8043CE9
:10671000F7D1DAF808302946204698473A68DAF87F
:106720000C302946204698470C37BD46BDE8F08F0F
:1067300001322DE9F04191FBF2F404FB121282B018
:10674000DDE90A67DDE90C4512B102B0BDE8F08170
:106750002022804600921846DDE90812012305F048
:106760007DF8B8F1000FF0DD04EB48020FFA87FE68
:106770000FFA86FC08E0634655F8041B944203FBBD
:10678000101345F8043CE0D034F9023BB342F2DC8C
:10679000BB42B8BF7346EFE72DE9F04F1446984669
:1067A000D31D85B023F0070300AFADEB030D9500BB
:1067B00079608346002168463A6013F0A2FA05F139
:1067C0000A0323F0070341462046EA46ADEB030DDA
:1067D000BB6B9847FB6B9847E94601462A464846FB
:1067E00013F084FA002C40F38880434608EB040140
:1067F00013F8012B01328B4203F8012CF8D14146EA
:106800003868BB6B9847FB6B9847043D04384D4490
:10681000A9F10403514642464FF0FF0C4FF0010E20
:1068200008E0AB4281F800E01C6001F1010102F1D7
:10683000010211D050F8044F53F8046FA642F0DB68
:106840001478AB4204F1FF3481F800C0147001F1F8
:10685000010102F10102EDD13B685E1E56440AF1CE
:10686000FF334FF0000A1D46C4461C46012209E0D2
:10687000786888420FDB00228CF80010B4420CF1DB
:10688000010C0ED014F9011F0029F7D09CF800006C
:1068900001448B45ECDDB44284F800A00CF1010CFE
:1068A000F0D182BBC7E9023241463868BB6B9847DA
:1068B000FB6B9847D7E9023284469E4605E049F8CB
:1068C0002200AC4202F1010215D015F9011F002986
:1068D000F7D05CF8220059F822308342EFDB18F839
:1068E0000200AC42A0EB010108F8021085F800A0FC
:1068F00002F10102E9D17346B5E7BB6B4146386846
:106900009847FB6B98471437BD46BDE8F08F00BF32
:106910002DE9F04F012683B00138B2F100080D4691
:1069200000AF9B4606FA00F640F39880013B03EB6C
:106930000800F1B203F8011F8342FBD1761000F08A
:106940009D804FEA880AAAF10409C7F804A07C6B6D
:10695000D7F830A059464046D047A047B8F1000FBD
:1069600013DD5B465FFA86FC011F00EB090E51F850
:10697000040F1A78A842A2EB0C00D6BF624418702C
:106980001A70714503F10103F1D17610E2D1594635
:1069900040463B6BD7F804A098477B6B98470AF1B9
:1069A0000A0323F00703ADEB030DB8F1000F024615
:1069B0006C465CDD043C161F20463146AAF1040AF1
:1069C00002EB0A0C51F8043F5B1B8C4540F8043F76
:1069D000F8D1D9465B46304602EB0A0E50F804CF98
:1069E0001978AC4501F1FF3CD6BF013183F800C0F6
:1069F0001970704503F10103F0D1594640463B6BD5
:106A00007A6098477B6B98477A68924456F8043FBF
:106A100054F8042F5B1B002A83EAE371A1EBE371B6
:106A2000B8BF52428A420ADA99F80020002B02F1DC
:106A3000FF31D6BF013289F8001089F80020B24535
:106A4000236009F10109E1D1594640463B6B984763
:106A50007B6B98470C37BD46BDE8F08F76107FF40E
:106A600070AF3B6B5946404698477B6B98473B6BF2
:106A70005946404698477B6B9847E5E7594640465C
:106A80003B6B98477B6B98474FEA880A0AF10A03E9
:106A900023F00703ADEB030D02466C468AE700BF07
:106AA0002DE9F04F83B00D9EDDE90F9C002E40DDF7
:106AB000DFF88480DF021D0388FB073B88FB053875
:106AC0000E9BFF17ED17013B5200C5EB6815002424
:106AD00000EB01084FF47A7E41F2301AA7EB6B17F6
:106AE0001E44411A01921AE008FB00FB59F82400E9
:106AF000019A381890FBF2F00EFB00F090FBF5F0D5
:106B00000EFB0BFB0AFB00F00C9A9E4202FB10B03E
:106B100090FBF1F04CF8240004F1010409D013F8C3
:106B2000010F0028E0D19E424CF8240004F101043A
:106B3000F5D103B0BDE8F08F1F85EB512DE9F04F83
:106B400017469A460646850097B02A46DDE9214950
:106B500008468846002113F0D4F82A46002138461A
:106B600013F0CFF872000021504613F0CAF83246F5
:106B70000021209813F0C5F82A464846002113F05A
:106B8000C0F8002E40F39980209BCE460993002345
:106B90000193249B221FC3EBC3730F925B002A4413
:106BA000CDF814A00B9711920E93CDF818800F9B7F
:106BB00053F8041F0F934FEA116BC1F307435B4572
:106BC0000C9156D80123249A26989A400BFB020276
:106BD0000292DDE924200BFB02020792019A934006
:106BE0000A93CBB20093C1F307230D930D99009B39
:106BF00099422FDB079B4FF0010C5E18DDF82C80CB
:106C000005E090065CD4009B01398B4222DC16F82B
:106C10000129019B9A42F4D1029B069C33F9112071
:106C20002368059D01FB023328882360D8F80030D3
:106C300010440BFB0233C8F8003028800998037811
:106C40009342E0DAFF2AA8BFFF22009B01398B4262
:106C50000270DCDD029A0E990C9B0A440292249980
:106C6000079A0BF1FF3BC3F30743521A5B450792A8
:106C7000BCDD059BB3F900205AB106990B685B0295
:106C800093FBF2F30B600B990B685B0293FBF2F240
:106C90000A60019B0F9A01330193059B0233059310
:106CA000069B043306930B9B04330B93099B013320
:106CB0000993119B93427FF47AAF17B0BDE8F08F30
:106CC00000234FF601701C464A4D16AF2D7847F849
:106CD000040D03952598484D0493149500EB010A83
:106CE00002F00F05089245FA03F0C2071AD514AA5C
:106CF000D056249A584402FB00A013F90790039A37
:106D000010F809900CFA09F0914540EA040009D204
:106D1000A04207D0049A044616A81044013200F895
:106D20000C9C04920133042BDDD10A9B089A1C426F
:106D30003FF469AF029B33F911300893D30613D4A3
:106D40009DF804307370069D08982B68059F01FB21
:106D500000333A882B60D8F8003002440BFB003334
:106D6000C8F800303A804EE74FF00009049B0DF15F
:106D70004B005A1E914500EB03070DF14C0A1846D3
:106D8000CDF840B01CDA09F10109484514DD54463C
:106D90009AF800B0039214F8013F9B452ABF1D46A4
:106DA0005D465B465EF825200CFA03F31343A742C9
:106DB0004EF82530EFD1039A91450AF1010AE2DB42
:106DC000049BDDF840B0032B0BD0042B05D0022B25
:106DD000B9D1089B5B100893B5E7089B9B100893FB
:106DE000B1E74AF6AB23089A03FB02F35B1408935E
:106DF000A9E700BF54B10100000001FF0288014B68
:106E00001A8070478C1C00202DE9F0414FF4614C32
:106E10004EF2B057184C069E94F8008094F801E0AA
:106E200006EB410611F1FF3123D336F9024D002C58
:106E3000F8D053F8215032F9214068B905F5807532
:106E400004F58074B8F1000F01D0C5F5F055BEF11E
:106E5000000F01D0C4F580440CFB05F507FB04F4DA
:106E60002D14241442F8215043F8214011F1FF3130
:106E7000DBD2BDE8F08100BF8C1C00202DE9F84377
:106E8000984604460F46164602F0B4FF437A40F691
:106E9000FE72022B14BF0D25002544F2507E49F6E8
:106EA0004E3CC5F57F6108EB04030F31A2EB0508EA
:106EB00014F1FF341FD313F8010D0028F8D037F96F
:106EC000140036F914900CFB00F000149042A8BF97
:106ED00010460EFB09F94FEA29494D4520EAE070BA
:106EE0000BDA4945D8BFC14627F8140026F814909C
:106EF00014F1FF34DFD2BDE8F883A946F4E700BF00
:106F00000288014B1A807047901C0020002318490A
:106F1000184A70B41848194E194D1A4CC1E900337B
:106F20000B81C2E9003318491381184AC6E90033BE
:106F3000C6E902333361C5E90033154EC5E90233B2
:106F40002B61C4E90033C4E902332361C0E9003393
:106F5000C0E902330361C1E90033C1E902330B61C7
:106F6000C2E90033C2E902331361337070BC704769
:106F7000CC2000201C200020A02000202820002061
:106F80003C20002078200020642000205020002099
:106F9000C82000202DE9F04F8BB09DF854607A4C4A
:106FA000CDE9026027786578784C01932478029BBC
:106FB00092469C4238BF754A0E468DF824708DF873
:106FC000255038BF1370149D092404F0C7FE039B9D
:106FD0000490DFF8D091DFF8D081DFF8D0B12544FC
:106FE000123603F1120739E018F804300AAA0A44ED
:106FF00012F804CC0133DBB265489C4508F8043034
:107000004FEA440230F914003BF914E0009745D2EE
:107010000023297808F8043009F804105D4B9852D1
:107020005D4B5B4823F802E0009BB3F900308352CC
:10703000B6F9003059482BF802303AF9143083522F
:10704000019B574833F914308352013C631C05F807
:107050000119A7F10207A6F102063CD005F086FC53
:1070600058B13AF91430002B07DDB6F90030B3F50A
:10707000007FBCBF01238DF8243019F804102B7851
:107080008B42B1D10023620008F80430404B3BF939
:1070900002E0985E039B13440093BFE7002BBDD032
:1070A0009DF858302BB92B781BB9384B1B78012B26
:1070B00018D038803BF902303380384B01989B5E02
:1070C0002AF81430364B9B5E20F8143018F8043040
:1070D000002BBAD1DAE7029B0BB92C4A13700BB024
:1070E000BDE8F08F049B132BE3DC2A4B9B5E0093DF
:1070F000294B33F902C0009B13B9BCF1000FD8D063
:10710000009BC31A002B0693B8BF5B420593AEEBFE
:107110000C0300930793059B772B2EDD41F6CC0CD7
:10712000A0F1C9039BB26345C3D86FF4C87343F29F
:107130004A6C73449BB26345BBD841F65C2C069BFA
:1071400003EB430303EBD37300EB63030093013BB7
:107150006345AED8079B03EB430C0CEBDC7C0EEBDA
:107160006C0E43F66A1C0EF1FF336345A1D8BDF8DF
:1071700000303B80A6F800E09FE7009B002BB8BFE3
:107180005B42772B95DDC9E7901C0020C8200020CA
:1071900078200020282000203C20002064200020AF
:1071A00050200020CC2000201C200020A020002007
:1071B000F8B505461A4C0146B022204612F096FD5D
:1071C0002E1D04F15C0C0FCEACE80F000FCEACE826
:1071D0000F0096E8030005F1300704F188068CE8FB
:1071E00003000FCF0FC60FCF0FC697E8030086E846
:1071F000030005F18807261D0FCF0FC60FCF0FC65E
:1072000097E803005C35303486E803000FCD0FC4E7
:107210000FCD0FC495E8030084E80300F8BD00BF5C
:10722000941C00202DE9F84F92460F461D46044657
:1072300002F0E0FD834604F091FD9BF80920012A4D
:1072400032D0414E05EB440506F1300906F1040841
:1072500014F1FF3428D335F9023D002BF8D057F84C
:107260002430B26D93423DDA9BF8091002295FD1B8
:107270007F209B1A00FB03F302EBA31247F82420A4
:107280005AF824103368994210DA9BF80920022A30
:1072900046D17F20C91A00FB01F103EBA1134AF884
:1072A000243014F1FF34D6D2BDE8F88FF36AC1F56B
:1072B000E0519942CCDA9BF80920022A42D008B268
:1072C000494604F037FB5AF82410F36AC1F5E0513F
:1072D000C91A00FB01F103EBA113C3F5E0534AF80F
:1072E0002430B5E7D6F88420C3F578539342C7DA43
:1072F0009BF80910022923D018B2144904F01AFB94
:1073000057F82430D6F88420C3F578539B1A00FB35
:1073100003F302EBA312C2F5785247F82420AFE73B
:1073200008B2414604F006FB33685AF82410B1E76E
:1073300018B2074904F0FEFAB26D57F8243098E706
:107340007F20E3E77F20C3E7941C00201C1D002062
:10735000F01C00200346997A254A0078012930B4B0
:1073600010701FD0197C01290BD009B92148017078
:1073700053F8120F20491B79C2F812000B7130BC70
:107380007047D089D989884220D0194651F80C0F0E
:107390001A4C8988D060A1800120022415491C74F0
:1073A0000870E5E710891989884214D0194651F808
:1073B000025F13484C680989C2F802504460018199
:1073C000002002240B499C720870CBE790899989B0
:1073D0008842DAD1E0E7D088D9888842E6D150885F
:1073E00059888842E2D1908899888842DED1E7E7BF
:1073F000441D0020A02B0020561D0020501D002001
:10740000461D002010B4314C314B04FB00F49C426B
:1074100029DB4FF4876202FB00F02E4AA2FB003208
:10742000801A02EB5002D20A40F6241303FB01F14A
:10743000284B294CA3FB01032078C91A03EB510305
:10744000DB0AD0B9A27C002A36D0B4F813209A42C5
:1074500038DCB4F8152010BCC2F5126204329A422E
:10746000B8BF032070471D4AE31782FB040214448F
:10747000C3EBE42404F58762D6E71949097891B98A
:10748000E18891421BDCA188914201DD642B19DC6B
:10749000218991420DDCA27C012072B1B4F8132045
:1074A0009A42D6DD0EE0A18991420BDCE18991423E
:1074B000F1DD022010BC7047104610BC7047618897
:1074C0009942E0DA032010BC704700BFC8FBFFFF01
:1074D0001E32DEFF01011000441D002081000880E3
:1074E000A02B0020F0B49DF81840079D022C25D059
:1074F000032C19D0012C02D00020F0BC70473B4B6C
:107500005B5D002B41D10922394B3A4EA3F10A05AC
:1075100013F8011D022908BF9455AB4202F1FF3256
:10752000F6D1F0BC01207047304B5B5DA3B1324B0C
:107530005B5D023B012B0FD90420DEE72B4E765D0D
:1075400086B12D4E765DB71E012F2DD92B4A042012
:1075500052F82530013314E00122264B03205A55FE
:10756000F0BC7047264C274E24F815002648274CBF
:1075700020F815300220012324F815201F4A26F890
:10758000151042F82530F0BC70471B4B5B5D022B99
:10759000C7D11A4B53F825302F2BC2DC1C4A1D4B88
:1075A00054551C702046A8E7032EDBD044F6C46671
:1075B000144A134B32F9152033F91530891A01FB9F
:1075C00001F1C01A00FB00100C4AB04252F825101D
:1075D00001F1010308DD2F2906DC01210D480C4CC7
:1075E000017061550420CCE72046CAE7D02B00206B
:1075F0007A2B002018340020702B0020482D00200A
:107600000034002024340020282D0020A42B00204A
:10761000C42B0020183300202DE9F04F00248FB038
:10762000CDE90C23804BCDE90A011C7002F0E2FB8E
:10763000437A002B56D17D4B1A78002A4FD0002375
:1076400009931C460A9B189DA3F102090B9BA3F109
:1076500002080C9BA3F1020B0D9BA3F1020A22E08E
:10766000734A125D022A00F097800023714A135575
:107670006F4A13552B78704A1355BDF814300134F6
:10768000A9F80030BDF818300A2CA8F80030BDF871
:107690001C30ABF80030BDF82030AAF8003005F8F7
:1076A000016B00F09180002739F9023F059338F90A
:1076B000023F06933BF9023F07933AF9023F0893D2
:1076C000199B1F555D4BE7542E78002E32D15A4B33
:1076D0001B5D002BC4D1564A1E461355CBE79B7C3D
:1076E000002BACD10023564ADFF860E1DFF860C11F
:1076F000544F524E4E4D504C4E48534902F11408CF
:1077000022F8023B42452EF8023B2CF8023B27F8B8
:10771000023B06F8013B05F8013B04F8013B00F889
:10772000013B41F8043BEBD10023099309980FB0CA
:10773000BDE8F08FBDF81810BDF81400FFF762FE29
:107740000A23199ACDE90204DDE90501CDE90032E9
:10775000DDE90723FFF7C6FE042830D0012804D94D
:107760003E46334B18552B7885E7314B1B5D022B7A
:10777000F7D10128F5D1334B344933F91430344A69
:1077800008932F4B31F9141032F9142033F91430C7
:10779000069107920593E4E72B4A52F824202F2AFA
:1077A0003FF763AF234A125D002A7FF45EAF1E46A7
:1077B00009930123199A13551B4A137055E71C4B63
:1077C0001B5D022BCDD1D6E7174B1B78002BADD01C
:1077D000DDE90ACEDDE90C89DDE918AB00230127DC
:1077E000164A174E194D1A4C164812F8011B11B9BA
:1077F0001BF8031089B136F913102CF8131035F962
:1078000013102EF8131034F9131028F8131030F950
:10781000131029F813100AF8037001330A2BE4D16E
:1078200009980FB0BDE8F08F18330020441D0020E8
:10783000702B002018340020D02B0020C42B0020F7
:1078400000340020282D0020482D00202434002062
:10785000A42B002001465422014812F047BA00BF71
:10786000E80700200021044B03F1780299600C33F3
:107870009342FBD1704700BF883300202DE9F04FC1
:107880003F4F85B03C68DDF83880012C08BF0022EE
:1078900000295AD04FEA400A0AEB0001394D89000D
:1078A0006E18B4680A2C59DDD3F800C00AEB000149
:1078B00005EB810149680AEB00094FEA8909044692
:1078C00055F809001E46D8F80030ACEB0000591AF4
:1078D0000028B8BF40420029B8BF4942039203F0D4
:1078E000D3FF039A834607EB0217D7E9022379688F
:1078F0003F69009703F0B2FF05EB090700283BD072
:10790000326855F8093002FB0BF203FB00230BEB46
:10791000000251100B4493FBF2F33360D8F80030AF
:107920007F6803FB0BFB07FB00B0084490FBF2F001
:10793000C8F8000033685444A4002B51D8F8003034
:107940002C44636005B0BDE8F08F0E4B00EB4000A7
:1079500003EB8000816005B0BDE8F08F0134B460B6
:10796000012CD3F800C0A1D145F801C0D8F800100F
:107970007160D3F800C09EE7D8F80000D8E700BFD8
:10798000E80700208833002030B40546064C6968BB
:10799000AA68EB6800680FC428696969AA69EB697D
:1079A0000FC430BC704700BF5C1D00202DE9F047BC
:1079B000DFF8C0800021D8F804208146920012F040
:1079C000A0F9D8F80430D8F81020581EA0EB6300B6
:1079D0009047D8F814309847D8E9006486B3671EFA
:1079E000002C37D009EB8404013ED8F818309847B2
:1079F00082469FB3D8F804007D1EA5EB6000D8F83E
:107A000010309847FE4202D0D8F814309847D8F882
:107A10001C30504698470022831E3E3033F9021F27
:107A200098420A44FAD154F8043D2F469A42B8BF0E
:107A30001A466B1C2260D8D1D8F80440002ECED153
:107A400004EBD4706410D8F81030C4EB6000BDE8CB
:107A5000F0471847013EF3D0013EBFE7D8F80420B5
:107A6000D8F81030501EA0EB620098474FF0FF3559
:107A7000C8E700BF5C1D00200E4BF0B45F68022F0A
:107A800015DD00EB87070C3F0438024600230A4946
:107A900000F10C0652F8045F11F9014B964205FB08
:107AA0000433F7D11B1140F8043F8742EDD1F0BCFD
:107AB000704700BF5C1D0020681D0020DFF868C013
:107AC000F0B4DCF804600024002E0ADD01EB860629
:107AD000043E0B1F53F8045FAC42B8BF2C469E42D5
:107AE000F8D1DCF808304610A34214DA002818DD7B
:107AF00000236FF00045043951F8044FAC42B8BF81
:107B00001F4603F10103B8BF25469842F4D1B81BC4
:107B10001560F0BC704751F826300020F0BC1360AF
:107B200070476FF00045F2E75C1D0020F0B404469A
:107B3000074E00F13007354620686168A268E368A7
:107B40001034BC4206F110060FC5F4D1F0BC7047EA
:107B50007C1D00202DE9F047DFF8E89002EB40059E
:107B600099F82C3099F82D2082B0441E0F468DF8DC
:107B700004208DF805304E464FF0000A4FF064089F
:107B800000E0013C631C17D035F9023D002BF8D012
:107B9000314637F9140003F0CDFEB5F900309842B4
:107BA0003EDBD9F8282008FB03F302FB00F29342E6
:107BB000C8BF4FF0020AE4E71F4B1878BAF1000F74
:107BC00013D11E4AC2F800A060B91D4999F82E4091
:107BD0000A680132A2420A6004DD01221046C1F89F
:107BE00000A01A7002B0BDE8F0870546AAF10200B5
:107BF000B0FA80F04009854217D0104C02A92268E3
:107C0000014411F8041C01328A42226011DD002275
:107C10001870226000220A4B1A6002B0BDE8F0879B
:107C20000020054B1D788542E7D10022034B1A60E6
:107C3000F0E72846EEE700BFE4200020D82000202F
:107C4000E02000207C1D0020014B1870704700BF11
:107C5000E4200020034B1B781BB9034A136801334F
:107C600013607047E4200020E02000200278014BE0
:107C70001A7070473C0800200022034B83F8F02064
:107C800083F8E421704700BF702D00202DE9F04FEC
:107C9000614D97B02C78002C69D000296BD0F4246A
:107CA00004FB00F4DFF874811E4608EB040C9CF81A
:107CB000F0301746FF2B68D00133DBB28CF8F03080
:107CC000D2F800E0D6F8009004F1D00B012BCDE9FA
:107CD00004E9C34461D00DF1100900234FF4807A08
:107CE0005A460EA808EB040B4946CDE90633039328
:107CF00000F096F80EAA06A9584600F045F9039B35
:107D000059461A46CDF800A00123484600F092FAE1
:107D1000012304F134011A460A904144CDF800A031
:107D2000484600F087FA04F168010B9041444FF493
:107D3000C8730222CDF800A0484600F07BFA04F197
:107D40009C010C90414449F640430122CDF800A02B
:107D5000484600F06FFA06AA0D900AAB594608A8EB
:107D600000F026FADDE908232C783A6033602046DB
:107D700017B0BDE8F08FF422284B02FB00332046F9
:107D800083F8F01017B0BDE8F08F1268336804F183
:107D9000D00BCDE90423C3449DE74FF0000A6146B0
:107DA000524653468CF8F1A08CF8F2A00132042A16
:107DB000C1F800E0C1F80C904B600B618B60C1E929
:107DC0000533C1E90733C1E90933CB6201F134015D
:107DD000ECD1F4214FF4C863FA2201FB00800DF1CD
:107DE000100902634266C0F89820C0F8CC20836175
:107DF000C3648365C0F88030C0F88C30C0F894301C
:107E0000C0F8B430C0F8C030C0F8C8304946584651
:107E100000F0A6F861E700BF3C080020702D0020AC
:107E2000F0B413680F684E685568DC1BAD1B002C5E
:107E3000B8BF6442002DB8BF6D422C44C82C84B03A
:107E400004DC4EF660251389AB4274D90125C2E9E2
:107E50000076D1E90034341B2E46FF1A002FB8BF3C
:107E60007F42002CB8BF64423C44134694FBF5F5B6
:107E7000002123F8086F02F11C0633F8024FA142DB
:107E8000B8BF21469E42F8D1937FA942B8BF294688
:107E9000082B02EB43048CBF0023013305296581C5
:107EA000937722DD27294ADC294B4A1F03FB02F284
:107EB000284BD41783FB02531344C4EB631303F220
:107EC000CA341429009413DD31293DDC6FF0D1024E
:107ED000143902FB01F1204ACB1782FB01520A44FC
:107EE000C3EB221303F28E3304E040F2CA34009451
:107EF00040F28E3301934FF42F730146CDE90233E4
:107F0000164F00F1280601ADC4F57A7287FB02C353
:107F1000A3EBE2739BB200F1080220F8023B82421D
:107F2000FBD121F80A4B8E4202D055F8044BEBE707
:107F300004B0F0BC704701339EB2354695E74FF46C
:107F40002F7431290094C1DD4FF42F73D2E700BFA5
:107F5000F2FEFFFFEBA00EEA89888888565555553A
:107F600070B4D1E90062034600256424C0E90062D0
:107F700000F11C0223F8085F23F8024F9342FBD163
:107F800070BC0023837770472DE9F04F0C46924672
:107F9000CFB003900146D0221AA8A4F1020B11F031
:107FA000A5FE5D46D6465046A046804F0AF108061B
:107FB000002213461AA930F833C00C6B0133042B8E
:107FC00004FB0C2201F13401F5D1B2F5FA6F34BF94
:107FD0000122A7FB023200F1020028BFC2F38F1278
:107FE000864225F8022FE3D144460023A11D8C468A
:107FF000CDE90633CDE908330AF1200A0DF1240951
:108000000DF1680806AA15464F465C467646D8F834
:108010003010029236F8022B34F8020F01FB02F204
:10802000B2FBF0F2A445134445F8043B47F8042F93
:1080300001D02B68EEE70EF1080EF24508F1340886
:1080400009F11009069BDDD1002108460C461AAD46
:1080500005F1D00C2A6B2F68EE683435AC4511441D
:1080600007FB024406FB0200F4D194FBF1F490FB01
:10807000F1F1039A10461460D160934604229046B1
:10808000CDE9040300218C460F460E460C460846F7
:108090000AAB019303EB080E1AAA00915EF8103B9D
:1080A0001168D2F8089001FB0300D168D2F814A03F
:1080B00001FB0344516809FB03CC01FB0366116912
:1080C000343201FB0377009995420AFB03130093B6
:1080D000E4D1194606AB53F8083008F1040890FBC8
:1080E000F3F094FBF3F496FBF3F697FBF3F79CFBAA
:1080F000F3FC91FBF3F1B8F1100FCBF83400CBF89F
:108100004040CBF83860CBF84470CBF83CC0CBF89B
:1081100048100BF1340BB5D1DDE904430399D0319C
:1081200003910025A846AE46AC462F462E46DDF804
:1081300004901AA9009359F8100B8B69D1F82CB050
:1081400003FB0066CB690BFB005503FB00770B6A52
:1081500003FB00CCD1E9093A34318A4203FB00EE3B
:108160000AFB0088E7D1009B96FBF3F697FBF3F739
:108170009EFBF3F09CFBF3FC98FBF3F195FBF3F50E
:10818000019BC4E9066704330193039BC4E908C05B
:10819000C4E90A153434A34204D0029951F8043FCB
:1081A0000291BEE74FB0BDE8F08F00BFD34D621023
:1081B0002DE9F0438C460C460026DFF87480971EAC
:1081C000043B063237F802EF53F8045FBA4205FB6E
:1081D0000EF5A8FB059ECCF8305006EB9E160CF170
:1081E000340CEFD101250A46D031136B3432B3FB86
:1081F000F6F3002B08BF2B4642F8043C9142F4D121
:1082000000210D460E46236BD4F800C0E7683434D5
:10821000A24219440CFB036607FB0355F3D196FBFE
:10822000F1F695FBF1F1C0E90061BDE8F08300BF14
:10823000D34D62102DE9F04FD2B28BB0012A0192DA
:10824000044600F05881C0F02881022A00F09D8089
:1082500000234FF480629C461F461D469E469B4667
:108260001E46984699469A46CDE9073305920393F0
:108270000293069304930093039AD4E90004A4EBB9
:10828000090406FB04290BFB0433A0EB0A0043F3AB
:10829000951308FB00EE06FB00550BFB007708FB6F
:1082A00004CC49F39519C1E90493029B4FEAAE2E21
:1082B0008B61019B45F3951547F395174FEAAC2C5D
:1082C000C1E900E5C1E9027C002B00F0E080009AE2
:1082D000059B764203FB02F3069A002B4FEA822AA3
:1082E000009AB8BF03F2FF3306FB02AABAF1000FEF
:1082F0004FEAA323B8BF0AF2FF3ACB614FEAAA23A1
:108300004B62019B022B00F037810023C1E90A3345
:108310000B6204FB04F400FB0040A94B984200F3FD
:10832000AE80642404FB00F0149BA64A90FBF3F497
:108330006310934200F3A38042F21071A24AE41743
:1083400082FB0302C4EB223201FB12309F4D561C0C
:1083500080EAE07401FB1633A4EBE07435F81600F4
:10836000002B00FB04F035F81220B8BF5B4202FB83
:108370000300974FA7FB0030400B01FB00F0149B5C
:1083800090FBF3F00BB0BDE8F08FD1F82090D1E96D
:1083900006073D1809EBD970D1E90ACED1F824A01F
:1083A00005EB60050EEBDE7809EB0C064FEA68087A
:1083B0000CEBDC7B3D4406EB08024FEA6B0B5744A9
:1083C000554404925F445D4402EBD27B8A684F447B
:1083D00003924A69674409920A687344914605EB1F
:1083E0006B05079307EB080300932B4648680AEBDD
:1083F0004C0A0290029AF24409EB2219039ACDF832
:1084000018A009EB621A099AD1E9036006EB20165D
:1084100006EB6219002D149AB8BF05F10F0302EBA9
:1084200023134FEA851898FBF3F8009A14939601EA
:10843000049AC8F580634FEA821B149A059396FB51
:10844000F2F69BFBF2FB029A03FB05F31546099F2C
:10845000002B3844F444039AB8BF03F2FF33800181
:10846000CDF820C003909812099B1544AD010290ED
:1084700097019B014FEA8A2E4FEA892CFCE642F2D3
:108480001070149B90FBF3F00BB0BDE8F08FC1E9C6
:108490000733C1E90933CB623BE78869149A034487
:1084A0001846002BB8BF03F10F0002EB20124FEA71
:1084B000831898FBF2F81492C8F5806202FB03F06F
:1084C00000230028D1F800A0D1F80C90B8BF00F22A
:1084D000FF3005928212CDE902231F461D469B46BE
:1084E0001E46CDE907330693049300934FEA8A2E84
:1084F0004FEA892CC0E6486AD1E9065605EB460EDC
:10850000864403440693734632184D6800920A6805
:108510000F6902EB251ACA68BEF1000F02EB27199A
:10852000149AB8BF0EF10F0302EB23134FEA8E1813
:1085300098FBF3F81493C8F5806303FB0EFE0593D4
:10854000009BBEF1000F4FEA8316149BB8BF0EF2DA
:10855000FF3E96FBF3F600234FEAAE220292BA01E9
:10856000AD0103921F469B46CDE9073304934FEAC2
:108570008A2E4FEA892C7FE6DDE9042303FB02F310
:10858000089A002BB8BF03F2FF334FEA822C9B12EC
:10859000049A0B62079B06FB02C6049A9B020BFB24
:1085A000123B002EB8BF06F2FF36BBF1000FB8BF7A
:1085B0000BF2FF3BB6124FEAAB238E62CB62A8E60A
:1085C00014AE47016F110100AD8BDB6860B1010093
:1085D0005917B7D130B40546044C00686968AA68D9
:1085E000EB680FC42869206030BC7047AC1D0020C8
:1085F0000268014B1A607047C01D00200146B0227E
:10860000014811F073BB00BFC41D00202DE9F043E9
:108610000746032200204FF0010803FB07F6079DE1
:10862000104C29448E5D94F80090DFF83CE0DFF8B0
:108630003CC006F00F0646FA02F4E4070CD512F926
:108640000E4012F90C503C4403FB0414645D4C458D
:108650003CBF08FA04F4204312F1FF32EBD2BDE82C
:10866000F08300BF58B1010070B1010078B1010082
:108670002DE9F04F8DB0189F0546059097F802B090
:10868000F87888468345CDE90832DDF870A04DDCE6
:108690000123B8461E9C0BFA03F20AFB0242049225
:1086A0001D9A97F801900BFB0A2603FA05F28B40FE
:1086B000134303934FEA4A030693EBB2CDE90A133F
:1086C000079298F800404C450CDD23E0FA0606D4EA
:1086D000079B834200F09780002800F0B1800134AE
:1086E000A14515DB375DB906F9D51D9B1B9A009393
:1086F000214653465846FFF789FF039B8342E5D145
:108700009DF81430335598F801900134A145E9DA09
:1087100098F80300049B069A0BF1010B134458458B
:1087200056440493CDDA4746DDF8288019993B6812
:108730000846059A40F8223050F828309400C3F3D8
:108740000741B1EB136F4FEA88003B6019DC944698
:108750001D9B97F801900AFB01353B7899450BD397
:108760002B4413F8016B464504BF03F801CC97F87E
:1087700001905A1B9145F4DAFB7801318B42554444
:10878000EBDA1A9B08F101011844099B8B420FDDBB
:1087900001279C461A9A059D161952F82550026821
:1087A00007FA01F3134001311D438C453560F6D1C2
:1087B00000231A9A984542F8283040F3838001221A
:1087C000059F1A9802FA08F10444BC4602FA07F021
:1087D000CD4316461A9F06E002432A4047F823205D
:1087E000013398456ED057F823200A42F8D09C45B3
:1087F000F2DCF2DA226806FA03FE42EA0E02226096
:1088000057F82320E9E79DF8143008983355049B66
:1088100098F8019033F91420036804FB02F103EB8C
:10882000412303600BFB02F1169B1B6803EB412302
:1088300016990B60179B1B681344179A13604EE739
:1088400007F00F03CDF860800325984648FA05F33A
:10885000DB072FD51D4B1B9AEF561D4B5F4415F9B7
:1088600003901D9BA1440093384653464946FFF7A9
:10887000CDFE039B83421DD11D9B0B9A0AFB07373C
:10888000049B07F80920325533F91420089804FB9B
:1088900002F1036803EB412303600BFB02F1169B1B
:1088A0001B6803EB412316990B60179B1B6813444D
:1088B000179A136015F1FF35C8D2DDF8608098F87B
:1088C00001900CE70DB0BDE8F08F00BF70B1010062
:1088D00078B101002DE9F04F814291B00546DDE904
:1088E0001A760C460B92984601DB04460D4636F983
:1088F000140057F8243058F8241003FB00F336F91D
:1089000015E001FB00F957F825100EEB000A01FBFA
:108910000E3C1D9BCDE90DCA53F8241058F82520B4
:108920008C4653F8253002FB0E99D8B25FFA81FECF
:10893000864588BF60F3070CC1F3072EC3F30720F9
:10894000864538BF60F30F2CC1F3074EC3F30740D1
:10895000209A86454FEA136388BF60F3174C06924E
:10896000B3EB116F1F9A88BF63F31F6C229B0592B4
:108970001E9A0893219B04921D9A0FA80EA9079393
:108980000DABCDE90110039200930B9A0CAB294675
:108990002046CDF83090CDF83CC0FFF769FE0CA919
:1089A0000EC991FBF3F192FBF3F24FEA84094FEA0F
:1089B000440B48F8091047F8092026F80B301C9A98
:1089C0001C9B115D5B5D00228B4238BF0B461C99DE
:1089D0004FEA450A0B5526F80A2011B0BDE8F08F82
:1089E0002DE9F04FDFF8C8B08BB09BF80C40002C9D
:1089F0005BD0002859DD00251F4637F9153005F1F9
:108A0000010A002B91468846064654464BDD5645E2
:108A100003DC4AE00134A6423DD037F91430002B84
:108A2000F8DD59F8243059F8250058F82510C01AF7
:108A30004EF2B05358F82420891A0029B8BF494291
:108A400003FB01F14FF461430028B8BF404203FB30
:108A500000F00914001402F017FFDBF81430834211
:108A6000D8DD1A9B21460893199BCDF800900793F7
:108A7000189B32460693179B28460593169B013494
:108A80000493159B0393149BCDE901734346FFF7B1
:108A900021FFA642C1D1554637F9153005F1010A2B
:108AA000002B5446B3DC5645F5DC0BB0BDE8F08F27
:108AB000C41D00202DE9F04F99B09E4C0AAF657B94
:108AC0006C4605B120B9A5463C37BD46BDE8F08FE0
:108AD00083467C6090464400C21DFB6122F0070281
:108AE00004F10803ADEB020D23F007030DF1280A92
:108AF000ADEB030D5A460AAD0E465046FF21BD6050
:108B000011F0FFF822462846FF2111F0FAF87A6E9C
:108B1000002A40F3A6803A6FFB69786E911E9A1E78
:108B200001EB4003FB621319FA607B6342464FF08E
:108B3000000933468846C7F824A0C7F818B038F9AA
:108B4000021F002940F38180B869B96F002851F8ED
:108B500029107ADD4FF0E17C0E0EC1F30744C1F31A
:108B600007205FFA81FE74490CFB06F601FB00F05A
:108B70000CFB04F401FB0EF1361424140014091448
:108B8000C83EC834C838C8313E63C7F82080D7F81B
:108B90000CA00025BC62786139611E46904603E056
:108BA0007B6B013553454CD03AF9021F0029F7DDA4
:108BB0004FF4614358F8254056F8251003FB04F4A0
:108BC0004EF2B05303FB01FBBB6E241433F91900C2
:108BD000FB6E001B33F919104FEA2B4BA1EB0B0175
:108BE0000028B8BF40420029B8BF494202F04CFEFD
:108BF0003B6BA342D4DDBB6AA342D1DA7B695B4500
:108C0000CEDD3B695B45CBDA7B6F33F91940494BCD
:108C100004EB44049969C4EBC404A142A8BF2146F3
:108C20008842BDDA7B6A595DFF297DD0BB6833F885
:108C300015108142B4DD7A6A23F8150002F8059018
:108C4000AEE733464246D7F82080F96A09F10109B8
:108C500041457FF474AF1E469046D7F824A0D7F85C
:108C600018B0BBF1000F59DD00254EF2B0590BF1E1
:108C7000FF333B636B1C7B631C463B6B9D4203D104
:108C80004CE00134A34547D058F8243058F825006B
:108C900056F82510C01A4FF4614356F82420891A5B
:108CA0000029B8BF49420028B8BF404203FB00F08A
:108CB00009FB01F10014091402F0E6FD40F64753E8
:108CC0009842DEDC1AF805201AF804309342D8D115
:108CD000FF2BD6D0D7F8903021460893D7F88C30A8
:108CE0005A460793D7F8883028460693D7F8843039
:108CF0000593D7F880300493FB6F03933B6E029388
:108D0000FB69CDE900833346FFF7E4FDFF230AF852
:108D100004300134A345B7D17D6BABE7D7F804D05D
:108D20003C37BD46BDE8F08F03F80590BB6823F8DB
:108D3000150035E7C41D00200060CB012DE9F04F80
:108D4000644C93B0247C34B3002824DD1F46904645
:108D50008A4681464FF0000B37F91B30BBB158F8FB
:108D60002B20209902F58072521201FB02F65AF86C
:108D70002B30219903F5807331445B12C95C56484E
:108D80005945057822D0A94209D388066FD40BF142
:108D9000010BD945E0D113B0BDE8F08F7746229B97
:108DA000CDF800800893219B4A460793209B5846A4
:108DB00006931F9B05931E9B04931D9B03931C9B73
:108DC000CDE901735346FFF785FDE0E74FF0FF3033
:108DD0006FF0FE1E844603243E49CDE90A57896898
:108DE000CDF844E00E913D490DF1400E10912299CD
:108DF00001EB46010D9159000C9111AE1CEB020CD8
:108E000018442CD400282ADB1F99614527DD2099BE
:108E1000814224DD01FB0CFC21990A9D6144095C1F
:108E2000A9421CD20C9F8B4507EB4C0C17D0642732
:108E3000229D35F90C500F950D9D35F913C00F9DEE
:108E400007FB05F50E9F07FB0CFC654507DD642558
:108E50000D9F37F9100005FB00F0604537DC24B1A9
:108E6000013C14F90EC0A057C8E70B9F8FE71D986F
:108E700050F82B00C0F307249C4224D0C0B2984283
:108E80000BBF032401244FF0020C4FF0000CBE4630
:108E900001F00F0021990B4440FA04F1C9070DD5E8
:108EA0000F49209F61560F4E114407FB0131A65711
:108EB000895DA94202D259457FF470AF013C6445F7
:108EC000EADA774663E703244FF0020CDFE70B9FF3
:108ED00065E700BFC41D002058B101000101FFFF7C
:108EE00070B1010078B101002DE9F04F83B0DDE9E8
:108EF0000D4704FB02FE07EB0E04E65C864245D0FC
:108F00008E4243D016F0200549D000250324AA46FE
:108F10004FF0010BDFF8A4C006F00F069CF800909C
:108F2000019307EB030C46FA04F7FB0715D5214F15
:108F3000214BE75714F903800D9B174403FB07C728
:108F400017F808800BFA08F7C84547EA050704D266
:108F5000AF421CBF3D460AF1010A14F1FF34E2D2D0
:108F6000012202FA00F002FA01F10843A842019B33
:108F700019D0284010D05B0003EB4E0E0F9B33F945
:108F80000E0090FBFAF003B0BDE8F08F5B0003EB3E
:108F90004E0E0F9B33F90E0003B0BDE8F08F28464C
:108FA00003B0BDE8F08F934003EB4E0E0F9B33F9F7
:108FB0000E00F1E770B1010078B1010058B1010075
:108FC0002DE9F04FB54CABB0E47B1C94002C00F0C5
:108FD0000E81002800F0038118930023CDE91A12B6
:108FE0001093431E14901F93109B1F9A934280F27C
:108FF000FE80369B109A194651F82230511CCB4006
:109000004FEA82021D9115920F9300F05581149B37
:1090100019461D9B994240F34F810E930023109AED
:109020001E93189B03EB420319930BE00E9B0F9AC0
:10903000013352080E930F9200F03A81149A9A422B
:1090400000F036810F9BDB07F0D51A9B15991C4663
:1090500058581B9B0E9A1D4654F82240595855F8F3
:109060002230051B0C940D93CC1A85EAE573A3EB13
:10907000E573169384EAE473A3EBE4731793189EE5
:10908000199B36F91220B3F90030002C40F0FB8018
:10909000002D40F014814FF4007BDDF870800C9EB1
:1090A0000D9F34463D4604FB03F402FB004405FBE0
:1090B00003F5134494FBF3F402FB015595FBF3F520
:1090C000359B159A9C469A5822941446CDE9236103
:1090D00000260E9B21905CF82330D0B2D9B2814299
:1090E00038BF61F30704C2F30720C3F307218842A6
:1090F00038BF61F30F24C2F30740C3F3074188422E
:109100004FEA136388BF61F31744B3EB126F88BF54
:1091100063F31F642595230EC4F307459D422697EC
:10912000CDE92766299600F3D08001331193E3B28D
:109130001293C4F30723139327AF129C139A9442FC
:109140005CDC9DF840306E020B93334646469846F1
:109150009DF838A002F101093A9B2A460393399BF6
:1091600051460293389B0B980193379B00932346FB
:10917000FFF7BAFE00283DDDDDE90C324FEA442C52
:109180000221ACEB030E0EB30BFB0EF3A2EB632339
:10919000A3EB0803002BB8BF5B42B3F5007F09DAED
:1091A000C3F5007300FB03F357F8212002EB6323A0
:1091B00047F82130F1B1013921AB53F8213024AA0D
:1091C00052F82120ACEB030E002EDDD1A8EB0202F9
:1091D0000BFB02F2A3EB6223A3EB0C03DAE76FF0C5
:1091E00000432F4C2F49304A23600B6010602BB096
:1091F000BDE8F08F01344C45AED1B046119B01352E
:109200009D429AD1DDE92842DDE91601279B6425BC
:109210009A42A8BF1A4605FB04F4154602F06CFBFF
:109220002D2801DDC0F15A001C4A0CCA03FB00F3D3
:10923000C0F12D0002FB00321C4B83FB0231D3171F
:109240000A44C3EB621305FB03F3A342BFF6EEAE81
:109250003A9B149A0893399B0E990793389B109860
:109260000693379B0593369B0493359B0393349B5E
:109270000293189B01931B9B00931A9BFFF72AFBF9
:109280001C9B1E93D2E6DDE91667BE4217DA6D021B
:1092900095FBF4FBDDF8708001E700BFC41D0020E2
:1092A000600800206408002000210020B7600BB691
:1092B0001E9B002B7FF498AE1D9B109394E66402D6
:1092C00094FBF5FB4FF00008E9E6DDE9160102F03A
:1092D00013FB2D287FF7AAAE00252C46A2E700BF7E
:1092E0002DE9F04FB64CADB0A47B002C00F02782E6
:1092F000002800F02482934600260A93023B18932C
:1093000003EB40030B9011930E91B246CDF848B099
:1093100005E00AF1010ABAF10A0F00F067811F2285
:1093200000211CA810F0EDFCA64B4FEA4A0233F9CD
:109330001A300C92002BECDDA34B33F91A30B3F545
:10934000967FE6DA0B9B002BE3DD13464FF0000817
:109350009E4ADDF860909A1814929D4ACDF840A07C
:109360001344CDF85C801593CA4605E0119B08F1C3
:109370000108534500F0B3803AF9023F002BF5DDB8
:10938000129E149D159F0E9B56F82820B5F90010CB
:10939000B7F9000053F82830891AC01A02F074FA9D
:1093A000662303FB00F08B49821237980D9251F827
:1093B000042C10F80800A1F12004139202F0BAFA6C
:1093C00004F148010F90BDF9340002F0B3FA0E9B8E
:1093D00056F82820B5F9001053F828301690B7F940
:1093E0000000891AC01A0029B8BF49420028B8BF36
:1093F0004042D4E91C9502F07FFA04464FF0660B18
:1094000040F2EC4C2D2CC8BFC4F15A0404FB05F506
:10941000C4F12D0409FB0459369C6F4D34F91840F2
:1094200085FB09650BFB04FB6C4E109CDFF8B8E173
:10943000345D109E28941EF806E00C9C624ECDF818
:1094400014C036F904C0664F664C04970394012794
:109450000024CDE9017404270D9C0097379F4D44EB
:1094600017F8086024944FEAE9790F9C24AB08228E
:109470006820C9EB651501214FEAAB27CDE92954D6
:10948000CDF8ACE0CDE925C72796F9F7DDF80C9CBF
:109490004D4B0F9A1B5F0D9C02FB04F0139A801139
:1094A0001A4405FB02F5B0EBA51FBFF65FAF444AB7
:1094B000926F82427FF75AAF169A9A42BFF656AF22
:1094C0004FF001021CAB03F80820179B08F10108BC
:1094D0000133DBB21793119B53457FF44DAF179BBC
:1094E000DDF840A0012B7FF614AF9DF87020002A14
:1094F00040F099811CA913460B9C04E011F8010F60
:10950000002840F07E8101339C42F7D1199B0E99CF
:109510009F0001EB070B12995B0001EB07083899DC
:109520000F440A9901EB03093699CB180D930026D5
:10953000CDF83CA0CDF83080DDF82CA0DDF86480BB
:1095400024AC1BAD002A34D0B04532D03D9B5246EE
:1095500008933C9B314607933B9B404606933A9BBE
:109560000593399B0493389B0393379B02930A9B83
:109570000193129B00930E9BFFF7ACF938680C9A8D
:10958000B9F900301268DBF8001002903D98CDE97F
:10959000005406903C9805903B9804903A980390AC
:1095A000404601F08BF924991B9802F06DF90D9B50
:1095B00018800136B24500F021811CAB9A5DC1E7ED
:1095C000C41D0020602C0020543300208C2B002070
:1095D0002C330020E41D0020B7600BB63C2D00208A
:1095E000D4B10100CCB101007C2B00200B9BDDF835
:1095F00038A0002BDDF848B040F3A1804FF00009FF
:109600000A9B33F91930002B40F393804FF0000888
:109610005D4602E00A9B33F91930002B40F382804B
:109620000A9B33F91830002B7CDDC8457AD055F8F9
:1096300028205AF8283055F829105AF82900891A94
:10964000C01A02F021F95AF8282055F828305AF8A3
:10965000294055F82970A41AFF1A379B002CB8BF6F
:1096600064420C90002F764913F80900B8BF7F427E
:1096700002F060F9379B0646714913F8080002F0C2
:1096800059F9704B39460D902046D3E92AB402F0BF
:1096900033F940F23B5E4FF0000C012104272D28E6
:1096A000C8BFC0F15A0000FB04F4C0F12D000BFB51
:1096B000004B654B0D9C83FB0B235B444FEAEB7B1C
:1096C000369ACBEB631B5F4B32F91900DB6F06FB5D
:1096D00000F60D935D4B32F9182004930D9B04FBAB
:1096E00002F403EBA6165A4BCDF814E00393379B14
:1096F000CDF808C006EBA41613F80940CDE90071B7
:1097000006FB0BFB0C9F13F80860CDE92470269232
:1097100024AB05224D2027942896F8F795FFB7EB48
:10972000AB1F0FDB0B9B08F1010843457FF472AFC1
:10973000AB460B9B09F101094B457FF461AF2DB09E
:10974000BDE8F08F3D9B0A9C08933C9BCDE90054FB
:1097500007933B9B0B9A06933A9B41460593399B93
:1097600048460493389B0393379B02935346FFF775
:10977000B1F8C84520DD3D9E389834F9193055F8C8
:1097800029205AF8291050F8290006963C9E1BAC57
:1097900005963B9E04963A9ECDE902061AA8CDE9AD
:1097A0000004484601F08AF8DDE91A0102F06CF87D
:1097B000369B23F81900B5E73D9E0A9B389833F98C
:1097C000183055F828205AF8281050F82800069626
:1097D0003C9E1BAC05963B9E04963A9ECDE9020644
:1097E0001AA8CDE90004404601F068F8DDE91A0145
:1097F00002F04AF8369B23F8180093E7DDF83CA006
:1098000087E50E989F00590019930A9B00EB070B00
:10981000129803EB0109369B00EB070838980B44BC
:1098200007440D9383E6369B389F0D930023DDF8A4
:109830002890DDF84880DDF838B0199377E600BF4E
:10984000441E0020C41D0020B7600BB6D4B1010037
:10985000DCB1010084B038B5174D04AC84E80F00CA
:10986000202240F21461154804AC00F087F80FCCB8
:1098700028606960AA6003CC1822286169612846C3
:109880004FF4B871EB6000F079F80D494FF4606067
:1098900000F0C2F80B494FF4905000F0BDF864207E
:1098A00000F0B8FC632000F0B5FCBDE83840602053
:1098B00004B000F0AFBC00BF282B00200421002022
:1098C000380A0020480A002084B030B402AC84E892
:1098D0000F000A4B9DF808209DF80A109DF81250C1
:1098E0009DF813401A7099709D72DC7230BC184656
:1098F00018224FF4B87104B000F06AB8282B002089
:1099000070B40446174D00686168A268E368164E9B
:109910000FC520696169154A03C57368A569207F71
:1099200051692B4373600870A37F657FCB71E17F22
:1099300093680F480570197094F820000D4958700D
:1099400094F821500C489D7094F82250DD70D36833
:10995000A28DD4E909651A811E605D60086070BC43
:10996000704700BFC02C0020880C0020100C002085
:109970004C210020882B0020359F0000F8B5134BA8
:109980000C0A53F824606EB1F468CFB2013C05E0D4
:1099900073681B5DFB1A002B05DA2C46631C04F16F
:1099A000FF35F5D1F8BD1546B368326833F8143089
:1099B000014652F824002A46184410F097F9B3687B
:1099C00033F814202A4423F81420F8BD680A002034
:1099D000104BF0B40C0A53F824706FB1FB68CEB290
:1099E000013B05E07C68E45C341B002C06DA2B4666
:1099F000591C03F1FF35F5D1F0BC7047BC683968DC
:109A000034F8134051F82350A41A01462819F0BC29
:109A100010F06CB9680A0020044B000A53F82020AB
:109A20001AB9142898BF43F820107047680A00201C
:109A300000232DE9F043036069B3CE68D2B206F18A
:109A4000804C06F100470CF1FF3C013F06F1FF3E60
:109A5000B342A7EB0308AEEB0305ACEB030915D04B
:109A60004C680133645D141BF2D40D6855F82990DD
:109A7000B9F1000F07D08D6835F818502D1B002D57
:109A8000E6DD0560A1444846BDE8F0834FF00009DB
:109A90004846BDE8F0838946F5E700BF0023B1F5ED
:109AA000704F70B4C1F30724036028DA132C1FD958
:109AB000144D06466A68E86889B2431E02EB40020C
:109AC00004E032F8020D081A07D52346581C03F1AA
:109AD000FF34F6D1002070BC7047AA68296852F89C
:109AE000232051F82330121A3260184470BC70479A
:109AF000054B8AB253F8241070BCFFF799BF184683
:109B0000E9E700BF580A0020680A002000B583B0CA
:109B1000014601A8FFF7C2FF044B186008B1019B82
:109B20001844034B186003B05DF804FB402100208B
:109B30004421002070B50E4E024635681DB10D4B14
:109B40001C68A54206D314460846002110F0D9F837
:109B5000204670BD641B8442A8BF044608462246C6
:109B60002946254410F0C2F83560204670BD00BF7C
:109B7000402100204421002070B50B4E35681DB1F6
:109B80000A4B1C68A54202D30024204670BD641B0A
:109B90008442A8BF044628462246254410F0A6F871
:109BA0003560204670BD00BF4021002044210020C8
:109BB000B0F5C06F16D0B0F5047F03DC0F4B5B69C6
:109BC000B3B118470E4B1B7803F07F0303F5047302
:109BD0008342F3DB42189342F0DA10B500F036F816
:109BE000012010BD0029E9DB064B1A78A02A01D01C
:109BF00000207047052201201A707047C02C0020F9
:109C000094210020080B0020024B1B6903B1184768
:109C100018467047C02C0020084B094A5B78DBB21D
:109C2000012B137006D0022B03D10122054B5A7071
:109C300070477047044B1B68184700BF1C0B00207F
:109C40008C210020080B0020C02C002008B50A4BF6
:109C50001B78012B0CD0022B02D10022074B5A702B
:109C6000074A137803F080036FF3C713137008BD1E
:109C7000044B5B689847F3E78C210020080B002019
:109C800094210020C02C00202DE9F843254EDFF858
:109C9000A8903378244DDFF89C80244F012B06D008
:109CA000022B1BD06A78934238D1BDE8F883D8F8EC
:109CB000083098470446B9F1000F28D1D8F804308D
:109CC0009847D8F800309847DFF870906B78327872
:109CD000DBB2934209D1002CE0D1E6E71A467C784A
:109CE0006B78E4B2DBB29342F5D0012A12D0022A9B
:109CF00002D100220D4B5A700D4A697813783170E9
:109D000003F080036FF3C7131370BDE8F88309F104
:109D1000FF39DBE7074B5B689847EDE71A46012AF6
:109D2000E5D1F7E78C2100201C0B0020080B002058
:109D300094210020C02C0020FF2C0100FE2C0100EB
:109D400038B5194C2378012B17D0022B0CD0174AA9
:109D50005278934206D0164A137803F080036FF3CB
:109D6000C7131370002038BD124B104A597852782F
:109D7000022AF7D000225A70EDE70F4DAB689847E2
:109D800018B16B6898472B6898470A4B07492278A7
:109D9000587849789142E5D0012A02D16B689847FA
:109DA000D9E7022AE6D0D6E78C2100201C0B002040
:109DB00094210020080B0020C02C0020A023034A7F
:109DC00013701378A02BFCD0704700BF080B002045
:109DD000014B1878704700BF1C0B0020014BD8784E
:109DE000704700BF1C0B0020014BD870704700BFAC
:109DF0001C0B002000487047200B0020014B987876
:109E0000704700BF1C0B0020014B9870704700BFCB
:109E10001C0B002008B5FFF793FF08B9014B186031
:109E200008BD00BF902100200A46F8B5094F0A4C32
:109E30003B6826689B79B51803EB830103EB41036C
:109E40009D4200D9FFDE0146B86830440FF04EFF56
:109E50002560F8BD5C0B00209021002070B50D46F8
:109E60000646FFF711FF094A094C1378094963F0C8
:109E70007F0365F306038D80A5681370A660FFF766
:109E8000CBFEFFF701FFA56070BD00BF942100204D
:109E90005C0B0020680B0020F0B50D46002185B05A
:109EA0002E79CDE9011103919DF828C0044638B3FD
:109EB0005EB31F4E3178814224D09DF805106008B2
:109EC00060F300019DF80470C4F3800E64F3820116
:109ED0006EF3C30162F303070A466CF307176EF3D0
:109EE000041201A80C21ADF809308DF805208DF879
:109EF0000470FFF799FF012334702B7105B0F0BD9A
:109F00002EB90B4E347005B0F0BD094ED5E79DF863
:109F1000043001A862F303036CF307130C218DF8DE
:109F20000430FFF781FF024E2C71347005B0F0BD94
:109F3000E22100202DE9F04F89B099469DF85C4060
:109F40009DF8603006460F46904602933CB1FFF7FD
:109F500061FF002800F0DA8009B0BDE8F08F704B97
:109F60001D460393FFF790FE2C600024A642CDE926
:109F70000544079440F3AE80DDF850B04FF0010A7D
:109F8000684D68E037F914E038F9140021B1B5F9EB
:109F90000030734500F0BD809DF81610159A4FEA09
:109FA0002E2C6CF303018DF817E08DF8180012F8D1
:109FB00004E00012129A60F307119DF8143004F1C6
:109FC000010C8DF8161032F914106CF30303FE29FE
:109FD0006AF307138DF81430C8BFFF239DF815C02E
:109FE00039F81400C8BF8DF81B30139B4CF0010CDE
:109FF000ADF8190053F824006EF3410CD8BF8DF86A
:10A000001B108DF815C0C1B2C0F3072CC0F3074375
:10A01000ACEB0101C3EB106399424FF04D024FDDF1
:10A0200002FB01F189118DF81E108DF81F300C21F3
:10A0300005A8FFF7F9FE37F914309BF800102B80C4
:10A0400038F914306B800134A64229710BF1010BF1
:10A0500005F106053ED09BF800302979002B91D1FF
:10A060000029F0D0B5F900109DF815C09DF8160034
:10A070009DF814E063F3000C0B1263F30300631C00
:10A0800063F3030E7346159AB5F902E08DF81710C5
:10A090008DF818E0115D4FEA2E2E6EF3071061F374
:10A0A000410C6AF307130C218DF8160005A88DF8F2
:10A0B00015C08DF81430FFF7B7FE9BF80010C2E70B
:10A0C00002FB03F3ACEB00009B118DF81E308DF802
:10A0D0001F00ACE70222B9F814300298009212492E
:10A0E0000B22FFF7D9FE039B1B68002B3FF434AF14
:10A0F0000E490F480A78838002F07F0263F306025C
:10A100000A70FFF789FD09B0BDE8F08F044B039397
:10A110002BE7B5F9023083427FF43EAF93E700BFEF
:10A120009021002098210020DC2100209421002093
:10A13000680B0020092300B583B08DF805000221CB
:10A1400001A88DF80430FFF789FE03B05DF804FB29
:10A15000F0B4224C82B025788DF80720854202D0D9
:10A1600002B0F0BC7047FF261D4802AD076B15F822
:10A17000012DBF681B4892000361C0E902151A4B0C
:10A180003A81069A26701A608A7822B30B79087889
:10A190004E7902FB003006F07F06144B06FB00F000
:10A1A0009F6838608B795BB10022013B01EB83052E
:10A1B0006D89013B2A445D1CF8D102FB06023A601E
:10A1C000A0230B4A13702378FF2BFCD005231370B8
:10A1D00002B0F0BC70474A78D8E700BFE421002005
:10A1E000680A0020880B002034210020580A002033
:10A1F000080B0020014BDB6858817047100C0020D1
:10A20000034B1879A0F10100B0FA80F040097047C3
:10A21000F421002000B583B00146202268460FF0EB
:10A2200041FD01230099064A019802EB8102D2F810
:10A23000051083400B43C2F8053003B05DF804FB02
:10A24000F4210020014B1878704700BF840C0020D7
:10A2500070B4184A184B90601960827802B942783D
:10A2600003790178457902FB013105F07F05134B35
:10A2700005FB01F19E68316083795BB10022013BEF
:10A2800000EB83046489013B22445C1CF8D102FB8F
:10A2900005123260A024FF2309480A4A04700A49C3
:10A2A000137002E00B78022B02D11378FF2BF9D048
:10A2B00070BC7047780C002034210020580A002020
:10A2C000080B0020840C00201C0B00200246024BCF
:10A2D0000068516803C37047741E0020002330B427
:10A2E0000C490D4A0D48C1E90033C1E90233C2E906
:10A2F0000033C2E90233C0E90033094D094C0B6158
:10A3000013610381C5E900332B81C4E90033238144
:10A3100030BC70478C200020B42000201822002080
:10A320000C220020F42000202DE9F04F374C85B09E
:10A330002579247883460294092335480395354CC2
:10A34000354EDFF8D890DFF8D8A00A3200913DE012
:10A3500007783BF91350002F3FD039F91380F75C91
:10A36000A5EB080E71460029B8BF494201914FEA9A
:10A37000430C002F44D00399E75C8E460299092FC5
:10A3800098BF8E46774601998F422EDD009931F9AC
:10A3900013E03AF90C10AEEB010EBEF1000FB8BF9E
:10A3A000CEF1000E774520DD2BF813803AF90C50E2
:10A3B000009921F81350E55C092D01D80135E554C9
:10A3C0001578013B591C00F801591BD012F8015DAA
:10A3D000002DBDD1E5549D55F2E7009929F81350A1
:10A3E00031F913502AF81350E5E7009929F80C5079
:10A3F00031F913504FF001012AF80C50F154DAE70B
:10A40000029FC0E705B0BDE8F08F00BF741E0020BA
:10A41000FD200020182200200C2200208C2000208B
:10A42000B420002030B40546044C00686968AA686E
:10A43000EB680FC42869206030BC70477C1E002088
:10A44000014B1878704700BF22220020014B18688A
:10A45000704700BF242200202DE9F04F6FF0004428
:10A460004FF0000EA446F2464FF0640987B03D4E0F
:10A47000CDE903123C4ADDF848801460726800920E
:10A48000B268019232690292F268059210F1FF30CF
:10A490004AD33478002CF9D033F91050009A954201
:10A4A0004CDD109A019932F910208A4246DD4FF0B6
:10A4B0000101A246119A115458F82070C7F30721E0
:10A4C0005FFA87FBC7F30742A1EB0B01C2EB1762F0
:10A4D000013201319142B5BF09FB01F109FB02F2E2
:10A4E00091FBF2F292FBF1F271786245BCBFA64695
:10A4F00094460029CAD002998D42C7DD039951F8CC
:10A5000020400499A4F50074A4B2B4F5705F51F82A
:10A51000201018D905999142B8DD4FF00101119A28
:10A52000115410F1FF30B4D2BEF1000F15D15046D6
:10A530000E4B83F800A007B0BDE8F08F4FF000018C
:10A54000119A1154B8E7A1F5007189B2B1F5D05F45
:10A550009CD905999142E0DC98E7034BC3F800C011
:10A56000E5E700BF7C1E00202422002022220020DC
:10A570002DE9F04FC3F307461C0E8BB0A642DDF861
:10A580005090DDE917E856DC06FB09FC12B2A2EB9D
:10A5900046220292621CDDB209920AB20795059228
:10A5A0006544159AC3F307276B1ED3180193169BB6
:10A5B000089703EB4C0C4FEA490301370693079BBE
:10A5C00008998B422ADC029A019D002AB8BF5242A8
:10A5D000039204E08A0631D40133BB421ED015F841
:10A5E000011F8142F6D13CF91340002CF4DD059A9D
:10A5F000A2EB432181EAE172A2EBE172DEF80010E6
:10A60000013304FB0211CEF80010D8F800200399A2
:10A61000BB4201FB0422C8F80020E0D1069B0136B2
:10A620009C44019B4B440193029BA3F5007302934E
:10A63000099B9E42C3D10BB0BDE8F08F0022159C50
:10A6400001F00F0104EB030B049341FA02F4E3075A
:10A650000BD5094C094B145712F903A0344409FBDC
:10A6600004B414F80A40A04204D00132042AECD108
:10A67000049BB1E7049BB6E774B101007CB1010013
:10A68000F0B404460F46124E00F1300C35462068F7
:10A690006168A268E3681034644506F110060FC5CE
:10A6A000F4D13D46206861680A4F03C605F13006C3
:10A6B0003C4628686968AA68EB681035B54207F11E
:10A6C00010070FC4F4D12868696803C7F0BC70474D
:10A6D00028220020602200202DE9F04F824693B00E
:10A6E0001F46BDF98C30840007939DF89030884652
:10A6F0009146002122461C9806930FF002FB224649
:10A700001D9800210FF0FDFABAF1000F72DD002450
:10A71000DFF8A4B102E00134A2456BD037F9143060
:10A72000002BF8DD0025229E1E9B12A853F8243032
:10A7300059F8242058F8241040F8245D0296219EF0
:10A7400004900196209E08A8039000962046089544
:10A75000FFF70EFFDDE9083237F9141093FBF1F330
:10A7600092FBF1F11C9A42F824301D9B43F824100F
:10A77000069B012B41D058F824005946C0F308002D
:10A78000B0F5807FC8BFC0F5007001F0D3F8064671
:10A7900059F824004549C0F30800B0F5807FC8BFD0
:10A7A000C0F5007001F0C6F81D9B054653F8241053
:10A7B0001C9B53F8240001F067F8DBF82C3083422F
:10A7C0004FDC4020064637F914C0DDE9082302FBC0
:10A7D00006F603FB00F34FEA8C1C96FBFCF693FB9A
:10A7E000FCF31C9A42F824601D9A42F8243001348C
:10A7F000A24593D113B0BDE8F08F1C9B58F82420DC
:10A8000053F8240059F82430C2F30802C3F30803B4
:10A81000B2F5807FC8BFC2F50072B3F5807FC8BFB4
:10A82000C3F50073CDE90B010D920E930A9401F06C
:10A830002BF8B3250026012104220F901C481D4B44
:10A84000CDE9040537F91450CDE90116079E0092B1
:10A85000039308220AAB6420CDE91065F7F7F4FEF4
:10A8600059E7DBF82830079A37F914C09A4202DC1E
:10A8700040200646A9E7C6F14003DBE90C1260461A
:10A880000093002300F0EAFF084B37F914C0D3E926
:10A890000C12C5F14003009306440023604600F00B
:10A8A000DDFF37F914C028448FE700BF6022002085
:10A8B000F0B10100F8B10100282200202DE9F04795
:10A8C000002688B01C1EDDE91087C8F800603E60D5
:10A8D0004FDD8A46169D08AB43F8046D0295159D21
:10A8E0000DF1180C0195149DCDE903C30095129B41
:10A8F00091460696FFF73CFE1F4ECAF30800B0F5DE
:10A90000807FC8BFC0F50070314601F013F8DFF852
:10A910006CA0C0F14003316BDAF834200546009397
:10A920002046002300F09AFFC9F30809B9F5807F9B
:10A93000C8BFC9F5007905441049484600F0FAFF40
:10A94000DAE90C12C0F140030646009320460023CA
:10A9500000F084FFDDE90623304403FB00F302FB33
:10A9600005F0A40193FBF4F390FBF4F4C8F8004065
:10A970003B6008B0BDE8F08728220020602200205C
:10A98000F0B40446094E00F130073546206861688E
:10A99000A268E3681034BC4206F110060FC5F4D17A
:10A9A0002068616803C6F0BC704700BF901E00209D
:10A9B0002DE9F04F061E83B026DD994690460191A1
:10A9C00000244FF0640ADFF84CB0114F02E001346C
:10A9D000A64219D01BF80450002DF8D038F9140005
:10A9E0000B4900F0A7FF019BFD6A33F9142005FB1A
:10A9F00000F00AFB02F28242B4BF0020012009F8F5
:10AA000004000134A642E5D103B0BDE8F08F00BFD9
:10AA1000901E0020B82B00202DE9F047061E1FDDF8
:10AA2000DFF840A04FF064085746941E04EB46063A
:10AA3000A1F102095D1E34F9020F394600F07AFFD8
:10AA4000DAF8282039F9023F02FB00F008FB03F393
:10AA50008342B4BF00230123B44205F8013FEAD189
:10AA6000BDE8F087901E002000283BDD2DE9F04373
:10AA7000002637468C1E04EB4008951E34F902EF81
:10AA800035F902CF7745B8BF77466645B8BF664609
:10AA90004445F3D100254FF06408A946124CD4E98F
:10AAA0000CC404FB06F60CFB07F7079C013C04EB07
:10AAB000000E14F8010F78B131F915C008FB0CFC39
:10AAC000BC4505DB32F9150008FB00F0B04203DAA3
:10AAD00084F8009003F80590A64505F10105E8D13A
:10AAE000BDE8F083704700BF901E0020034610B4FD
:10AAF000034C59689A680068DB680FC410BC704743
:10AB0000C81E00200023F0B42E492F4D2F4C304A90
:10AB1000304F3148314EC5E90033C5E902332B616E
:10AB2000C1E900332E4DC1E902330B61C4E90033A2
:10AB30002C49C4E9023323612B4CC2E90033C2E93A
:10AB4000023313613B60294A7B603B81C0E90033DB
:10AB5000C0E902330361C6E9003325483381C5E902
:10AB60000033244EC5E902330B604B602B618B60D0
:10AB7000214DCB600B61236020496360A360E360DB
:10AB800023611F4C136053609360D3601361336083
:10AB90001C4A736033812B606B602B8103604360C0
:10ABA0008360C36003610B604B608B60C4E900335A
:10ABB000CB600B61136053609360D360136123819A
:10ABC000F0BC7047EC220020D82200200023002097
:10ABD000C4220020B82B002014230020AC22002027
:10ABE00098220020142D00205433002040330020F0
:10ABF000602C00207C2B00203C2D00202C330020DA
:10AC0000B82200208C2B00202DE9F04F460006F1E1
:10AC100008058BB0044625F00705073020F0070033
:10AC200000AFADEB050DE846D7E91EABADEB000D6F
:10AC300068467D6FF961E91D21F007017B61D7F856
:10AC40009030ADEB010DBA61002122467B62C7F85E
:10AC5000088078600FF055F82A464FF0FF316846BB
:10AC60000FF04FF83246F96E4046C7F810D00FF09B
:10AC70003DF8002C7B6A6CDD3A6E002602F1FF394C
:10AC800009EB04027A62C7F890305A46D34603E0D3
:10AC90007B6A0136994558D019F8011F0029F7D071
:10ACA000FB6E002D33F916A0584B596801EB4A0A88
:10ACB000EEDD4FF0FF333B62D7F88030C7F80C90E1
:10ACC0000024A3F10208914602E00134A5421BD002
:10ACD00038F9023F002BF8D0BB6E59F8241033F935
:10ACE00016C07B6EA1EB0C0133F916005BF8243023
:10ACF000181A00F0C9FD5045B8BF3C6204F10104C8
:10AD0000B8BF8246A542E3D13B6A4A46591CD7F8F0
:10AD10000C90BDD03969C9564B1C6CD0BB6833F957
:10AD200011008245B4DA4FF0000C4FF0010E7C6840
:10AD300023F816A004F801C03B69396A04F806E05C
:10AD40005E547B6A01369945A6D1DA469346D7F818
:10AD50009030002D4BDDD7E9216C00221046396977
:10AD6000013D0D44D7F88CE04C1E7D6214F9011FA3
:10AD70004D1C38D05AF822505BF82280A946FD6954
:10AD800025F81190BD6925F81180D7F880501CF87E
:10AD9000028035F912907D6925F8119036F91290EC
:10ADA0003D6D25F811907D6D05F801801EF802803B
:10ADB000BD6D05F801803D6F6A54FD6DA84653F8DE
:10ADC000225048F82150D7F880104AF822004BF85A
:10ADD000220021F8120026F812000CF802000EF8EA
:10ADE000020043F82200796A0132A142BED12C3719
:10ADF000BD46BDE8F08F0121BB68386A23F816A074
:10AE00003B691E547B68995542E700BFC81E00206D
:10AE10002DE9F04F044699B006AFD7F880500730BF
:10AE2000073525F00705ADEB050D20F0070006AD51
:10AE3000ADEB000D0DF1180BC7E90C215846224669
:10AE40000021BD6098467B600EF05BFF0022D7F8C2
:10AE50008010FA63914252DDC44EC7F82CB006E070
:10AE6000FA6BD7F8803001329A42FA6345DAD7F8A4
:10AE70008C3033F91230002BF2DD0023D7F8B820E4
:10AE80009C42C7E91023FA6B40F36C814FF0FF3905
:10AE900004E07B6C0133A3427B6420DA38F91310A1
:10AEA0000029F6DD786B396B31F9131030F9133066
:10AEB000D7F8880050F82250D7F88400691A50F863
:10AEC0002200C01A00F0E0FC3B6C0546834200F310
:10AED00005817B6CFA6B0133A3427B64DEDB4FFAA6
:10AEE00089F30121B8688354FB6A013203F8091021
:10AEF000D7F88030FA639A42B9DBD7F82CB0002C2F
:10AF000040F3E8804FF00009013C0BEB0402D7F856
:10AF10008030FA60BA68013B0BF1FF3BD318CA4698
:10AF2000FB62D84605E0FB6809F10109984500F08D
:10AF3000D18018F8013F002BF5D07B6833F919E078
:10AF40007B6B33F919203B6B0EFB02F233F919309E
:10AF5000FA610EFB03F33B623B6F33F919307B62FE
:10AF6000BB6F13F80930BB627B6F13F809B0FB6F3E
:10AF700053F82900D7F88030002B40F38680C7F8BB
:10AF800000800023D846F346BA68013A12F9011F3F
:10AF9000894572D1D7F88C00FD6930F913C0D7F814
:10AFA0008400E34450F82360D7F8880006FB0C5671
:10AFB00050F823003D6AB861FE61BE69F96F06FB77
:10AFC0000C553D62D7F8945051F82940EE5CE0B240
:10AFD000BE617E6A3861B446D7F89000D7F89850C1
:10AFE00030F91300ED5C78617E692046B444BE6997
:10AFF00051F8231048EA0608BE6A5FFA81FEAE42A5
:10B00000B8BF2E463D69BE627545C4F30726C1F33D
:10B01000072588BF6EF30700AE4238BF65F30F20E7
:10B02000C4F30746C1F30745AE424FEA116188BF3A
:10B0300065F31740B1EB146F88BF61F31F60D7F859
:10B040008410C7F824C041F823A0D7F8881041F82D
:10B0500023A0D7F88C1021F813A0D7F8901021F86E
:10B0600013A0D7F8941001F803A0D7F8981001F8AE
:10B0700003A0D7F89C1041F823A0F96A013391424C
:10B0800084D1DE46C346D7F80080FB693A6A93FB59
:10B09000FEF392FBFEF2796821F819E0796B21F852
:10B0A00019303B6B23F819203B6FBA8C23F8192019
:10B0B0007B6F03F809B0BB6F1A4697F8283002F887
:10B0C0000930FB6F43F82900FB6809F10109984535
:10B0D0007FF42FAF4C37BD46BDE8F08F40F22732EA
:10B0E00000920022334622496D2093464FF0040A15
:10B0F0003D64D7F844900125F7F7F8FA4FF44A7306
:10B100001C4A0593039229462A4607F13C030496FC
:10B11000CDE9015BCDF800A06420F7F795FA40F285
:10B120002933154A2946039205932A4607F1440319
:10B13000CDE9015BCDF800A004966420F7F784FA0E
:10B1400040F22A300D4B05900393CDE9015BCDF819
:10B1500000A004962A46294607F140036420F7F729
:10B1600073FAB6E64FF0FF339946BAE604B201002F
:10B1700010B201001CB2010020B2010024B2010093
:10B180002DE9F04F071E83B040F3A98092469B46FD
:10B1900089460025B8463BF91530002B40F39B80CB
:10B1A0004FF0FF360024169FA54213D03BF9143010
:10B1B000002B0FDD5AF825105AF8242059F82500E5
:10B1C00059F82430891AC01A00F05EFBB842BCBF9F
:10B1D000074626460134A045E6D1731C7BD03BF9D7
:10B1E000160059F826203BF9151002FB00F359F818
:10B1F00025200C1802FB013292FBF4F249F82520BD
:10B200005AF826305AF8252003FB00F302FB0132DE
:10B2100092FBF4F20C9B4AF825200C9A2BF815406F
:10B2200032F8161033F815300D9A0B440C99925DD4
:10B2300021F815300D9B71005A550E9B0E9A9B5D9F
:10B24000525D0191934238BF13460E9AB100535597
:10B250000F9B53F8252053F826301046DFB23C46AA
:10B260000D9F5FFA82FE07EB060C0E9FA6453E443B
:10B27000C2F3072EC3F3072788BF64F30700BE4558
:10B2800038BF67F30F20C2F3074EC3F30747BE452D
:10B290004FEA136388BF67F31740B3EB126F88BFA1
:10B2A00063F31F600F9B4FF0000243F8250000235B
:10B2B00049F801304AF80130019B01982BF803202E
:10B2C0000C9B1A524FF000038CF8003033700F9B28
:10B2D0001A46002353500135A8457FF45CAF03B0F4
:10B2E000BDE8F08F2DE9F04FB0F1000B83B0DDE940
:10B2F00011C9DDE918A843DD00264FF0FF34DFF85F
:10B3000088E002E00136B3453AD01EF80600002876
:10B31000F8D1013408EB040002E00134A4452FDD2C
:10B32000077805460130002FF7D06445019527DAEC
:10B33000139859F8247050F8240021F8167022F858
:10B34000160014980C9D30F914701698005D23F8BF
:10B350001670159F37F9147025F816700D9D0F9F04
:10B36000A85517980E9D005DA8555AF824500198CD
:10B37000007847F82650109DA8550136B345C4D132
:10B3800003B0BDE8F08F00BFB82B00202DE9F04FCF
:10B390001D464FF01F339BB004460E46904614AF37
:10B3A0007960DFF894C16049C7E90333D7E9129A9D
:10B3B000CDE9061CB96EBB820391796E07F10C03CF
:10B3C000089302913B6C396E584A59480D9301918C
:10B3D0007B6CF96DCDE90E390592BB6D7A6DCDE9C7
:10B3E0000946CDE90B85CDF840A00091396D049058
:10B3F0000A20FFF709FC4F4AD7F88400D2E902324D
:10B4000000210092642200F029FA00284FD03B6FFF
:10B41000002B4CD0FB6F002B49D083463B6FCDE90E
:10B420000568CDE90BA37B6C07F10C0609933B6C17
:10B430001196CDE90753BB6ED7F8806003937B6EFE
:10B440001096FE6F02933B6E0F96BE6F0193FB6DDD
:10B450000E967E6F0093396DD7E915230A20CDF83B
:10B4600028900494CDF848B00D96FFF7D1FCD7F89A
:10B470008430E3B107F10C030993D7F88030CDF89D
:10B4800028B00893FB6FCDF808900793BB6F424636
:10B4900006937B6F796805933B6F2046CDE903A344
:10B4A0007B6C01933B6C00932B46FFF769FEE31D19
:10B4B00023F00703ADEB030D002C0DF1500C10DD54
:10B4C000AA1E7E6802EB44000DF14F0132F9023FE3
:10B4D000002BD4BF00230123824201F8013FF5D1A4
:10B4E0007E607B6C396D0A933B6C0A20CDE9085372
:10B4F0007B68CDE90CACCDE90543FB6ECDF82C9013
:10B500000493BB6ECDF81C8003937B6E02933B6E5D
:10B510000193FB6D0093D7E91523FFF7E3FE1C377A
:10B52000BD46BDE8F08F00BF14230020002300209B
:10B53000B82B0020C81E0020982200202DE9F04FD3
:10B540004FF0000883B001928246894644460D9D23
:10B550004F4E504ADFF854B125E000232354002910
:10B5600059D13AF914104C4F22F8141039F914003B
:10B570004A4B27F814003AF9140049492BF81400F3
:10B5800039F9140023F81400019B33F914002B78C7
:10B5900021F8140031190B7008F1010801340A2C4C
:10B5A00005F1010533D02B78311900913D48315D0B
:10B5B000002BD2D13B48DFF8E4C0DFF8F4E00029EB
:10B5C000ECD0215C3BF81470013149B2DEF800E0A8
:10B5D000215422F814703CF814002F4F714527F8BD
:10B5E0001400DBDD30482E4927F8143022F81430DF
:10B5F00037192BF814302CF8143020F8143021F8B7
:10B60000143001340A2C3B7005F10105CBD14046C2
:10B6100003B0BDE8F08F204F32F9143039F914C06F
:10B6200037F914103AF91400ACEB0101C01A00927A
:10B6300000F02AF91C4B3BF914C023F814003AF926
:10B640001430009AA3EB0C0C144903EB6C0322F8A2
:10B65000143039F9143031F914C01148A3EB0C0C33
:10B6600003EB6C0327F814303AF9143095F800C056
:10B670002BF8143039F9143021F81430019B3119AA
:10B6800033F9143081F800C020F8143084E700BF8B
:10B69000B82B00200023002014230020EC220020DF
:10B6A000C4220020AC22002098220020D8220020B2
:10B6B000C81E00202DE9F04F4FF0000983B0CDE9FE
:10B6C00000129846594D5A4B824695E8070003C32D
:10B6D0004C460D9EDFF880B11A8034E00021544FB3
:10B6E0009E42DFF864E1DFF868C15248524A39559A
:10B6F0005DDB3AF91410514FA35CE9530099504FA8
:10B7000031F91410E9533AF914104E4F25F80B1083
:10B71000009931F9141025F80E10019931F914101F
:10B7200025F80C1038F9141079530C99095D21543F
:10B730000C99095D8B4238BF0B46A35409F10109EE
:10B7400001340A2C2FD038F914203E4BB2424FEA74
:10B75000440533F91430C1DC9E423B4A3B49EFDAE1
:10B76000334F35F80B003B5D096801335BB23B5545
:10B77000324F35F802C0E85331488B4225F800C0FB
:10B78000DEDD0023AB522E4A2A49AB522D4A304807
:10B790005353294A6354A35401340A2C25F80B301F
:10B7A000EB532B52CFD1484603B0BDE8F08F244B6A
:10B7B000009FEA5E214B37F91410EB5E3AF9140052
:10B7C000891AC01A00F060F8224B35F90B10585353
:10B7D0003AF914301C4A591A03EB61031749A85E61
:10B7E0006B5237F914301A49181A03EB60031448E6
:10B7F0002B523AF914300F4825F80B3037F9143032
:10B80000104FAB52019B0C4A33F914306B5238F98C
:10B810001430A15C7B530C9B1B5D23540C9B1B5D64
:10B820008B4238BF0B46A35488E700BFAC220020F0
:10B83000B82200203C2D00207C2B00202C3300203F
:10B840008C2B0020602C002040330020C81E0020DC
:10B850005433002098220020142D0020884210DB51
:10B86000904210B40ADA441A0198521AC01A04FB22
:10B8700000F494FBF2F210BCD0187047019810BC91
:10B8800070471846704700BF81EAE173A3EBE1738C
:10B8900018B30028B8BF4042F1B198421FDA8201C4
:10B8A00092FBF3F2402AA8BF402211498A5CC2F100
:10B8B0005A028AB10F4910B4C2F15A0431F8122069
:10B8C00031F8141003FB02F300FB01F01B1403EB2F
:10B8D0002043184610BC70470346184670479A012B
:10B8E00092FBF0F2402AA8BF402201498A5CE0E7BF
:10B8F00014B3010058B3010088420ADB40B189014A
:10B9000091FBF0F04028A8BF4020094B185C70471D
:10B91000704751B1800190FBF1F14029A8BF40214F
:10B92000034B595CC1F15A0070470846704700BF8D
:10B9300014B3010070B40E680C89022E25DDA042FC
:10B9400023DB0B460125013E02E0844206DC15465E
:10B950006A1C96429C8903F10403F6D101EB85052C
:10B96000AE88ED88A6420DD001EB8201CB88001B8A
:10B970005D1B00FB05F0A41B90FBF4F41C4420B2FB
:10B9800070BC704728B270BC704700250122E5E703
:10B990007F280CDC402824DA0F2824DC082827DA4A
:10B9A000022829DB0428B4BF012002207047B0F52B
:10B9B000806F08DAB0F5007F1CDAB0F5807FB4BF85
:10B9C000072008207047B0F5805F05DAB0F5006FFA
:10B9D000ACBF0B200A207047B0F5005F0CDA0C20DA
:10B9E0007047062070472028B4BF04200520704708
:10B9F0000320704709207047002070472DE9F04F61
:10BA0000056889B01446ADB1394D3A4F3A4E4FF4FE
:10BA100080722B460092394600226020F6F766FEBF
:10BA200040F201122B460092314622466420F6F77E
:10BA30005DFEECE7314A81461368084601338A46C9
:10BA400013600EF043F9C9F8000020B12C4B00EB55
:10BA50000A029A423CD9264F0025B846DFF8B0B01A
:10BA600040F20B1243460092264900226420F6F76A
:10BA70003DFE0426012240F20F13D9F800001146C2
:10BA800000EB0A0C0593069006ABCDE903B7CDE9B0
:10BA9000015500966420CDF81CC0F6F7D5FD0122B3
:10BAA0004FF4887318490593CDE9025107AB11464D
:10BAB0000096049701956420F6F7C6FD40F2111236
:10BAC00043460092214600226420F6F70FFEC7E7A6
:10BAD0000E4A2B46114602E00133322B05D051F8B5
:10BAE000044B002CF8D142F8230009B0BDE8F08FD8
:10BAF000BCB20100C4B20100C8B20100F0230020B2
:10BB00005C440020E8B2010008B3010028230020B3
:10BB1000FCB201002DE9F04F8046006889B08946EB
:10BB2000C0B12F4D00232A4602E00133322B1DD035
:10BB300052F8041B8142F8D1002445F823400EF04E
:10BB4000CDF8284AC8F800401368013B136009B0DB
:10BB5000BDE8F08F4FF491730A4600932249234BBE
:10BB60006420F6F7C3FD09B0BDE8F08F1F4E002436
:10BB70003746DFF880B0DFF880A04FF497723B467D
:10BB800000921B4900226420F6F7B0FD0425012233
:10BB90004FF49873D8F8001064200791059311466C
:10BBA00007ABCDE903B6CDE901440095F6F74CFDAE
:10BBB00040F231123B460092494600226420F6F7DB
:10BBC00095FD4FF499730A2205930095CDE903A6DC
:10BBD000CDE901441146024B0020F6F735FDCCE7D4
:10BBE00028230020F023002060B20100BCB2010035
:10BBF00080B201000CB30100A8B20100134B1B6816
:10BC0000002B22DD2DE9F041114C4FF000082746B2
:10BC1000104E114D86B040F23F123B46009229462D
:10BC200000226420F6F762FD01224FF4A071042384
:10BC300005910093CDE90364CDF808800192114687
:10BC4000024B6420F6F700FDE5E77047F023002083
:10BC5000BCB201002CB4010010B4010010B50446C0
:10BC6000FCF7CCFC04F1E80104F1B000FEF708FD9C
:10BC700004F59070FBF79CFA04F5E870FBF7BEF84A
:10BC800004F5EA70FEF7CEFB04F5F470FBF74EFF07
:10BC900004F50670FEF774FE04F51470FEF726FF37
:10BCA00004F51870FCF7A4FC04F2D92001F038FB6D
:10BCB00004F26620FBF7DAFF94F866320BB9FBF763
:10BCC000DBFF04F51A70FBF7C5FD04F52F70FEF7D6
:10BCD000FDFA04F53170FCF77DFC04F5377000F0D7
:10BCE0003DFE0023044C194623604FF47072BDE8FA
:10BCF000104002480EF005B8DC200020582F00202C
:10BD000038B9064A136801338B4205DD1060012003
:10BD1000704700231846014A13607047DC2000205A
:10BD200008B5FBF7F3F8FEF7D9FAFEF7EBFEFBF7E1
:10BD3000A3FFFBF797FDBDE8084001F0E9BA00BF9B
:10BD40000022014B1A607047F4230020024A136856
:10BD500001331360704700BFF4230020014B1868C3
:10BD6000704700BFF4230020014B33F810007047E8
:10BD70003CB4010038B500240A4B0B4D21464FF46A
:10BD80002072C3E90044C3E902441C6107482C60E7
:10BD90000DF0B7FF2146BDE838404FF496720448D5
:10BDA0000DF0AFBF402B0020FC230020002400201A
:10BDB000802600202DE9F04F00261F460D4691B049
:10BDC0000DF1200881461446314640462022CDE937
:10BDD00005660496CDF81B600DF093FFBB10DFF8ED
:10BDE00008B10A2BB8BF0A23B542CBE90066CBE9FC
:10BDF0000266CBF8106060DDCDE9016604AF4FEA62
:10BE0000490AC9EBC97E039607EB050C04EB0A024D
:10BE10004FEA4E0EB9F1000F14DD00210EEB0200C7
:10BE200030F9024B9C4207DD3E7811F8085001368C
:10BE300001353E7001F80850022901F1010131DDA0
:10BE40009042EDD1013767455244E3D1019BBBBB22
:10BE50009DF820509DF81030002630463746314678
:10BE60000DF111020DF11F040BB1012630448B427C
:10BE7000C4BF19460127944202D012F8013BF3E7F0
:10BE80007FBB5EBB00210B460DF125020DB10121E8
:10BE90000B44904502D018F8015FF7E7D9B911B00B
:10BEA000BDE8F08F039DA542B8BF25460395012547
:10BEB0000195029D25440295C2E733463546CBE7FE
:10BEC000029B9DF82050CBF80C30039BCBF8103030
:10BED0009DF81030C0E7CBF80830E0E7CBF8000061
:10BEE000D0E7CBF80410CCE75C2B00202DE9F04F15
:10BEF00095B000AFC7E90432D7E91ECED7F8943029
:10BF00000028BB61D7F89830F961D7F8B840D7E975
:10BF10002C517B607862386240F37181BF4EC04B18
:10BF20003068994603EB8013786A023A4000B860A3
:10BF3000023B02EB000832F9020F904523F8020F92
:10BF4000F9D12368FB60FB69002B19DD3B6932687E
:10BF5000A3F102084346B348C2EB021200EB4202CF
:10BF6000F869023A08EB400633F9020FB34222F8AF
:10BF7000020FF9D13B6A002B40F36281A84B99462E
:10BF80000022C7F8B84047F6FF764C46C7F8B41011
:10BF9000DFF8A88279697A6200234FEA420B786A57
:10BFA00004EB0B09C34439F940ABCB455344FAD1F8
:10BFB000824678629C4880FB0309DB17C3EBA90328
:10BFC0001BB2002B21F81230994602DD504618446E
:10BFD00078629E42A8BF1E469C450CDAB5F80890D0
:10BFE0002B6809F10109A5F8089031F91290A9EB25
:10BFF0000C0A53442B60CE450CDDB5F80A906B68F3
:10C0000009F10109A5F80A9031F91290A9EB0E097E
:10C010004B446B60022A40F327813B6A0132934212
:10C02000BADCD7E92D14FA68AE8115467F4B786AE1
:10C0300083FB0553A3EBE2732360E3683A6AFB607A
:10C04000FB6990FBF2F0002B40F3E3803B69A3F126
:10C050000208002247F6FF7C96464646714DDFF8FF
:10C06000C881D7F8049038612846002305F5967BEF
:10C0700030F91EAB83455344FAD188FB03A0DB178C
:10C08000C3EBA0031BB29E45B869B8BF9E469C4552
:10C09000A8BF9C46834226F8023F0CDD0B89086846
:10C0A00001330B817862B6F90030B869A3EB000A5E
:10C0B000786A50440860994509DD4B894868013326
:10C0C0004B81B6F90030A3EB090A50444860012ABD
:10C0D00023EAE37002DD0E2A40F0C1806369034465
:10C0E0006361FB690132934205F10205BCD13869F5
:10C0F0000FFA8EFE0FFA8CFCBD68A1F80EC02B461D
:10C10000083323F00703ADEB030DFB69A1F80CE046
:10C11000A3F1040C3B6A6946002B38DD7B690026DD
:10C120009A1E154440F24458A946A1F1020E32F974
:10C1300002AF256AAAEB000323EAE3731BB2AAF15C
:10C14000970AAB421FFA8AFAC8BFC4E90763C2451F
:10C150002EF8023F06F1010602D8A3690133A3615C
:10C160009145E4D1B1F90030002B10DDA36A3A6AA1
:10C170001A441046013304E031F9022F002A40F33B
:10C18000968098421D4603F10103F5D1A06247F65F
:10C19000FF70FB680326984293FBFCF1B8BF18467A
:10C1A0000023234AC7E90E33C7E91033C7E9123326
:10C1B000204D214BA16000B207F12801C7E90C23F3
:10C1C000C7E90A65FFF7B6FBE2686369012A114611
:10C1D000B8BF01219B0193FBF1F323EAE37398427B
:10C1E00009DAE369B34206DD41F287339A4202DCA1
:10C1F000012384F824305437BD46BDE8F08F23680E
:10C20000FB60FB69002B40DD3B6A044E5B00BB60BA
:10C210009CE647F6FF7C4FF0000E6DE7FC23002004
:10C220000024002080260020676666665655555516
:10C23000E8034000F4013200D007400080260020CF
:10C2400047F6FF72AA81FA681A4B104683FB000377
:10C25000A3EBE2732360E3680020FB60F9E6FB6870
:10C260000344FB60E3603CE731F91290F868D7F8CB
:10C27000B830B9F1000FA8BF48445B68F860994432
:10C28000D7F8B830C3E90009C7E647F6FF70FA6986
:10C29000084BA2F1040CFA68A88183FB0263E068F2
:10C2A000A3EBE273044A2360F860CA606FE7A562FB
:10C2B0006DE700BF565555550000FF7F0020F0B4D4
:10C2C000384E8C1E186058609860D8601861043130
:10C2D0001D1F34F9020F002821DD87B207F1FF3C52
:10C2E000BCF1090F11D9A7F10B0CBCF1090F1CD936
:10C2F000A7F1150CBCF1090F1FD800EB400040005E
:10C30000A6FB0070C008033080B2A14245F8040FBC
:10C31000DFD1F0BC2449DA600A791A617047002045
:10C32000A14245F8040FD4D1F3E74010053080B2A4
:10C33000A14245F8040FCCD1EBE7A7F11F0CBCF1EB
:10C34000090F0BD9A7F1290CBCF1090F11D8C000B6
:10C35000A6FB0070C008043880B2D6E7C0EBC0006E
:10C36000A6FB0070A1424FEAD00045F8040FB0D1FF
:10C37000CFE7A7F1330CBCF1090F0BD93D3F272FB5
:10C38000C3D8C0EBC0004000A6FB0070C008263830
:10C3900080B2BAE700EBC000A6FB0070C008093805
:10C3A00080B2B2E7CDCCCCCC402B002084B02DE9BC
:10C3B000F047002482B081460BA880E80E00524D61
:10C3C0009DF85070DFF86C81504EDFF86CA115F8C5
:10C3D000013BD3B9119B122B02DCB9F1000F34D011
:10C3E0004FB340F28512334600924949002249205A
:10C3F000F6F77CF9002305F8043C0134032CE6D160
:10C4000002B0BDE8F04704B0704708EB4403DB8896
:10C410000B9A9A4202DD0D9B1E2B3BDC4FF4CC7233
:10C4200033460092514600224920F6F75FF9002377
:10C4300005F8043CE1E740F28912334600923549A1
:10C440003A464920F6F752F9D7E74FF4B6722F4B28
:10C45000009231494A464920F6F748F9129B062BCB
:10C46000CBDD002F44D1109BB3F57A7F36DD159BD1
:10C47000052B33DC139BB3F5FA7F2FDA4FF4BC7234
:10C480003346009225493A464920F6F72FF905F838
:10C49000047CB2E74FF4C7721C4B00922049002283
:10C4A0004920F6F723F9012305F8043C67B14FF45E
:10C4B000C972334600921B4900224920F6F716F94B
:10C4C000002305F8043C98E740F2951233460092A9
:10C4D00015493A464920F6F709F98EE740F27D12F0
:10C4E00033460092114900226420F6F7FFF884E7F2
:10C4F00040F27112334600920D494A464920F6F740
:10C50000F5F805F8049C78E7432B002064B501009A
:10C5100024B6010060B6010078B50100C8B501007D
:10C5200094B60100B0B60100E0B60100ECB5010020
:10C53000A0B501003CB40100F0B6010082B000B526
:10C5400083B0069A0593012A23D0E8B1591001EB74
:10C550004301914202DCD91E032926D9023A032A5B
:10C5600012D8079A012A0FDD023B032B0CD84FF497
:10C57000E472134B0092134900224920F6F7B6F8F3
:10C580000022114B5A709A7003B05DF804EB02B0B0
:10C590007047042BD9DC4FF4DC72094B00920B4935
:10C5A00000224920F6F7A2F8EAE74FF4E072044BC4
:10C5B0000092074900224920F6F798F8E0E700BF0B
:10C5C00064B5010034B50100402B0020C8B401005F
:10C5D00008B5010084B0F0B587B00CAC84E80F005A
:10C5E0000D9B002B45DB40F2EB13294D00930022FD
:10C5F0002B4628494920F6F779F84FF4F6722B4676
:10C600000092254900224920F6F770F801240026FF
:10C6100040F2ED120427214BCDE904522146224677
:10C62000039364200DABCDE901460097F6F70CF8B3
:10C630004FF4F7701A4B22460590039304951AABFA
:10C64000CDE90146009721466420F5F7FDFF40F251
:10C65000DC530C9A9A4207DC41F288331A9A9A42C8
:10C66000104BCCBF9C709E7007B0BDE8F04004B08A
:10C6700070471B9B642B07DD1A9BB3F57A7F03DDA4
:10C680000122084B1A70AEE70022064B1A70AAE787
:10C6900064B5010060B401007CB4010094B40100F1
:10C6A000ACB40100402B00202DE9F043204C214F79
:10C6B000DFF88490DFF8848083B0E61CE07814F81B
:10C6C000015BB8B9E5B163790133DBB20A2B637161
:10C6D0000BD940F2092301250246009360713B46C5
:10C6E00041466420A570F6F701F8B442E6D103B0E4
:10C6F000BDE8F08345B10023B4422372DED1F6E7F2
:10C70000B4426571DAD1F2E7237A0133DBB2282B28
:10C710002372EAD940F213223B46009249462A4648
:10C720006420A570F5F7E2FFB4422572C6D1DEE7BA
:10C73000402B002064B501002CB701001CB701009C
:10C7400000212DE9F047984601270B468CB025487B
:10C75000DDF850A0179D199E234C914601808170F1
:10C76000C21C12F8011B31B934F813108D4202DDDE
:10C770001E2EC8BFC7540133032BF2D16C461AAD2D
:10C780000FCD0FC495E80F0084E80F006C4617AF7B
:10C7900097E80E004046FFF709FE23AB0FCB8DE86C
:10C7A0000F0014AE52464146484656F8383FFFF750
:10C7B000C5FE0FCE0DF11C0CACE80F0033681BADAD
:10C7C000CCF800300FCD0FC495E8070084E80700CF
:10C7D00097E80F00FFF7FEFE0CB0BDE8F047FFF74B
:10C7E00063BF00BF402B00203CB401002DE9F04F97
:10C7F000A3B00025DDE93D876E4681468A4617AC29
:10C80000159220462C2200219B460DF07AFACDE9A4
:10C810000F74CDF838800DF1D80C0DF11C0EBCE86A
:10C820000F00AEE80F009CE807008EE807000DF14E
:10C83000BC0CBCE80F00C8F80050C8F80450C8F899
:10C840000850C8F80C50C8F810503D607D60BD60BD
:10C85000FD603D610FC69CE807002E9B86E807003F
:10C86000314E2D9A514648460EAFFFF73FFB0FCE93
:10C870000FC736680FCC3E6003AE0FC60FCC0FC695
:10C8800094E8070086E807002E99284E02912C991B
:10C890005B4600912D99159A019148465146FFF744
:10C8A0004FFF33682D9901330A2B14BF1C462C46C9
:10C8B00048463F9B179A3460FFF700FD3F9B1C4A98
:10C8C000D9684098D37881828DF85B50E3B91179AB
:10C8D00018465279F1B91ABBF8B9012240F27A210F
:10C8E0000023144C14480591CDE90133CDE903042C
:10C8F000009211460DF15B036420F5F7A5FE9DF84B
:10C900005B0023B0BDE8F08F012011790346527916
:10C910000029E0D043F0020312B98DF85B30DCE768
:10C9200043F00403F9E700BF5C2B0020FC23002048
:10C93000402B002064B50100E0B5010030B9064B82
:10C94000187810B10138C0B2187070471423024A29
:10C9500018461370704700BFF823002001464FF4BB
:10C96000A07201480DF0C2B9D81E0020014B187802
:10C97000704700BFB52700202DE9F04F4FF00008A9
:10C98000C146D5B014AD029200218022284634AEB3
:10C990000393629C0DF0B5F98022002130460DF022
:10C9A000B0F905A83C2200210DF0ABF9631E0193FC
:10C9B0004A4BDFF830C193F9024093F801A005AF6C
:10C9C000CDF80080019B13F801EF0193002301E0F3
:10C9D000202B28D03CF91320A24207DA55F8231067
:10C9E000501D014409F1010945F8231092450BDA65
:10C9F00056F823003968A2F1050B5844594408F150
:10CA0000010846F823003960BEF11F0F03F101034E
:10CA1000DED1A242DCDA61990029D9DD0099202B10
:10CA200011440091D6D10437BD420CF1400CC9D15C
:10CA300000210F46294BDDF800E09C88B3F9066021
:10CA4000B3F908C053A833AB53F8042F002A08DD0C
:10CA5000A24206DA55F82120B24202DAF445B8BF04
:10CA60000137984201F10101EED1029BB3F57A6FD3
:10CA70001BD9B8F1500FD4BF0021012140F2EE23A1
:10CA8000059A9A420FDD13989842D4BF00200120E6
:10CA900017B1B8F1050F0ADC00231846104A1360DD
:10CAA00055B0BDE8F08F0020F2E70021E6E7B9F1CC
:10CAB0000A0FF1DD039B052BEEDD0029ECD10028E8
:10CAC000EAD1064B064A1978639C136821449942BF
:10CAD000CBBF0133106013600120E1E7D81E0020B6
:10CAE000AC270020582F002070B588B09DF8685002
:10CAF0009DF86C60C0B9B9B9354C2178C9B1132A19
:10CB000047DC0D9A632A44DC133342DB0C9B092B70
:10CB10003FD8304B304AD9691368994251DD012121
:10CB20000B44136021701BE00022294B1A7008B0DF
:10CB300070BD1999104604911799CDE905560391D6
:10CB40001699029115990191149900911946DDE900
:10CB50000C23FFF711FF207010B12048FAF74EF9AF
:10CB6000FDF748F924780546FCB11D4C1D4E23887D
:10CB7000327801331BB22380002AD8D1632BD6DD53
:10CB80000220FDF7D7FA01236422AB7733702280AD
:10CB9000CDE7104B0D99B3F918209142BADC002271
:10CBA00001210D4B21701A60DAE70E4E0C4A3378E2
:10CBB0001480002BBBD00320FDF7BCFAAC77347097
:10CBC000B5E70023084813602370FAF717F9C7E7A1
:10CBD000B5270020D81E0020B027002064DB01000C
:10CBE000B6270020B427002008DA0100054A92F891
:10CBF0004E30834204DA8B42B4BF002001207047DC
:10CC000001207047D81E00204B28CCBF00200120F7
:10CC1000704700BF2DE9F04F013883B00028019123
:10CC20006CDD012872D04FF000094FF0010C09EBC8
:10CC3000000303EBD3735B1032F9131032F9104089
:10CC40004500A14204DD22F813400C4622F81010E2
:10CC500032F919104FEA490BA14202EB0B0A04DD2D
:10CC600022F81940515332F9191032F913408C420D
:10CC700005DD22F8131022F80B4032F91340064666
:10CC80000BF10201555E02EB4C0E22F81350545288
:10CC900032F90B503EF9028F0CF1010CA845F9DB7B
:10CCA000711E02EB410301E00E4601391F4633F9C4
:10CCB0000249AC42F8DC8C4507DCAEF80040A7F82E
:10CCC00000800E46BAF90050E4E7019B22F80B40C1
:10CCD0008B423D8018DBE14616DD48450EDD09F14B
:10CCE000010C8445A3D102EB49094000B9F9003099
:10CCF000115E8B42C4BFA9F800101352019B32F998
:10CD0000130003B0BDE8F08FB01EE6E791460220A5
:10CD1000ECE700BF2DE9F04F013800EBD07383B092
:10CD20005B10002801936CDD012872D04FF00009E0
:10CD30004FF0010C09EB000303EBD3735B1031F9E7
:10CD4000132031F910404500A24204DD21F81340C0
:10CD5000144621F8102031F919204FEA490BA2425C
:10CD600001EB0B0A04DD21F819404A5331F919206F
:10CD700031F91340944205DD21F8132021F80B40CE
:10CD800031F9134006460BF102028D5E01EB4C0EA9
:10CD900021F813508C5231F90B503EF9028F0CF1EF
:10CDA000010CA845F9DB721E01EB420301E01646B7
:10CDB000013A1F4633F90249AC42F8DC944507DCDE
:10CDC000AEF80040A7F800801646BAF90050E4E734
:10CDD000019B21F80B4093423D8018DBE14616DDB4
:10CDE00048450EDD09F1010C8445A3D101EB490949
:10CDF0004000B9F900300A5E9342C4BFA9F8002090
:10CE00000B52019B31F9130003B0BDE8F08FB01E47
:10CE1000E6E789460220ECE7831A042B10B413DD01
:10CE2000DC1EB1F90430002A0B804B8031F914303C
:10CE300008DD4000A0EB42020A44014421F8023D13
:10CE40008A42FBD110BC70475C1E032C08BF9C1E9D
:10CE5000E7E700BFF0B40446049E0846DDE905514B
:10CE6000A642DDF81CC019DD04F10044AF1E013CF0
:10CE700007EB460705EB44058E1C06E09C42B8BF55
:10CE80001C46BD4226F8024F08D035F9024F9442A5
:10CE9000F4DD1446BD4226F8024FF6D1F0BC6246DE
:10CEA000FFF7BABFF0B400280F46DDE90561DDF8F1
:10CEB0001CC014DB013006EB40048D1C06E09842D8
:10CEC000B8BF1846B44225F8020F08D034F9020D55
:10CED0009042F4DD1046B44225F8020FF6D13846F0
:10CEE000F0BC6246FFF798BF2DE9F043B1F900901E
:10CEF00002284FEA4918DDE90767C2E90088DDE941
:10CF000009CE21DD8C1E5B0176017F01043204EB2A
:10CF10004000023103E0A84631F9029C0432B1F925
:10CF20000050B1F9024006FB05F503FB04541568F7
:10CF300002310CFB054407FB094408FB0E44814207
:10CF40004FEAA4245460E6D1BDE8F0832DE9F04116
:10CF5000884684B04C00083404AFBD6B24F007044D
:10CF6000ADEB040DBE690395FD6904AC0195009617
:10CF700002947D6BFFF76EFF3B6B21460293FB6AC9
:10CF800003950193BB6A40460093D7E90823FFF756
:10CF9000ABFFBD46BDE8F0812DE9F041884684B085
:10CFA0004C00083404AFBD6B24F00704ADEB040D56
:10CFB000BE690395FD6904AC0195009602947D6BF2
:10CFC000FFF770FF3B6B21460293FB6A03950193C9
:10CFD000BB6A40460093D7E90823FFF785FFBD46AB
:10CFE000BDE8F0812DE9F04F8FB00AAF7D6D9A4614
:10CFF0001B1A023300F103088B465919FB6B18EB1F
:10D00000050804461646FB6000F0AA804FEA88092E
:10D01000002934D109F10A0929F00709C7F808D015
:10D02000ADEB090D08953E6D0DF128090796FE6CD4
:10D0300013460696BE6C5A4605967E6C414604968B
:10D040003E6C0396BE6BCDF80890CDE900A6FFF7C5
:10D05000A3FF002C0DDBFE680235013409EB8509C6
:10D0600006EB440459F8043B5B1124F8023DA64248
:10D07000F8D1D7F808D01437BD46BDE8F08F8B0043
:10D080000A3323F00703C7F804D0ADEB030D08956E
:10D090003A6D0AAB0792FA6C09F10A090692BA6C6A
:10D0A00029F0070905927A6C04923A6C0392BA6BE4
:10D0B000CDE900A2BB605A4602933346FFF746FF14
:10D0C000ADEB090D0895396D0DF128090791F96C43
:10D0D00033460691B96C5A460591796C2046049105
:10D0E000396C0391B96BCDF80890CDE900A14146A8
:10D0F000FFF752FF631C9A4511DDFE68BA68E91C10
:10D10000B31E02EB810103EB4A0A06EB440251F81D
:10D11000043B5B1122F8023F5245F8D1FE60002C1F
:10D120000DDDFE68E91C09EB810106EB440251F8B4
:10D13000043B5B1122F8023D9642F8D1FE60BB68C9
:10D14000023559F8252053F825301344FA689B110D
:10D1500022F81430D7F804D01437BD46BDE8F08F5C
:10D160008B000A3323F00703E946ADEB030D089566
:10D170003E6D0DF128080796FE6C13460696BE6CB0
:10D180005A4605967E6C04963E6C0396BE6BCDF8AF
:10D190000880CDE900A6FFF7D9FE544512DAFA68F7
:10D1A00004F10044013C0335931E02EB440608EBF6
:10D1B000850803EB4A0A58F8043B5B1126F8023F46
:10D1C000B245F8D1CD461437BD46BDE8F08F00BF5B
:10D1D0002DE9F04788B099464FEA430808F1080462
:10D1E00024F0070408AFADEB040DD7E90D563C6BF6
:10D1F000CDE90656BD6AFE6A059403953C6A7D6AD0
:10D20000049608AECDE901650094FD6BFFF7EAFED8
:10D21000B9F1000F10DD023CA044A6F1020A34F976
:10D22000023F3AF9022F9B1AAB42CCBF5B1B03EAC9
:10D23000E37344452380F2D1BD46BDE8F08700BFCB
:10D240001E232DE9F041264E86B00D468046009300
:10D2500024493346642014460022F5F747FA002794
:10D260004FF01F0C012204211F482B46CDF814C09B
:10D2700000910390114664200496CDE90177F5F7FB
:10D28000E3F94FF0240C0120184AA5EB08014909E5
:10D29000009003920496CDE901774346CDF814C07F
:10D2A00020226420F5F7D0F9294651F8043BA34227
:10D2B000FBD02B2700220124C5F11F030C48194481
:10D2C000CDE901220390049649092B460597009465
:10D2D00020226420F5F7B8F906B0BDE8F08100BF60
:10D2E0003CB7010048B701005CB7010068B7010016
:10D2F00080B701000B68934209D070B50D46144603
:10D300000646224629463046FFF79AFFF9E770475E
:10D310000022024BC3E900221A8170473028002006
:10D320000278014B1A70704718200020314B1B788F
:10D33000002B5AD02DE9F04F16462F4A87B0894668
:10D34000804600242D4F1368DFF8B4B0DFF8B4A096
:10D35000013E14E03D5D38F91410022D2BF8101039
:10D3600005F1010E39F914109CBF5FFA8EF53D5599
:10D37000032D2AF8101017D001340A2C0CD04FEAD4
:10D38000440C0CEB0401C81816F8011F0029E1D168
:10D39000395501340A2CF2D10133022BC8BF0023C6
:10D3A000136007B0BDE8F08F0CEB04035B000BEBE0
:10D3B00003010868534402901868B1F804C09B88C0
:10D3C000049002A928460192ADF81430ADF80CC0C3
:10D3D000FFF7A0FC04A928F814002846FFF79AFCE0
:10D3E000019A29F814001368C6E7044AC2E9003319
:10D3F00013817047182000203C280020302800208E
:10D40000B8270020F4270020F0B483000A3323F06B
:10D410000703002800AFADEB030D30DD6B4600269F
:10D420000439B20002F1804292F880C292F881522F
:10D4300092F8824292F883225FFA8CFCEDB2E4B259
:10D44000D2B2013683F800C05D709C70DA70BCF116
:10D45000000F03D00CF1FF3C83F800C01E2D9CBFD1
:10D4600001355D700CB1013C9C700D2A9CBF0132EE
:10D47000DA7053F8042BB04241F8042FD1D1BD46E5
:10D48000F0BC704792F83230002B43D1F0B5002841
:10D490008BB00E460546144610DD936A42189A4238
:10D4A00010DB00231A4684F8313094F8243093427C
:10D4B0009CBF012384F830300BB0F0BDF1D1D36AAA
:10D4C0008B42EEDD2E2294F83130134F013384F875
:10D4D000313012493B46009264200022F5F706F9EC
:10D4E0004FF0340C0020012104220D4B049794F8D6
:10D4F0003170CDE90110009203930322CDF814C0DE
:10D5000007AB6420CDE908650797F5F79DF894F817
:10D510003120CAE7704700BF94B70100A8B70100E7
:10D52000D0B701002DE9F04F98468DB0DDE91653D4
:10D53000012DA946B8BF4FF00109012B9C464FF0C1
:10D540000004B8BF4FF0010C189E09923788B6F856
:10D5500004E01268D8F8006005FB072503FB0E669F
:10D56000002895FBF9F596FBFCF6CDE90A442ADD87
:10D57000A446A146A246023901EB40000894CEF130
:10D58000000B079031F9023F5A1B22EAE272334442
:10D5900003EAE37397420EEB030403DC0120D21B82
:10D5A000089092445B4505DC4FF0010C002CB8BF9D
:10D5B0006442A144079B9942E4D1089B002B49D1C6
:10D5C000BCF1000F49D10124002604255C22244F20
:10D5D000DDF82490234B059221462246CDE90337FE
:10D5E000CDE901464B4600956420F5F72DF85D2006
:10D5F0001D4B224621460590039304974346CDE9EF
:10D60000014600956420F5F71FF85F20174B22466E
:10D6100021460590039304970AABCDE90146009596
:10D620006420F5F711F86020114B22460590039312
:10D6300004970BABCDE90146009521466420F5F730
:10D6400003F8DDE90A23C9F80020C8F800300DB05E
:10D65000BDE8F08FCDF828A0B2E7CDF82C90B2E766
:10D6600094B70100E0B70100F0B7010000B8010075
:10D6700014B8010070B19A4215DC0F4A1368C72B29
:10D6800001DC013313600D4B187808B181F0010003
:10D6900019707047084B1A68C72AF4DD1860074BE9
:10D6A0000120197070470022034B1A60034B187851
:10D6B0000028EDD0EAE700BF4428002050280020D1
:10D6C0002DE9F04FBC48ADF2A44D1893DDF8E044CD
:10D6D0000378CDE915121993002C00F082850DF521
:10D6E0008C7ACEAD3C220021504630AE12950CF023
:10D6F00008FB78220021284613960CF002FB1E221C
:10D70000002130460CF0FDFA002325AAC2E90033BF
:10D71000ADF89C3001232046294617921E93FFF74F
:10D7200073FEDDF8E04420220F23DDF8D814CDE9A4
:10D7300003320691DDF8DC14B0AB05911299204656
:10D74000019113990293009192AA74A95346F9F793
:10D75000F5F9DDF8E004002840F3918553460024F4
:10D760000AEB400133F9022B02B101348B42F9D1AB
:10D7700020940A2420260F25DDF8D83401940C9338
:10D78000DDF8DC348D4C0B93B0ABDFF848C2129F50
:10D790008B498C4A08930694139B8B4CCDE902C2AB
:10D7A000CDE90414009392AA534674A90797CDE9D2
:10D7B0000956FBF77FF940F22F2000240123059042
:10D7C000DFF814B281483246294600930390DDF811
:10D7D000DC346C20CDE90144CDF810B0F4F734FF0F
:10D7E000DDF8D824139B0692DDF8DC24DDF8E00494
:10D7F0000592B0AACDE901720093CDE903565346D4
:10D8000092AA74A9FBF79AFADDF8E004A04208DDB9
:10D8100053460AEB400133F9022B02B101348B422B
:10D82000F9D11F9420250F24DDF8D834129E0693D9
:10D83000DDF8DC34139F0593B0AB0293CDE90345CB
:10D84000534692AA74A901960097FBF7B9FBDDF83D
:10D85000D834CDE903450693DDF8DC34DDF8E00487
:10D860000593B0ABCDE901630097534692AA74A922
:10D87000FBF7B6F8DDF8E044002C40F30485002205
:10D88000534610460AEB440133F9022B02B1013032
:10D890008B42F9D12190ECAE782200210DF58565FF
:10D8A00030460CF02EFA7822002128460CF029FA96
:10D8B00020210F22464B20461C68DDF80435647891
:10D8C000B3F924300894DDF8D844CDE90321069457
:10D8D000DDF8DC4407930594129C534601950096AD
:10D8E000029492AA74A9FCF7F7FEDDF8E034002B4D
:10D8F00040F3C184002455AF149755F8041B56F823
:10D90000040BFDF7C1FFDDF8E0340134A34227F832
:10D91000020BF2DC0F252026DDF8D814DDF80425F3
:10D92000149FB2F924200791DDF8DC141846069103
:10D93000B0A903911299CDE9045602911399089266
:10D940000191534692AA74A90097FBF7C9FC0024E1
:10D9500040F28F20012329461C4D3246059000934A
:10D960006C20DDF8DC34CDF810B00395CDE901442E
:10D97000F4F76AFE534692AA74A9DDF8E004F9F7B9
:10D9800051FC2046DDF8E014CDF800A092AB74AA5B
:10D99000F9F73AFADDF8E004A0421FDD3A466624C2
:10D9A00007EB4001B2F9003004FB03F39B1222F8AD
:10D9B000023B8A42F6D111E05D1600206828002063
:10D9C000602C00208C2B00205428002028B8010057
:10D9D000340A00202C33002094B70100129B92AA35
:10D9E0000293149B74A9009328AB01935346FCF750
:10D9F00033FDFCF7FFF91C90FEF7B8FF0446002842
:10DA000033D1199B022B1C9B9B7927D0DDF80C2569
:10DA100003F0FF0102F50675002B40F03884199BD6
:10DA2000012B1FD11C9BDB7FE3B1242265A80CF0E6
:10DA300068F94FF4AF720A2364204621022564ACD2
:10DA4000C4E90A01E2802046628123812560C4E99D
:10DA50000C330DF1E009FCF793FF09E0002B40F0D7
:10DA60004B84AD4D2846FCF78BFF0DF1E00964AC0B
:10DA70000026DDF8E0342660B3424EDDCDF8689034
:10DA8000DFF8AC82DDF850904FF43F7243460092CD
:10DA9000A24900227020F4F729FE012540F2FD2260
:10DAA00004239F490592CDE902612A462946009345
:10DAB00070202346CDF810B00195F4F7C5FD02277C
:10DAC00040F2FE202368974A2946CDE9026205907C
:10DAD0002A4609EB430370200195CDF810B000975A
:10DAE000F4F7B2FD40F2FF2023688F4A0590CDE99C
:10DAF00002620AEB43032A46CDE90075CDF810B067
:10DB000029467020F4F7A0FD2368DDF8E0242B44BB
:10DB100093422360B8DBDDF86890012240F20131C6
:10DB200000250420814BCDE904B1009003936D20C2
:10DB3000CDE9012511460DF59C63F4F785FDDDF86F
:10DB4000E004A84236DD149F5646DFF8F88103E072
:10DB5000DDF8E004A8422DDD4FF4427337F9020BE3
:10DB6000B6F900C0002200934146C4E90050704B52
:10DB70004120C4F808C0F4F7B9FD36F9023B01357D
:10DB8000002BE5D040F20A30002201214FF0040CB6
:10DB9000684B05900393CDE901124120CDF810B0F8
:10DBA000CDF800C023460322F4F74EFDDDF8E00473
:10DBB000A842D1DC0F262027B0AB0C93DDF8CC3483
:10DBC000169A0B93DDF8D4340592159A0A93179B95
:10DBD0000492129A0993DDF8D034DDF820550392AF
:10DBE000139A0893DDF8C8340292119528AADDF83B
:10DBF000D85407930192189B149A1095DDF8DC54C1
:10DC000006930092534692AA74A90D96CDE90E751B
:10DC1000FDF7BCFB002540F2233001233146464E80
:10DC20003A4605900093CDF810B00396CDE9015522
:10DC3000DDF8DC346C20F4F707FDDDF8E024AA42BF
:10DC40002CDD189BDDF8C8149F1EDDF8CC34AA46E5
:10DC5000A1F102085E1E01E0AA421FDD38F9023F71
:10DC600037F9021F636016F8013F2560A160013596
:10DC7000002BF1D040F2293201210423CDE904B276
:10DC80002E4ACDE90031CDE902A2234603224120EC
:10DC9000F4F7DAFCDDF8E024AA42DFDC1423189E56
:10DCA000179DDDF85880159FCDE90053DDF8C82495
:10DCB000334641463846FDF7FDFC3146DDF8CC34AD
:10DCC000DDF8C8240A20FCF7A7FE3146DDF8CC3485
:10DCD000DDF8C8240A20FCF76BFEDDF8CC343246B0
:10DCE0000093DDF8C814DDF8D0340A20FCF7BCFE40
:10DCF000DDF8CC343246CDE900534146DDF8C83476
:10DD00003846FDF71BFC002317900D49DDF8C85479
:10DD1000DDF8D46425E000BF94C8010030B80100EC
:10DD20001CB2010048B8010054B8010060B80100FD
:10DD300094B701007CB8010028B801008CB801003C
:10DD4000602C00206CB8010035F91300994F56F88B
:10DD5000232027F81300984840F8232001330A2B8A
:10DD60000CD031F9022B002AEED1924820F8132072
:10DD7000914840F8232001330A2BF2D1169F159DBC
:10DD80003946DDF8CC242846FFF7D0FAFEF7EEFD41
:10DD9000199B0026022B08BF40F00100C3B21D935F
:10DDA000AB1E1393BB1E1293DDF8CC7423ABDFF8CC
:10DDB0001082DFF810A214931B94139A129932F96F
:10DDC000023F1498139231F9022F2293129139785D
:10DDD00024930260C9F800203C46002949D041F64E
:10DDE0009C006FF4E17EA3F1E10C744D8445734413
:10DDF00041F2D86015F806E002D8E42A00F3108258
:10DE0000834230D843F2D450A2F5E6739BB28342EA
:10DE10008CBF00230123BEF1000F00F0158243B335
:10DE20004FF00000654A5AF826309055B20019921A
:10DE300033BB0F22614BC8F800209B5D002B00F024
:10DE400091810A2324AAC8F8003030464B46F9F7DE
:10DE50001DFF08BB39780246CDF8009024AB304650
:10DE6000F9F70CFD18E0BEF1000F02D10123534A6F
:10DE700093555AF82630B20019920BB90029D8D11F
:10DE8000D8F800300E2B00F36D814B4624AA3046A3
:10DE9000F9F7FCFE0028DDD0149D217822AB009517
:10DEA00000223046F9F7EAFC1B9DDFF81CC12C4626
:10DEB000BCE80F000FC4BCE80F000FC4BCE80F00A3
:10DEC0000FC49CE80F0084E80F0058F8040BD9F841
:10DED000003055F82040249DC0F10F0103FB01F3F1
:10DEE0001A95229A149D02FB04F22D6805FB043357
:10DEF0001A9D05FB0122214492FBF1F293FBF1F301
:10DF0000139C17F8011B2280129A1380002900F03D
:10DF10003081179B022B00F35B81284B9B5D002B0C
:10DF200040F03B811D9B002B40F03282179B022B5F
:10DF300040F04581199B4AF80310002E00F02B8118
:10DF40000225159B1B9C5F19169B5E19DDF8CC34CE
:10DF500003F1010837F9020F36F902CF18F8011F53
:10DF60004B4600940022C9F80000C4F800C02846BF
:10DF7000F9F784FC0135D9F8002023680A2D3A808E
:10DF80003380E7D1179B002B40F3628100252822C4
:10DF9000002148460BF0B5FEDDF8E0242560AA42DA
:10DFA00053DDCDF848904FF4737A2B46DDF8D494C6
:10DFB00011E000BF542800206828002040280020DD
:10DFC0009028002048280020289F01002368013362
:10DFD0009342236036DADDF8CC14CB5C002BF5D00D
:10DFE000012600274FF00408BB4B32463146CDE9ED
:10DFF0000273019623466D20CDE904BACDF8008066
:10E00000F4F722FB40F2CD30236831460096B34E40
:10E010004246059009EB83036D20CDE90177CDF8E9
:10E0200010B00396F4F710FB2368DDF8E02459F8EC
:10E03000231012980133934240F82510236005F114
:10E040000105C8DBDDF84890EDB24FF47573012788
:10E0500000269DF87C20CDE904B3A14B9DF85C001F
:10E0600003938DF891209DF880309DF884203946E7
:10E07000CDE9016600978DF890308DF8922024ABA1
:10E0800004228DF893006D20F4F7DEFA40F2D530CB
:10E09000944A3946CDE901660097DDF804350590CC
:10E0A00003926D209A22CDF810B0F4F7CDFA40F229
:10E0B000D73102228C4BCDE90176CDE904B1009233
:10E0C00003932022DDF8D8340F216D20F4F7BCFA39
:10E0D0004FF47672854BCDE9016600970393059264
:10E0E000DDF8DC3420220F216D20CDF810B0F4F7DC
:10E0F000ABFA31463E220DF5C9700BF002FE202727
:10E1000042F20F0C8226DDF8D834214600932A46CD
:10E110004B460320A4F800C0A7706671FCF718F8FE
:10E120001C9B159C5A792046CDE90152169DDDF8BD
:10E13000CC24DDF8C83400922946189AF8F72AFF53
:10E14000DDF8CC2429462046FCF7EEF8DDF8CC3487
:10E150002A4621460A20F8F791FE1E980DF2A44D9A
:10E16000BDE8F08F4B4624AA00213046F9F78EFD1A
:10E1700092E61D9B0BB10E2811DD199A179B4AF8E8
:10E180000210002B7FF4D9AE48F8043C4AF8023064
:10E19000002E7FF4D5AE01260FE60E2866DC013096
:10E1A00048F8040C0029E8D0179B012B3FF7C2AEBA
:10E1B0004F4B9B5D002BE0D11D9B002BDDD158F810
:10E1C000043C002BC4BF03F1FF3348F8043CD4E700
:10E1D0000E283FF7AFAE013048F8040C0029E3D118
:10E1E000CBE70DF58C7ACEAD3C22214650461295F8
:10E1F0000BF087FD30AB2846782221461E4613934C
:10E200000BF07FFD25AB1D4630461E22214617939D
:10E210000BF077FD1E942C606C602C81FFF783BAA5
:10E22000834217D843F2D450A2F5E6739BB28342DF
:10E230008CBF00230123BEF1000F7FF4F0AD43F645
:10E24000870082427FF715AE012229488255E6E514
:10E25000002565E7BEF1000F7FF40BAE43F68703A0
:10E260009A427FF706AE0123AB5502E6179B022BBD
:10E270003FF460AE81E755AA1492FFF74BBB002331
:10E280002093FFF776BA00232193FFF704BB524691
:10E290001499DDF8E0040DF1E009F9F75BFC4F4655
:10E2A000DFF850C00646BCE80F000FC7BCE80F00FF
:10E2B0000FC7BCE80F000FC79CE8030087E8030006
:10E2C00064AC26B14846FCF75BFBFFF7D1BB2846A0
:10E2D000FCF756FBFFF7CCBBA4B80100A8B80100BF
:10E2E000BCB80100C0B80100C0B4010028B80100EA
:10E2F00040280020689F010052461499DDF8E00490
:10E30000F9F728FC21462422064665A80BF0F9FC03
:10E31000072064AC20604FF0140020824FF0D20040
:10E3200060824FF01E00A0824FF0FA00E0824FF0B2
:10E3300028004FF00C0C20834FF03200A4F808C0E6
:10E34000A0830A2346204FF0640C50214FF49B72A7
:10E350004FF00F0E4FF0A0080DF1E00925464F4693
:10E36000C4E90AC0C4E90C33A4F80CE0A4F80E8098
:10E37000E18061816283E2830FCD0FC70FCD0FC7AC
:10E380000FCD0FC795E80300034D87E8030098E71A
:10E390000E287FF704AF07E794C801002DE9F04F7E
:10E3A000C7B2C0F3072883B0474501900C992BDC16
:10E3B0009DF806A052000AF100499DF807B009F146
:10E3C000FF390AFB023301EB490901EB4B0C0D99B4
:10E3D00008F1010801EB470EDA4518D849461C46FA
:10E3E0000C4D34F9170031F9026F8542B8BF05466C
:10E3F0008642B8BF08808C451444F2D12DB2013753
:10E4000047452EF8025BE7D103B0BDE8F08F014D20
:10E41000F5E700BF0080FFFF2DE9F04F05468FB004
:10E420004FEA410A08AF18467A60884652460021F2
:10E430006C00BB60D7F844900BF063FC2246386C4C
:10E4400000210BF05EFC002D64DD0AF108033E6C38
:10E4500023F0070B4FEAA8033B617B683119F96091
:10E460009C1EC7F814D0ADEB0B0D08ABA51C1846CD
:10E47000294652460BF03AFC396902464046FEF7FF
:10E48000C9FBB8F1000F014650DD002022460346CB
:10E4900032F902CF8C4508BF184601339845F7D1B1
:10E4A0000522ADEB0B0D152340F23E6C4FF0290E0B
:10E4B00007926FF42472009508ADCDE901530692DE
:10E4C000CDE903E3A1F11E02CDF814C03C3143466F
:10E4D000FEF788FDBA68023D0AEB040134F9023FF9
:10E4E00035F9020F1B1AA3EB0903002B238006DD6D
:10E4F00010889BB2184410803088034433808C42CB
:10E5000002F10202EAD1FB6802369E42D7F814D02B
:10E510000C46A6D100237A68C8EBC8084FEA480821
:10E520001C3722F80830BD46BDE8F08F6FF4247226
:10E530004FF0050E152340F23E6C2920ADEB0B0D7C
:10E54000CDE9062E08AA0390019204930293A1F14B
:10E550001E0200953C31CDF814C043460020FEF762
:10E5600041FD04EB0A01CEE72DE9F04F9FB08A0090
:10E5700008AF7A61083222F00702ADEB020DB861F4
:10E580004E0008A800297963B860FE6119DD4FF4D8
:10E59000004E47F6FF7C0025B11ED7F884200144C9
:10E5A000D7F88C00023A96190DF11E04023822F8B1
:10E5B000025FB24221F802EF20F8025F24F802CF96
:10E5C000F5D1B969786B4A0000FB02F2083222F0FB
:10E5D0000702ADEB020D08AA00297A6040F3E38040
:10E5E0007A6400223A6300EBD07222F00102043B0D
:10E5F0000A32D7F88010BB6322F007033B617B69C6
:10E600000439CB18F9603B653B69C7F82CD0ADEBFA
:10E61000030D08AAADEB030D08ABBB647B6BFA647A
:10E62000002B40F33981D7F890200023013A14469B
:10E6300047F6FF797A629046D7F88C209A46951E65
:10E640007A6CC7E90F33CB46FE68D7F838E0A2F101
:10E65000020C3C620BE0FC6C4A4524F8130002DA21
:10E6600001468146FB633A6D0133964221D056F84C
:10E67000040F5EF8042F35F8021FC2EBA0121144FC
:10E68000298018F8014F10B2E4072CF8020F494610
:10E69000C7F854B0DFD4BC6C5A4524F81A0003DA2A
:10E6A00083467865C7F840A03A6D0AF1010A9642A0
:10E6B000DDD1C7F828A015254FF0000B05266FF413
:10E6C000247840F23E694FF0290AFA6C3C6A0092C5
:10E6D000F86B6431CDE9066B0395CDE9015A4FF033
:10E6E0000042CDE90498FEF773FDCDE902A5CDE91E
:10E6F000066BCDE904980195BE6C4FF00042009680
:10E70000796DBB6A6431386CFEF762FD796B7B6AA8
:10E71000FD6C0B44594618467B6C14F8012F0233EC
:10E72000D2074BBF35F81B2036F811200BF1010B37
:10E730000131844223F8022CEFD17A6CF9693B6BEA
:10E740000A447A647969BA6B01330A44BA63BA69D4
:10E750003B639A42D7F82CD07FF456AFD7E90C89A7
:10E760007A68FB69A2F1020CBA6800269E469246BE
:10E770009D1E1544B9F1000F11DD29466046AAF12E
:10E78000020230F9023F31F9024F9C42B8BF0B80C0
:10E7900032F9024F9C42C8BF1380AA42F1D1013620
:10E7A0004645F444E6D17B6B002B71DDBB68D7F89E
:10E7B00088109C1E2646FA69881ED7F88C10A2F194
:10E7C000020CD7F81880023903EB0C0500EB020E9F
:10E7D00035F8023F36F8022F9B1A20F8023F31F934
:10E7E000023F704593FBF8F30B80F1D1D7F88430EA
:10E7F000991E0A46BB6803EB0C0534F9023F32F957
:10E80000020F002BB8BF5B42984200DA1380A5428A
:10E81000F3D1BB68084663449C46FB690B441A4627
:10E820003CF9023F30F9024F002BB8BF5B429C42DB
:10E83000B8BF03809042F3D16FF00044D7F8903016
:10E840002646581E7B6B03449C46034604E09442D4
:10E85000A8BF14469C450AD013F8015F31F9022F76
:10E86000ED07F4D49642A8BF16469C45F4D1D7F8DC
:10E87000842010F8015F118815F0010FA1EB040549
:10E880000ABF891B15801180834202F10202F0D178
:10E890005C37BD46BDE8F08F0024152505266FF4D2
:10E8A000247840F23E694FF0290AFB6C2046009321
:10E8B00007942346CDE90586CDE90359CDE9015AF0
:10E8C0004FF0004248F26301FEF782FCCDE9066496
:10E8D000CDE90498CDE902A50195BB6C20460093D3
:10E8E0004FF00042234648F26301FEF771FC24E733
:10E8F000002824DDF0B400258E1EAC464FF0FF3713
:10E9000000E01D4636F9024F6B1C944203DD64455E
:10E91000C4BFA4462F469842F3D17B1C11D07B0084
:10E9200031F917001FB1CA1832F9022C1044AF4256
:10E9300003DA1944B1F902301844F0BC70470020E2
:10E9400070470020F0BC704770B40024061E1C60A5
:10E9500020460EDD023901EB460631F9024F9442A2
:10E9600002DD1D6801351D60A042B8BF2046B142DE
:10E97000F3D170BC704700BF2DE9F04F82461646B8
:10E98000524600258BB000AF8846386D52000021FA
:10E990003C6E9946BB61C7F808A00BF0B2F90AEBD0
:10E9A000DA7323F001030A3323F00703ADEB030D01
:10E9B000C7F820D0AA45ADEB030D2561C7F81CD0E0
:10E9C00025606560A560E56084F811A0257440F3BA
:10E9D000F980504647F6FF7E7A6DCC46013A7A6060
:10E9E0009246321F02EB80037B613B6DAB46714662
:10E9F000A8F10408A3F102097D623C6611E07345A9
:10EA0000A8BF7346D7E9084524F81500A8BF1846E3
:10EA10007C6A86467869013490427C620CF1010C74
:10EA200031D0B86952F8043F20B19CF8000000FBD7
:10EA30000333DB1158F8040FBD6DC3EBA01347F689
:10EA4000FF708342A8BF034661480E468342B8BFA9
:10EA5000034618B229F8020F1AF8014F2C57002C60
:10EA6000CDD18B42A8BF0B46FC691E4624F81B0083
:10EA7000A8BF184601467869734690420BF1010B16
:10EA80000CF1010CCDD1D7E918429342A8BF13462F
:10EA90009642A8BF16461BB2524236B29342B8BF46
:10EAA00013469642B8BF164632464FF0000C4FF060
:10EAB0000040FE60FE6D7968D6E900E9BE683B6102
:10EAC0000E44B346B7F9106012B27E61E0464E467E
:10EAD00063466FF00045BA617862D7F8509041E024
:10EAE0003A6A786932F91820002A5ADB002802DBDA
:10EAF0003869121A12B229F8132008F10108724578
:10EB000018DDB4F808A022680AF1010AA4F808A0E8
:10EB100039F913A094F91100AAEB0E0A52442260AD
:10EB200094F910209842C8BF63749A42B8BF237406
:10EB300039F9132096420ADD6289606801326281E8
:10EB400039F91320A2EB060A8244C4F804A0786ABB
:10EB500001339042B8BF10469542A8BF15468B4579
:10EB6000786227D011F8012FB86D8256002AB7D1EC
:10EB7000FA69B86932F91C20002A09DB002802DB97
:10EB8000F868121A12B229F813200CF1010CB6E73A
:10EB90000028F5DA121A02EAE27212B229F81320FA
:10EBA000F3E70028A4DA121A02EAE27212B229F894
:10EBB0001320A2E72DB203B22C37A381E581BD4615
:10EBC000BDE8F08F2B464FF000404FF0FF35F3E7E4
:10EBD0000080FFFF2DE9F04786B08246DDE91298FC
:10EBE00016461C460D46149FF3F7F4F91423159AA4
:10EBF0000397CDE90423D0F801300F98153332463E
:10EC00002946CDE9010300940E9B5046FFF7B4FE60
:10EC100000254FF02E0C012102271848184E2346DC
:10EC2000CDE9030652466920CDF814C0CDE901159F
:10EC30000097F3F709FDAA4528460FDDA31E03EB55
:10EC40004A0A33F9021FA1EB0902002AC8BFAD1816
:10EC5000B1EB080148BF40185345F2D1109BAB42BD
:10EC600007DB119B8342D4BF0020012006B0BDE822
:10EC7000F087012006B0BDE8F08700BFC0B40100F6
:10EC8000D8B80100002820DDF0B48E1E06EB400647
:10EC9000B14218D0571C38460B46B1F9004033F941
:10ECA000025FAC4207DD0D801C8092F9004090F9B4
:10ECB000005015700470B34200F10100EDD1023133
:10ECC000B1423A46E6D1F0BC704770472DE9F04FAB
:10ECD0008046450005F1080485B000EBD07A24F0A9
:10ECE000070407302AF0010A00AF20F00700ADEB5F
:10ECF000040D08F1090424F00704EB46ADEB000D08
:10ED00000AF10A0020F007006E46ADEB040D6C46D8
:10ED1000ADEB000DE946C7E902210AF1020A08F14C
:10ED200002021F2120467B600AF0EBFF5246484654
:10ED300000210AF0E6FFB8F1000F7B6807DD3246DC
:10ED400006EB0800911B02F8011B8242FAD14FF03A
:10ED5000FF3A2A46F96858467B600AF0C7FF5946D1
:10ED600032464046FFF78EFF023D08F1FF3E7B68CA
:10ED700006EB0E01AB44013EB14218D03BF90259FB
:10ED800011F901299D4202F1010C10DBA05C224423
:10ED90001F28927860D01E2860D81E2A96BF4FF098
:10EDA000FF3204F80C0004F80C20B142E6D1B8F1AF
:10EDB000020F04F1010113DD0B46FF20A64402E01F
:10EDC000013373450CD05A781F2AF9D11A781E2ABC
:10EDD000F6D89A7801331E2A98BF18707345F2D17D
:10EDE000B8F1000F2EDDFB6804EB0806F96004E0C3
:10EDF0000134A64203F1020323D06278FF2AF7D13F
:10EE0000257894F802C039F8150039F81CE08346DB
:10EE1000704528BFF346B3F90020B96B0A44934507
:10EE2000E6DA704538BF7046013465458CBF29F875
:10EE30001C0029F81500A6420AF1FF3A03F102036B
:10EE4000DBD1F9684246B8680AF050FF0AF10100C8
:10EE50001437BD46BDE8F08F1F2A06D01E2A88BF92
:10EE60006FF0690204F80C2086E70AF1010A04F841
:10EE70000CA029F81A507FE7FFF728BF0048704719
:10EE800098080020014B036020207047F8B801006B
:10EE9000014B03600F20704718B90100014B03605C
:10EEA0000F207047E8B8010030B44FF080430022D3
:10EEB0000E211F2020250F2483F8082183F80A2122
:10EEC00083F8090183F80B111A739A735873D97375
:10EED0001D725C72DA7793F8211041F0010183F81A
:10EEE000211093F8211062F3410183F8211030BC06
:10EEF000704700BF10B44FF0804485B00DF1100C86
:10EF00000CE90F00BDF800302382BDF802306382A7
:10EF1000BDF90430A382BDF90630E382BDF80830A4
:10EF20002383BDF80A306383BDF80C30A38305B09A
:10EF300010BC70474FF08043988370474FF0804378
:10EF4000988B70474FF0804383F82000704700BFD4
:10EF50000123002110B50A4A0A4C2377917210B997
:10EF60004FF08042D3704FF080430122987000210F
:10EF70001A700A2000F094F90022024B1A7710BD93
:10EF8000982800200000105001234FF080401021ED
:10EF900010B4034A034CA372436010BC1160704765
:10EFA000A40C00209828002001234FF0804010215D
:10EFB00010B4044A044C6372C0F8043110BC1160F0
:10EFC000704700BFA40C002098280020E0220021F8
:10EFD00001480AF096BE00BF800100402DE9F041D3
:10EFE00005461F4B1F4886B06A1E13F8011B83425B
:10EFF00002F8011FF9D101242B464FF0A90C00277C
:10F0000002262868184AC11782FB00E2DFF86480F4
:10F0100002441648C1EB222243F8242B2146CDF8A6
:10F0200014C02246CDE90308CDE9014700966220CD
:10F03000F3F70AFB4FF0AA0C0D48CDF810800390AF
:10F04000CDE90147009605F1260322462146CDF879
:10F0500014C06220F3F7F8FA06B0BDE8F08100BFF3
:10F0600028000040540000408988888898DE01000C
:10F070002CB9010028B9010070B5E0220646002134
:10F080000B480AF03EFE002401234FF08042094D58
:10F0900009492B770A208C7293702146137000F077
:10F0A000FFF82C773046BDE87040FFF797BF00BFF0
:10F0B00080010040000010509828002010B5044640
:10F0C000FFF78CFF2E234FF0804004F14E0203F136
:10F0D000600150F82110013B1F2B22F8021DF6D1D0
:10F0E0004FF0804004F1960203F1600150F82110C6
:10F0F000013B22F8021D591CF6D110BD4FF0804291
:10F1000070B5037909B201FB03F1948B8B11A34213
:10F11000B8BF234601250024022106889BB2438004
:10F12000A2F80C61A2F80E31074E084B3577092082
:10F130005C7282F8035182F802112146A2F8005154
:10F1400000F0AEF8347770BD000010509828002011
:10F150004FF0804393F81401704700BF4FF0804395
:10F1600093F81701704700BF0023094A82F8323034
:10F170005064916472B6012382F8403000BFB2F847
:10F1800052309BB2002BFAD062B6B2F850007047F2
:10F19000000010502DE9F04750221020202130248B
:10F1A0004FF0400A4FF060094FF001084FF4807EA5
:10F1B0004FF4007C4FF480674FF400660825104B35
:10F1C00083F8000383F8041383F8084383F80343A8
:10F1D00083F805A383F8092383F80A2383F80B2314
:10F1E00083F80F93C3F8008018601960C3F800E03B
:10F1F000C3F800C01F601E601D60BDE8F08700BF3F
:10F2000000E100E04FF40042034BC3F88020BFF35D
:10F210004F8FBFF36F8F704700E100E000220121A4
:10F22000034BA3F86E20A3F86A20A3F86810704778
:10F230000000105010B5174C84B094E80300029001
:10F2400002A88DF80C1000F061F800F069F8FFF7E3
:10F25000A1FF62B600F014FAA36804A840F80C3DC0
:10F2600000F008FA00F050FA00F05EF900F0C0FA81
:10F27000094B1A6922F004021A61BFF34F8F07216C
:10F28000064A82F824105A6942F010025A6104B00A
:10F2900010BD00BFA09F010000ED00E00000105075
:10F2A00008B500BF72B6084A135C3BB900BF30BF57
:10F2B00062B600BF72B6135C002BF7D00023135464
:10F2C00001B1884762B608BD9828002000200A4B8B
:10F2D0000A4913F8012B10448B42C0B2F9D1064BF6
:10F2E0001A78AA2A01D000207047DB7B181AB0FADE
:10F2F00080F04009704700BF800040008F00400050
:10F300004FF0A04301225A74704700BF0246034BDE
:10F310000068127918601A71704700BFA828002091
:10F3200070B5FFF7D3FF01220021334BD9705A7219
:10F33000DA7200285CD0314AD278D2B21A72002236
:10F3400001242F492C4B8D789A725A731D734D7876
:10F350000E781E751D77CD78097983F8215083F8D2
:10F3600020105A749A741C749A7018B3234A5178F6
:10F370001A78C9B2D2B28A4208D08A42B4BF0132E6
:10F3800002F1FF32D0B28A421870F6D11B4B1A49F3
:10F390001A794B78D2B2DBB29A420AD09A4203F180
:10F3A000010096BF03F1FF33C3B2DBB29A424B7048
:10F3B000F4D170BD1A78D2B2B02A08D0AF2AD4BF27
:10F3C000013202F1FF32D1B2B02A1970F6D10A4AE5
:10F3D0005378DBB2082BECD0072B03F101018ABF75
:10F3E00003F1FF33CBB2DBB2082B5370F4D1E0E76B
:10F3F000E0221A72A3E700BF000010508000400016
:10F40000A828002007490B78DBB2834208D0984235
:10F41000CCBF013303F1FF33DAB283420A70F6D175
:10F42000704700BF0000105008B5FFF74FFF18B13C
:10F43000024B5878C0B208BDB02008BD8000400023
:10F44000014B1878704700BF00001050084A5378ED
:10F45000DBB283420AD0984203F1010196BF03F167
:10F46000FF33CBB2DBB283425370F4D1704700BF9D
:10F4700000001050014B5878704700BF000010503A
:10F4800010B50446FFF73CFF4FF0A04320686168C9
:10F49000A26807C310BD00BF38B54FF0A044E37D9C
:10F4A000DBB2042B28D0082B19D0022B09D0012362
:10F4B000184A137000BF4FF0A042137300BF53737C
:10F4C00038BD154D15496079FAF756FB6179286802
:10F4D000FAF79AFB62792B6813442B60E7E7104B2D
:10F4E000D0E9051259609A60236A5BBA0A4A184645
:10F4F0001360FAF70BFBDAE7074D0A492079FAF7B0
:10F5000019FB21792868FAF753FB22792B681344F9
:10F510002B60CCE798280020B02800202000005065
:10F520004C21002024000050274B0022D3F88010EB
:10F5300041F00101C3F88010196C21F00101196438
:10F54000196841F001011960D3F8801021F002011F
:10F55000C3F88010196C21F002011964196841F098
:10F5600002011960D3F8801041F01001C3F8801037
:10F57000196C41F010011964196841F0100119600B
:10F58000D3F8801021F02001C3F88010196C21F00D
:10F5900020011964196841F020011960D3F8801026
:10F5A00021F04001C3F88010196C21F0400119646A
:10F5B000196841F040011960C3F80821C3F804211B
:10F5C000C3F80021704700BF00000250034BD3F87E
:10F5D000C03018420CBF01200020704700000250CC
:10F5E00038B54FF040540125642084F8245000F0D1
:10F5F000D1F900F07FF900234FF47A7084F82530B8
:10F6000084F8815000F0C6F9BDE8384000F072B9C6
:10F6100010B501234FF04054642084F8253000F0E9
:10F62000B9F900F067F9002384F8243084F88130B8
:10F6300010BD00BF14200122002130B50A4D89B051
:10F640002D780A4C05900A4808AB03F8015DCDE916
:10F650000111CDE90304009211466420F2F7F4FF92
:10F660009DF81F0009B030BDB700400040B901004F
:10F6700048B901000268014B1A607047B4280020A5
:10F6800038B5FFF723FE0F23F0B94FF040524FF08B
:10F690000104D9B2013B072B82F82B1082F82840D5
:10F6A00082F82800F5D1042382F82F304FF0405320
:10F6B0000121002283F8281083F828204FF47A7063
:10F6C000BDE8384000F0F6B94FF040510125002464
:10F6D0000C4806E081F82B20013B81F8285081F886
:10F6E0002840027A0E2A8EBF0F22027AD2B29342AB
:10F6F000DAB2EFDA4FF04052024B5B7ADBB282F8BB
:10F700002F30D3E780004000F8B5FFF7DFFD4FF062
:10F71000405401250026074684F825604FF47A708E
:10F7200084F8205084F8275000F0C4F9642084F84D
:10F73000255000F0BFF984F82450642000F0BAF995
:10F7400084F8256007BB06231C4D84F82730EB782E
:10F7500084F826302B7884F842304FF0405401234F
:10F760000022697840F24C4084F8461084F8442026
:10F7700084F8453084F8413084F8403000F09AF93C
:10F78000AB7884F84430F8BDFFF754FF0C4B9B7AFC
:10F7900088B94FF04052DBB2084D84F82730E97841
:10F7A000074B82F82610DB7A29780B440B3BDBB23F
:10F7B00082F84230D1E7053BEBE700BFB4280020D8
:10F7C0008000400020B9064A064B10601860704760
:10F7D00003490548034B054A08601A60704700BF9B
:10F7E000BC280020B8280020E1F5000011F6000038
:10F7F0004FF04053F0B40624012200250A26FF20D2
:10F8000083F8D64093F8D7100F2764F3030183F8E9
:10F81000D710042183F8D86083F8402183F8D00002
:10F8200083F87F5093F88C004FF0050C104383F859
:10F830008C0093F88C00072640F0020083F88C00BF
:10F8400093F8910064F30300032483F8910083F894
:10F85000901083F88D1083F8A02093F8A10065F331
:10F86000010083F8A10083F8947093F88800104396
:10F8700083F8880093F88900104383F8890083F89F
:10F88000F12083F8874083F88E4083F8D22083F8F4
:10F89000D52083F8ABC083F8AD5083F8AC4083F833
:10F8A000AE1083F8AF1093F88B1041F0700183F81D
:10F8B0008B1083F8936083F8B020F0BC704700BFD2
:10F8C00000220521034B04481A6058609A601960B1
:10F8D000704700BF10E000E0FFFF0F000022044B64
:10F8E00098681A60C0F57F2000F6FF70704700BF6F
:10F8F00010E000E0002382B000280193B8BF073079
:10F90000019BC010984206DD00BF019B01330193AB
:10F91000019B8342F8DB02B0704700BF054A0649ED
:10F92000937CD27801335B00934000FB03F091FBA2
:10F93000F0F070470000105000B4C404054A937AF8
:10F94000D27ADBB20AB101339840034B93FBF0F05B
:10F95000704700BF0000105040420F00054A937AE4
:10F96000D27ADBB22AB10122134402FA03F390FBEC
:10F97000F3F0704700001050054A00EB8000937CC4
:10F98000D27801335B009340000190FBF3F07047A5
:10F9900000001050124B00EB80001B7B0001DBB21B
:10F9A0005A1E062A0DD9082B12D0092B15D0A3F107
:10F9B0000B02032A0ED90F2B0CBF01234FF0FF338C
:10F9C00000E00133064AD278934090FBF3F0704791
:10F9D0000A23F7E7063B9B00F4E70C23F2E700BF9E
:10F9E00000001050034B044A5B7C03F0010352F803
:10F9F000233018470000105054B90100034B044A4B
:10FA00005B7C03F0010352F82330184700001050CC
:10FA10004CB9010008B5044B1868FFF7EFFFBDE8CB
:10FA2000084000F0A1B800BFC428002038B50C4B36
:10FA3000054693FBF1F00C46FFF7ACFF3A2303FBBE
:10FA400004F39B1103FB00F090FBF5F0834203DB12
:10FA5000462404FB00F4A411024B1C6038BD00BF17
:10FA600040420F00C428002070B501220024452127
:10FA7000042688B008AB43F8040D0B4D0B48CDE9C4
:10FA800001240591CDE90305114600966420F2F7A3
:10FA9000DBFD074B07985C7100F042F8214605201A
:10FAA000FFF7FEFB08B070BD5CB9010064B901004E
:10FAB0009828002008B5FFF795FFBDE80840FFF73C
:10FAC000D3BF00BF08B5044B1860FFF797FFBDE830
:10FAD000084000F00DB800BFC4280020002000F04E
:10FAE00049B800BF012000F045B800BF00F030B8B1
:10FAF000012830B44FF000024FF0020438BF01205B
:10FB00000121054B054D1A702A719C709860DA60CE
:10FB10005A70197030BC70470000085098280020B7
:10FB200001284FF000024FF0010138BF012010B44E
:10FB3000054B064C1A70627199709860DA605A70C1
:10FB4000197010BC704700BF0000095098280020B1
:10FB5000012000220249034B08711A70704700BF50
:10FB60009828002000000850014B9860704700BFA3
:10FB70000000085010B40B4A0B4983B0CDE90012C5
:10FB800002AB03EB800353F8082C9378DBB2012B14
:10FB900004D10021054C04302354117003B010BC73
:10FBA000704700BF0000095000000850982800204E
:10FBB000034AD2F8803023F00103C2F88030704746
:10FBC00000000250034AD2F8803043F00103C2F82B
:10FBD0008030704700000250034BD3F88000C043D0
:10FBE00000F00100704700BF00000250002822DD35
:10FBF000F0B5DCF80460002496F80EE00CE0DCF8C8
:10FC000000703F5D07FB033305FB03F35B1242F813
:10FC100024300134A0420DD051F8043B356ABEF1C6
:10FC2000000FECD103FB05F39B1042F824300134A4
:10FC3000A042F1D1F0BD7047002822DDF0B5DCF81C
:10FC40000460002496F80EE00CE0DCF800703F5DE4
:10FC500007FB033305FB03F35B1242F82430013446
:10FC6000A0420DD051F8043B356ABEF1000FECD133
:10FC700003FB05F39B1042F824300134A042F1D17C
:10FC8000F0BD7047002822DDF0B5DCF804600024E8
:10FC900096F80EE00CE0DCF800703F5D07FB0333E4
:10FCA00005FB03F35B1242F824300134A0420DD06F
:10FCB00051F8043B356ABEF1000FECD103FB05F3AC
:10FCC0009B1042F824300134A042F1D1F0BD7047BE
:10FCD000002822DDF0B5DCF80460002496F80EE080
:10FCE0000CE0DCF800703F5D07FB033305FB03F31A
:10FCF0005B1242F824300134A0420DD051F8043B8D
:10FD0000356ABEF1000FECD103FB05F39B1042F8FE
:10FD100024300134A042F1D1F0BD7047DCF8083046
:10FD2000F0B49C7BBCB9002813DDDCF80430D3F8B8
:10FD30000D301B681E89DD8851F8043B013403FB3C
:10FD400006F393FBF5F3A0424FEA831342F8043B1A
:10FD5000F2D1F0BC70470028FBDDDCE90043D3F8AA
:10FD60000D30013C1B6820441F89DE8814F8015FB8
:10FD700051F8043BA04205FB033307FB03F393FB5D
:10FD8000F6F34FEA630342F8043BEFD1F0BC70474F
:10FD9000704700BF00280BDD10B4002451F8043B6D
:10FDA00001349B01A04242F8043BF7D110BC7047DC
:10FDB000704700BF00232DE9F041DCF80C5088B0FB
:10FDC0000793D5F809200028644617680EDDDCF893
:10FDD0000820D2681618013E013A12F8011F795C1A
:10FDE00096420B440793F8D193FBF0F360680793B6
:10FDF0004288002A53D00689921B11029B1B91FB5B
:10FE0000F3F3B3F5DC7FA8BF4FF4DC730362D5F8DE
:10FE10000D504FF0020E2989002603FB01F3191241
:10FE2000FF29A8BFFF2101224FF0AB081E4FDFF8CA
:10FE300084C0698100EB0E03CDF800E0CDE903C773
:10FE40001146CDF81480CDE901666420F2F7FCFB81
:10FE500001254FF00408AC22144B059229462A468E
:10FE60000393049707AB02960195CDF800806420B8
:10FE7000F2F7EAFB4FF0AD0C63680D48049703906E
:10FE8000CDE90156CDF8008020332A462946CDF829
:10FE900014C06420F2F7D8FB08B0BDE8F0814FF43D
:10FEA00080730362B3E700BF68B9010090B9010035
:10FEB00098B9010074B9010000232DE9F041DCF884
:10FEC0000C5088B00793D5F80920002864461768BD
:10FED0000EDDDCF80820D2681618013E013A12F84F
:10FEE000011F795C96420B440793F8D193FBF0F322
:10FEF00060680793C288002A52D08688921B11023C
:10FF00009B1B91FBF3F3B3F5DC7FA8BF4FF4DC73CD
:10FF10000362D5F80D504FF0020E2989002603FB2D
:10FF200001F31912FF29A8BFFF2101224FF0F408A5
:10FF30001D4FDFF880C06981831DCDF800E0CDE959
:10FF400003C71146CDF81480CDE901666420F2F7AD
:10FF50007BFB01254FF00408F522144B059229463E
:10FF60002A460393049707AB02960195CDF80080CB
:10FF70006420F2F769FB4FF0F60C63680C480497B5
:10FF80000390CDE90156CDF8008020332A4629465A
:10FF9000CDF814C06420F2F757FB08B0BDE8F0813B
:10FFA0004FF480730362B4E768B9010090B90100AF
:10FFB00098B90100A4B9010000232DE9F041DCF853
:10FFC0000C5088B00793D5F80920002864461768BC
:10FFD0000EDDDCF80820D2681618013E013A12F84E
:10FFE000011F795C96420B440793F8D193FBF0F321
:10FFF000606807934288002A54D00689921B110238
:020000021000EC
:100000009B1B91FBF3F3B3F5DC7FA8BF4FF4DC73CC
:100010000362D5F80D504FF0020E2989002603FB2C
:1000200001F31912FF29A8BFFF2101224FF4C5785F
:100030001E4FDFF884C0698100EB0E03CDF800E0AD
:10004000CDE903C71146CDF81480CDE901666420DF
:10005000F2F7FAFA01254FF0040840F28B12144B24
:10006000059229462A460393049707AB0296019509
:10007000CDF800806420F2F7E7FA4FF4C67C63689D
:100080000C4804970390CDE90156CDF80080203349
:100090002A462946CDF814C06420F2F7D5FA08B0F4
:1000A000BDE8F0814FF480730362B2E768B90100E4
:1000B00090B9010098B9010074B9010000232DE93D
:1000C000F041DCF80C5088B00793D5F809200028DF
:1000D000644617680EDDDCF80820D2681618013E69
:1000E000013A12F8011F795C96420B440793F8D14C
:1000F00093FBF0F360680793C288002A53D0868888
:10010000921B11029B1B91FBF3F3B3F5DC7FA8BF9D
:100110004FF4DC730362D5F80D504FF0020E2989BD
:10012000002603FB01F31912FF29A8BFFF210122BA
:1001300040F2D3181E4FDFF884C06981831DCDF8CB
:1001400000E0CDE903C71146CDF81480CDE9016682
:100150006420F2F779FA01254FF004084FF4EA72AF
:10016000144B059229462A460393049707AB02963F
:100170000195CDF800806420F2F766FA40F2D51CB4
:1001800063680D4804970390CDE90156CDF80080CF
:1001900020332A462946CDF814C06420F2F754FAD9
:1001A00008B0BDE8F0814FF480730362B3E700BF8D
:1001B00068B9010090B9010098B90100A4B9010023
:1001C00000232DE9F0411C46DCF80C2088B0D2F861
:1001D00009206646D76801F5F06501F5006C0793C4
:1001E000043F57F8041FA5F5F062890952F8803BD7
:1001F0005B1A95421C44F9D10435AC450794F0D103
:1002000094FBF0F4B36807945A88002A54D0998874
:10021000521A1202641A92FBF4F4B4F5DC7FA8BF00
:100220004FF4DC741C62726840F23A2ED2F80D2052
:100230004FF0020C10680025C188012204FB01F474
:100240002112FF29A8BFFF211D4F1E4C01816344CD
:10025000CDF814E0CDF800C01146CDE90347CDE953
:1002600001556420F2F7F0F901244FF0040840F240
:100270003B22154B0592214622460393049707AB78
:1002800002950194CDF800806420F2F7DDF94FF477
:100290000F7CB3680D4804970390CDE90145CDF874
:1002A0000080203322462146CDF814C06420F2F7A6
:1002B000CBF908B0BDE8F0814FF480741C62B2E75E
:1002C00068B90100C0B90100E4B90100F0B901004A
:1002D00030B595B0202200210CA809F012FD294C60
:1002E00029492A4D2A48CDE90854CDE90A01294A6D
:1002F000294B0E9293F8812002AC8DF83C2093F8A4
:1003000081308DF83D30F6F78FF98DF83E00F6F725
:1003100091F98DF83F00F6F793F98DF84000F6F764
:1003200095F98DF84100F6F797F98DF84200F6F748
:1003300099F91190F6F79CF91290F6F79FF9ADF83C
:100340004C0008A8F9F7DCFAF6F798F9F9F752FF2C
:100350000023022202930120A382C4E90133C4E9ED
:1003600003338DF81D20FBF7FFFC06ABADF81E0034
:1003700093E803008DE8030094E80F00F9F76AFAA8
:1003800015B030BDC5FB0000B5FA0000B1FB0000A0
:10039000D9FB00006E0016780000105070B50023E5
:1003A00001223F2148260825022484B001A8CDE976
:1003B000013303938DF807608DF808508DF80920FC
:1003C0008DF80F208DF80A408DF80D10FFF758F8C2
:1003D00004B070BD02FB01F21212FF2AA8BFFF2277
:1003E000028070472DE9F042224E92B0224D0DACB2
:1003F00005AF99460691089296E80F0084E80F0031
:1004000018ABC4E90275204611A91193EFF738FF24
:1004100096E80F00194E09AD85E80F00C5E9027690
:1004200021462846EFF72CFF089B069A44F001046A
:100430001169D3F8012005910792D3F80D201049D6
:100440001089189E5081CDE9021445F001050196EE
:100450000495D3F8093080225B690021184609F021
:1004600050FC2022034601A94846F6F70DF912B0C8
:10047000BDE8F082AC9F0100B5FD0000EDFB00007F
:10048000995900002DE9F042224E92B0224D0DAC58
:1004900005AF99460691089296E80F0084E80F0090
:1004A00018ABC4E90275204611A91193EFF7E8FED5
:1004B00096E80F00194E09AD85E80F00C5E90276F0
:1004C00021462846EFF7DCFE089B069A44F001041B
:1004D0001169D3F8012005910792D3F80D20104936
:1004E0001089189E5081CDE9021445F0010501964E
:1004F0000495D3F809303C225B690021184609F0C5
:1005000000FC0F22034601A94846F6F7BDF812B0D9
:10051000BDE8F082AC9F0100B9FE000039FC00008C
:10052000FD5900002DE9F042224E92B0224D0DAC53
:1005300005AF99460691089296E80F0084E80F00EF
:1005400018ABC4E90275204611A91193EFF798FE84
:1005500096E80F00194E09AD85E80F00C5E902764F
:1005600021462846EFF78CFE089B069A44F00104CA
:100570001169D3F8012005910792D3F80D20104995
:100580001089189E5081CDE9021445F001050196AD
:100590000495D3F8093080225B690021184609F0E0
:1005A000B0FB2022034601A94846F6F76DF812B0C9
:1005B000BDE8F082AC9F0100B9FF000085FC00009F
:1005C000B15900002DE9F042224E92B0224D0DACFF
:1005D00005AF99460691089296E80F0084E80F004F
:1005E00018ABC4E90275204611A91193EFF748FE34
:1005F00096E80F00194E09AD85E80F00C5E90276AF
:1006000021462846EFF73CFE089B069A44F0010479
:100610001169D3F8012005910792D3F80D201049F4
:100620001089189E5081CDE9021445F0010501960C
:100630000495D3F809303C225B690021184609F083
:1006400060FB0F22034601A94846F6F71DF812B0D9
:10065000BDE8F082AC9F0100BD000100D1FC0000AC
:10066000595A00000269054B0548013A12F8011F6A
:10067000013303F8011C8342F8D170470000836006
:10068000E00183602DE9F041234E92B0234D0DAC83
:1006900005AF9846CDE90610089296E80F0084E869
:1006A0000F0018ABC4E90275204611A91193EFF7AA
:1006B000E7FD96E80F001A4E09AD85E80F00C5E981
:1006C000027621462846EFF7DBFD069B4FF4F062E9
:1006D000D3F8093000211B69124F184609F011FBAD
:1006E000DDE906210969104E0591D2F80D20034677
:1006F000126844F00104D18845F00105118140469B
:100700004FF4F07201A9CDE90345CDE90176F5F783
:10071000BBFF12B0BDE8F081AC9F0100C101010038
:100720001DFD000055420000013C000030B4D0F82F
:100730000D30D0F809001B68C068DC8801F1800525
:1007400004FB02F21212FF2AA8BFFF221A8192B202
:1007500051F8043B03FB02F393FBF4F38D4240F8A2
:10076000043BF5D130BC7047F0B50F46D0F80D30E2
:10077000D0F809201B68D468DA8885B01A81F3F7AD
:1007800069FDF3F733FA20468022002109F0B9FA17
:10079000074A0849084E094D009201912346384600
:1007A00020226946CDE90265F5F76EFF05B0F0BD80
:1007B00055420000ED3B000091FD000095FD00005A
:1007C000002825DD2DE9F0039046043982B04FEA78
:1007D000E27901EB800051F8042FD317CDE9002313
:1007E000DDE9002302FB09FCA2FB086708FB03C349
:1007F000B40B1F4444EA8744BD13CDE90045DDE94D
:10080000002388420A60E6D102B0BDE8F0037047D9
:10081000704700BFF0B5002685B0FFF759FDF5F72A
:1008200067FB1E491E4F334632460C6802200121E9
:100830000096A0473C46FFF7B1FDFEF71FFBF3F71C
:100840001BFAFEF7F7FCFEF72FFB164B164DA3F82D
:1008500068600FCD0FC40FCD0FC40FCD0FC43B6820
:100860002A680133226006D0082304A800F8043D5A
:100870000121F9F7F3FA01220A4B0C4CA3F8682086
:10088000F9F7B8FA00F06CFB2568FEF7D9FDA870FF
:100890002468FEF7EFFDE07005B0F0BDB0DF0100A9
:1008A000582100200000105000FE0100340A0020F2
:1008B0000246034B51680068926807C3704700BF47
:1008C000C82800202DE9F04F964683B0544E9DF87D
:1008D00034709DF830C09846009763460D46B6F9CF
:1008E0000620B6F90410044670469DF83870FAF7F1
:1008F000B5FF3378800290FBF8F0002B4BD0A91C99
:1009000096F801904B002A4604EB030E03F102080F
:10091000B9F1000F50D13EF8069C05F1FF3C24F8D8
:100920000890A3F108053EF8043C254424F8113052
:100930006189238961802380531ED2B31A4602F154
:10094000010B4FEA4B0104EB010A063134F8019028
:100950003AF8028C34F81B30C84407FB08F9BAF89F
:10096000048096F903B043440BFB0398BAF80230B5
:1009700096F90290624509FB03834FEAA31300FB3B
:1009800003F34FEA2343635246D0012AD4D1E388CC
:1009900000226380D3E765B1A91C04EB4101043454
:1009A00031F8022D00FB02F28C424FEA22428A808B
:1009B000F6D103B0BDE8F08F00236380238024F8D4
:1009C000113024F80830002DF3D07F0004EB4501EE
:1009D00031F802E996F90350B1F808C00B88CA88CB
:1009E0009C4538BF9C46964538BF96460CFB07F39E
:1009F0006A000EFB02338D8896F902208C4205FBBB
:100A000002324FEAA21200FB02F24FEA22420A81AE
:100A1000DED103B0BDE8F08F2B88AEF800308BE755
:100A2000C8280020F0B505462C4C426994F90330E3
:100A300094F90270C3F12003E07AC7EB4307A37A6D
:100A400085B0C7F34707CDE90107009305F12C00F6
:100A500020230E460F21FFF735FF617A237A05F137
:100A600052046A692046CDE90117009320210F2323
:100A7000FFF728FFFEF7AAFA20462E234FF0804406
:100A800003F1600230F8021D013B1F2B44F82210D5
:100A9000F6D14FF0804405F19A0232F8020D03F1CD
:100AA0006001013B44F82100591CF6D10120FEF7FA
:100AB0004FFA2846FEF792FAB4F84C301BB2336076
:100AC00094F85030337294F85130737294F8523075
:100AD000B37294F85330F37205B0F0BDC82800200B
:100AE00038B504220125144B144C1D712260FEF709
:100AF000F5FFFEF78FFFF9F77DF9837E43B9104BC1
:100B00001B682BB10F4A126812B90F4A157098472B
:100B10000E4BD3F80021120708D5002208250C48F7
:100B20000C49C3F880510270C1F840210121102303
:100B3000094AD160236038BD98280020A40C002009
:100B400098170020881C00209717002000E100E083
:100B5000A00C0020000002500000085001220521D6
:100B600038B50D4B0D4C5A712160FEF7BBFF0C4B95
:100B7000D3F80021120708D50022082509480A49A0
:100B8000C3F880510270C1F8402101211023074AA7
:100B9000D160236038BD00BF98280020A40C00203D
:100BA00000E100E0A00C002000000250000009500D
:100BB0000121032238B50B4B0B4DD9700B4C2B7810
:100BC00022601BB1FEF78AFE094B186001232B70CF
:100BD000FEF776FE00211023064AC2F8401123607A
:100BE00038BD00BF98280020A00C0020A40C0020D5
:100BF000C02800200000025001234FF06050102157
:100C000010B4034A034CE372836210BC1160704756
:100C1000A40C0020982800200F21124A124B1160CA
:100C20005B6F84B00193019B23F4FF6323F0070300
:100C30000293019B23F07F030393029BB3F5800F84
:100C40000AD0039A094B9A4206D0019A084B9A425D
:100C500002D20122074B1A700122034BA3F86C2029
:100C600004B07047A40C00200000105080FF010069
:100C700000FC0100D428002008B5FFF7CBFD00F0F0
:100C8000D5FD002008BD00BF704700BF08B54FF07C
:100C9000CD3203490348FCF7D3FA002008BD00BF5A
:100CA0005C4400205C340020704700BF08B5F1F7B9
:100CB000A5F8D0F80930986808BD00BF40F21513B8
:100CC0002DE9F0431C4A1D4D1D4C83B0126821468E
:100CD000009363202B46F1F709FDF1F78BF881466D
:100CE000F1F78CF880460027D0F80960F3F74AF94D
:100CF0004846F3F799F84046F3F796F808F0A0FF56
:100D0000F760F1F7ABF83760F1F77CF8064601467B
:100D10000120F3F779F831460220F3F775F84FF424
:100D20009770084A2B461268214600906320F1F71D
:100D3000DDFC03B0BDE8F0834C07002030BA0100B1
:100D400020BA01005007002051222DE9F041304B1C
:100D500082B000921A682F492F4B6320F1F7C6FC2E
:100D6000FEF78CF80546F1F74DF8044601462A4691
:100D70000120F2F7FBFF2A4621460220F2F7F6FF98
:100D8000F1F738F80746F1F739F8044608F042FF62
:100D9000804608F043FFC7F80D0008F043FF2946DE
:100DA000C4F80D003846D4F80960F3F765F8F3F796
:100DB0008DF829462046F3F75FF8F3F787F8F368D4
:100DC00003B33368DBB120460221FFF7CDFC39467F
:100DD000022322464046FFF755FCD8F82020F16850
:100DE0002046FFF7A3FC7A220C4B00921A680949AF
:100DF000094B6320F1F77AFC02B0BDE8F081F1F70E
:100E000023F8E0E708F012FF08F022FFF060D8E7CF
:100E10004C07002000BA010030BA01005007002042
:100E20002DE9F047A8B0F0F7E9FF064607A8D6F885
:100E30000940FEF727F8D6F80D30079A5968A368DD
:100E400009780492276818ADCDE9025708AA0192E3
:100E5000E268C5B2009208461A222946FDF784FBD3
:100E600065B1236803EB45010239023B33F9022FD8
:100E7000002AB8BF52428B421A80F7D101274FF0A7
:100E8000040AAB200621DFF880901C4AE368059035
:100E9000CDE90171CDE9032939462A46CDF800A0F4
:100EA0006220F1F7D1FB4FF00008AD20D6F80D20FD
:100EB000A3685168124A0978CDE904900392CDF8ED
:100EC00000A02A46CDE901887220F1F7BDFB022679
:100ED0004FF0AF0C0B4823682A460390CDF81090D2
:100EE000CDE901783946CDF814C000966920F1F7B4
:100EF000ABFB206828B0BDE8F08700BF14C4010038
:100F00002CC4010044C4010030BA010008B502201D
:100F1000F3F762F9BDE80840F3F7EEB930B50446DF
:100F200087B0FEF781FA8321012200230334094DA3
:100F30000444059108480949CDE90133049003911F
:100F400000922B46114664202C70F1F77DFB07B010
:100F500030BD00BF8407002030BA01003CAC010066
:100F60000148F6F711BD00BF400800202DE9F04F01
:100F70008FB006AFFEF758FA01244FF00009D222D5
:100F80000426DFF8B0C29E4D07F1200343F8140D8C
:100F900021460592CDE903C5CDE9014922460096D7
:100FA0006420F1F751FB03224FF0D40C954807F170
:100FB0002003DFF8848243F8102D21460390049526
:100FC000CDE9014900962246CDF814C06420F1F71E
:100FD0003BFBD8F80410FB68CA1D22F007023869F1
:100FE000ADEB020D034406AA49457A60FB600DDDB6
:100FF00001EBD170A3EB60031046DBB2084402F8AA
:10100000013B824203F10103DBB2F8D189000A31CE
:1010100021F00701ADEB010D0DF118094846F6F777
:10102000C5FCDF22764B0092774900226420F1F75D
:101030005DFB494607F11802D8F804000124F6F7D1
:101040003DFD00264FF0040BE422704B07F1200A0F
:10105000049521464AF8040D0592CDE90263224623
:101060006B4B6420CDE900B4F1F7EEFAE523D8F834
:1010700004200593674B2146039364207B68049505
:10108000CDE901660094F1F7DFFAE6236249D8F86A
:1010900004206420059303914B4621460495CDE935
:1010A0000146CDF800B0F1F7CFFAE82305935B4B8A
:1010B00022460393214607F1180364200495CDE9E5
:1010C0000146CDF800B0F1F7BFFAE923544A2146B2
:1010D000059303925346224664200495CDE90146C8
:1010E000CDF800B0F1F7B0FA4846F6F7C5FCEE23AC
:1010F000324600934B49424B6420F1F7F7FAD8F897
:1011000004304946023B184607F11402C7E905635B
:10111000F6F7D4FC00B10138012400264FF0040B8F
:10112000F822F861404807F118030592214622464B
:1011300003900495CDE90146CDF800B06420F1F7A5
:1011400083FAF920334BD8F8042021460393059005
:101150007B68CDE90166009404956420F1F774FA88
:10116000FA202D4BD8F804202146039305904B46D6
:10117000CDE90146CDF800B004956420F1F764FA9A
:10118000FC20264B22460393214607F114030590C9
:10119000CDE90146CDF800B004956420F1F754FA8A
:1011A000FD2040F201181E4B224603932146534670
:1011B0000590CDE90146CDF800B004956420F1F723
:1011C00043FAF969FB68194ADFF870E012680B44CA
:1011D00017485FFA83FC82F802C073460390CDE99A
:1011E000016600940495CDF81480224621466420BF
:1011F0008EF800C0F1F728FA2437BD46BDE8F08F1D
:1012000030BA01004CBA01005CBA010088BA010092
:101210004408002094BA0100A0BA01009CBA010061
:10122000ACBA0100BCBA0100F4BA0100340A0020D3
:101230003CAC010040BA01004008002084070020B7
:1012400040F2091330B50D4A0D4D0E4C83B01268B3
:101250002146009363202B46F1F748FAFFF786FEFC
:1012600040F20D10084A2B46126821460090632078
:10127000F1F73CFA002003B030BD00BF4C0700205E
:1012800030BA010010BA01005007002040F2571395
:101290002DE9F041174A184D184C82B012682146CA
:1012A000009363202B46F1F721FAF0F7A3FD804667
:1012B000F0F7F2FD0746F0F78DFE0646F2F762FE04
:1012C0004046F2F7B1FD3846F2F7AEFD3046F2F790
:1012D000ABFDF0F70BFEF0F7A7FE4FF4B670084A2F
:1012E0002B461268214600906320F1F7FFF902B007
:1012F000BDE8F0814C07002038BB0100FCBA0100BA
:1013000050070020CF222DE9F04FD44BADF66C0DE5
:1013100000921A68D249D34B6320F1F7E7F9F0F74E
:1013200069FDD0F80940F0F7B7FDD0F80930042581
:10133000079308F09FFCF0F74DFED0F8098008F005
:10134000ADFC4FF4707200213AA808F0DAFC40229C
:1013500000211AA808F0D5FC1E2200210AA808F0D6
:10136000D0FC4FF4707200210DF5956008F0C9FCB7
:10137000402200212AA808F0C4FC1E2212A8002145
:1013800008F0BFFCE268DDF81CA00992043A08925C
:101390000DF6A60919AF0DF1E606F2F75BFFF2F7BD
:1013A000ABFFDDF820C00DF2E6446046A4F1400139
:1013B00031F8022F50F8043FA14213440B80F7D1BB
:1013C00040344C450CF1800CEFD1D8F810000DF1F1
:1013D0004601043831F8022F50F8043FB942134453
:1013E0000B80F7D1DAF810300DF1A602A3F1040C4E
:1013F00032F8020F5CF8043FB24203441380F7D185
:10140000013DCAD10DF2A6400DF6660600F1400579
:1014100030F9023F002BB8BF03339B10A842038072
:10142000F6D1B042F2D10DF1460636F9023F002B5B
:10143000B8BF03339B108E423380F6D10DF1A60561
:1014400035F9023F002BB8BF03339B1095422B8028
:10145000F6D1F8F7BDFC0B28824F40F0F880F2F788
:10146000F9FEF2F749FF4FF491723B4600927E4934
:1014700000226020F1F73AF92AAB0DF59562DDF80C
:1014800020A00DF2E649A3EB020B5046A646A9F1B7
:1014900040020BEB090132F9023F50F8044F31F9D9
:1014A00002CF1B1B9C45B8BF0B809145F3D109F1BE
:1014B0004009F14574460AF1800AE6D1D8F81000D7
:1014C0000DF146020DF12601043832F9023F50F8C1
:1014D000044F31F902CF1B1B9C45B8BF0B80B242B1
:1014E000F3D1079B0DF1A60218690DF166010438CE
:1014F00032F9023F50F8044F31F902CF1B1B9C45D3
:10150000B8BF0B80AA42F3D14FF0000A4FF0040B92
:1015100040F23713554A05930392CDF800B0099B6A
:1015200020220F2172200497CDE901AA4FF0010972
:101530007446F1F789F84FF49C714D4AD8F8103091
:101540007220CDF800B0CDE90471039249460F2214
:10155000CDF808A0CDF80490F1F776F840F23910F4
:10156000079B444A1B694946CDF800B00590039299
:1015700072202022CDE9019A0497F1F765F84FF027
:10158000020B40F23B123C4BCDE904720393202244
:101590000DF595630F216220CDE9019ACDF800B0D9
:1015A000F1F752F84FF49E72344B4946059203937B
:1015B0000F2212AB6220CDE9019ACDF800B004975A
:1015C000F1F742F840F23D122D4B49460592039344
:1015D00020222AAB6220CDE9019ACDF800B0049711
:1015E000F1F732F840F23F12264BCDE90472039333
:1015F00020223AAB0F216920CDE9019ACDF800B045
:10160000F1F722F84FF4A0721F4B4946059203935D
:101610000F220AAB6920CDE9019ACDF800B00497FA
:10162000F1F712F840F24112184B4946CDE9047225
:10163000039320221AAB6920CDE9019ACDF800B0BE
:10164000F1F702F8F8F7C4FB0B283FF408AF40F2BB
:101650004F120F4B00921A681CE000BF4C0700208D
:1016600024BB010038BB0100C4B201004CBB010027
:1016700060BB010074BB010088BB010098BB010086
:10168000A0BB0100A8BB0100B8BB0100C4BB0100A6
:10169000500700200449054B6320F1F727F800208C
:1016A0000DF66C0DBDE8F08F24BB010038BB0100C6
:1016B000A6222DE9F041554B82B000921A68544998
:1016C000544B6320F1F712F8FDF7D8FB0446F0F70E
:1016D00091FB0746F0F7E0FB0546F0F77BFC06467A
:1016E00008F0C4FAC5F80D0008F0D4FAC6F80D00E9
:1016F0002046F0F7D5FB2046F0F770FC2146304637
:10170000F2F7BAFBF2F7E2FB21462846F2F7B4FB08
:10171000F2F7DCFB21463846F2F7AEFBF2F7D6FBD8
:10172000F0F768FB0446F0F7B7FB0646F0F752FC0B
:10173000054608F09FFA08F0B1FAFDF79FFB07464F
:1017400000212078F2F71EFD21463846F2F772F8A4
:10175000D4F80130DB7A1BB120782F49F2F712FD63
:10176000F2F778FDF2F7C8FD00213078F2F70AFDB4
:10177000FDF784FB294A3146F3F712FC30782849FB
:10178000F2F700FD00212878F2F7FCFCFDF776FB6C
:10179000224A2946F3F74AFF22492878F2F7F2FC59
:1017A000F0F728FB0446F0F777FB0746F0F712FC4A
:1017B000054608F02FFA804608F05CFA064608F065
:1017C0006DFAD4F80D30046A1868D8F82020C18862
:1017D0000830366AFEF7FEFDD7F80D003246018963
:1017E0000A30FEF7F7FDD5F80D00224601890A30D0
:1017F000FEF7F0FDC9220C4B00921A680449054B14
:101800006320F0F773FF02B0BDE8F0814C070020C1
:1018100010BB010038BB01003D36000055420000FE
:10182000C951000011580000500700202DE9F04771
:1018300084B0F8F7CDFA3522254B264900920546AB
:1018400000226420F0F752FFFDF7EEFD224A234B01
:1018500010701C68FDF7E8FD214EA070DFF88CA029
:101860000024DFF86C90DFF888801E4FFEB1102C4A
:101870001DD833689847AC4201D0F8F79FFA01258C
:10188000CDB94FF0CD3239461748FBF733FDF8F7A5
:101890009FFA8442F4D0B36803909847FAF7AEF900
:1018A0000398254604465AF82460002EDFD1F8F745
:1018B0008FFA0446F7E74B224B460092414600223E
:1018C0006020F0F713FF736898470546D9E700BF1B
:1018D00030BC010038BC010084070020340A00201D
:1018E000400700205C4400205C340020ECBB010079
:1018F000C4B2010084B02DE9F0438FB0BDF87AC2C4
:10190000A79DDFF8D0E005FB0CF58EFB0564EF1713
:10191000B5F5C84FC7EB64174FF00006B4BFB84623
:101920004FF0FF08A89C054604FB0CF00DF15C0C81
:10193000B0F5C84FCDE90866CDE90A668DF820807C
:10194000CDE90C668CE80E003DDA8EFB003EC41734
:10195000C4EB6E14E4B201264FF000087022DFF8E9
:1019600078901A4B059231463246CDE90339CDE9DC
:10197000018808AB009664208DF82A40F0F764FED9
:1019800004244FF0750C12480EAB43F81C7D324610
:10199000314600940390CDF81090CDE90168CDF860
:1019A00014C0642008ACF0F74FFE0FCC28606960CB
:1019B00003CC28612846AA60EB6069610FB0BDE8DE
:1019C000F04304B07047FF24C5E700BFD0BB01005F
:1019D000B0C301001F85EB5130BC0100472370B537
:1019E0000E4A0F4D0F4C82B01268214600936320BF
:1019F0002B46F0F77BFEF0F7FDF90646F2F7C2FA48
:101A00003046F2F711FA4F20074A2B46126821465A
:101A100000906320F0F76AFE02B070BD4C07002012
:101A20007CBC010060BC010050070020382370B569
:101A30000F4A104D104C82B012682146009363206B
:101A40002B46F0F753FEFDF719FA0646F0F7D2F9E8
:101A500001463046F0F796FF3F20084A2B461268B1
:101A6000214600906320F0F741FE002002B070BDD7
:101A70004C0700207CBC010044BC01005007002042
:101A8000262370B5144A154D154C82B012682146B4
:101A9000009363202B46F0F729FEFDF7EFF9064689
:101AA000F0F7A8F93146F2F7E7F9F2F70FFA08F084
:101AB000B1F80646807BFDF745FA3046FEF7D2FDC9
:101AC0003220084A2B461268214600906320F0F726
:101AD0000DFE02B070BD00BF4C0700207CBC0100B1
:101AE000F8AB0100500700204B23F0B5114A124D0E
:101AF000124C83B012682146009363202B46F0F706
:101B0000F5FDF0F777F90746F0F778F90646F2F7B2
:101B100039FA3846F2F788F93046F2F785F9552058
:101B2000074A2B461268214600906320F0F7DEFD3D
:101B300003B0F0BD4C070020C0BC0100ACBC0100EC
:101B4000500700203A23F0B5114A124D124C83B0D1
:101B500012682146009363202B46F0F7C7FDFDF77E
:101B60008DF90646F0F746F90746F0F747F939468A
:101B70003046F1F757FF4320084A2B4612682146AA
:101B800000906320F0F7B2FD002003B0F0BD00BF6D
:101B90004C070020C0BC010098BC01005007002089
:101BA00026232DE9F0411A4A1A4D1B4C82B01268C7
:101BB0002146009363202B46F0F798FDF0F71AF9C1
:101BC0008046F0F71BF90746FDF758F9064601462F
:101BD0004046F2F751F9F2F779F931463846F2F713
:101BE0004BF9F2F773F908F015F80646807BFDF71C
:101BF000A9F93046FEF736FD3420084A2B46126814
:101C0000214600906320F0F771FD02B0BDE8F0813D
